:100000000C94451B0C94851B0C94851B0C94851B30
:100010000C94851B0C94851B0C94851B0C94851BE0
:100020000C94851B0C94851B0C94851B0C94851BD0
:100030000C94851B0C94851B0C94851B0C94851BC0
:100040000C94851B0C94D3E40C94851B0C94851B99
:100050000C94851B0C9466DA0C94851B0C9427C7B2
:100060000C94851B0C9419550C94E3540C94851B2B
:100070000C94851B0C94851B0C94851B0C94851B80
:100080000C94851B0C94851B0C94851B0C94851B70
:100090000C94851B0C94851B0C94851B0C94851B60
:1000A0000C94851B0C94851B0C94851B0C94851B50
:1000B0000C94851B0C94851B0C94851B0C94851B40
:1000C0000C94851B0C94851B0C94851B0C94E227C7
:1000D0000C94AC270C94851B0C94851B0C94851BED
:1000E0000C94851B084AD73B3BCE016E84BCBFFDF8
:1000F000C12F3D6C74319ABD56833DDA3D00C77FF8
:1001000011BED9E4BB4C3E916BAAAABE0000008090
:100110003F05A84CCDB2D44EB93836A9020C50B91F
:10012000918688083CA6AAAA2ABE000000803F004B
:100130000C94BB260D94162F0D942E2F0C949555D0
:100140000C9497260D9440010C94D5550C942EBA1E
:100150000C942AB40D94E92D0C94C6A20D948E2E05
:100160000C94B7260D94F4090D94E8090D94992C7C
:100170000D94ED2E0D9452010C949EF30D942801D4
:100180000D94E5090C94BB550D944E010C9476B476
:100190000C946B260D94382F0D9439320C947C28D6
:1001A0000C9474280C94B1F30D9432010C94202813
:1001B0000D940D010C948C280D94EE090D944801BA
:1001C0000C949E280D943E2E0C9495260C944CC4B1
:1001D0000C9499F30C9404C70C94B3550D94E42E2D
:1001E0000D943E2F0C94AB550C9403270D94082FBF
:1001F0000C94E5B30C9469C40C941EB40C9457553C
:100200000D941B010C946D280D942D320D94FA0958
:100210000D945D2D0D943A010C94DB260D94232F43
:100220000D94E2090C9480280C9410A30D94EC31E9
:100230000C9418B40C94B6F30C94B9260C94DD55B8
:100240000C9402C50C945E280D94E0310D94F62EAA
:100250000D94BF2D0C94A7B40D942C010C942DB4C7
:100260000C9478280D94D02E0C94A3B40C9457BA07
:100270000C9486550D943B2F0C946CBA0D94CF3F83
:100280000C947FA30C947BA20C94C3550C9461C571
:100290000D94DB2E0C94F1C50C9498F20C94EBA207
:1002A0000C944F280C9456A20C94A4550D94213212
:1002B0000C9424B40C9477260C9421B40D94220150
:1002C0000D947C2E0D9444010C9446C50C941EC6CE
:1002D0000D94FF2E0D9410320C9431A20D94152E16
:1002E0000C94DD260C94A6280D94182F0D94CD2C7B
:1002F0000D9413010D94F7090D94DA090D94B13F93
:100300000C9430B40C9486F30C94DF260C94B755FF
:100310000D944D010D9448320C94AF550C94E1C4EA
:100320000C9435A30D94DF090D9436010C9433B46D
:100330000D9417010D94F1090C9436B40D94FD0938
:100340000C949EBA0C9488F20C9493280D945D2E14
:100350000C94EFA10C9401270C9427B40C941BB4BB
:100360000C9484280C947AF30D941F010C9458C0BB
:100370000C94DFC50C94CA550C9488280C94FF2665
:100380000D94EB090D94352F0C9459C00D94122F38
:100390000C945AA30C94BF550C94D6BF0D94F22D17
:1003A0004E414E494E495459494E46CDCCCC3D0A5A
:1003B000D7233C17B7D13877CC2B329595E6241F3D
:1003C000B14F0A000020410000C84200401C4620F6
:1003D000BCBE4CCA1B0E5AAEC59D7400407A10F3C9
:1003E0005A00A0724E18090010A5D4E80000E87663
:1003F00048170000E40B54020000CA9A3B000000BA
:10040000E1F505000080969800000040420F0000D2
:1004100000A08601000000102700000000E8030093
:100420000000006400000000000A0000000000015D
:1004300000000000002C76D888DC674F0823DFC15D
:10044000DFAE59E1B1B796E5E3E453C63AE6519918
:100450007696E8E6C28426EB898C9B62ED407C6F41
:10046000FCEFBC9C9F40F2BAA56FA5F490055A2AF8
:10047000F75C936B6CF9676DC11BFCE0E40D47FE04
:10048000F520E6B500D0ED902E03009435770500F9
:1004900080841E080000204E0A000000C80C333380
:1004A00033330F986E12831141EF8D2114893BE68F
:1004B0005516CFFEE6DB18D1844B381BF77C1D9018
:1004C0001DA4BBE424203284725E228100C9F12481
:1004D000ECA1E53D27434F4D4D554E49434154490D
:1004E0004F4E0044525952554E004552524F5253AE
:1004F00000494E464F004543484F004572726F72A7
:100500002077726974696E6720746F204545505278
:100510004F4D210A0053544F505045442E20005057
:1005200072696E7465722073746F70706564206494
:10053000756520746F206572726F72732E20466924
:100540007820746865206572726F7220616E642015
:10055000757365204D39393920746F207265737455
:100560006172742E202854656D70657261747572A5
:10057000652069732072657365742E20536574203D
:100580006974206166746572207265737461727437
:10059000696E67290A004E6F20436865636B737547
:1005A0006D2077697468206C696E65206E756D6268
:1005B00065722C204C617374204C696E653A200082
:1005C0004E6F20436865636B73756D20776974683F
:1005D000206C696E65206E756D6265722C204C61B1
:1005E0007374204C696E653A2000636865636B73B1
:1005F000756D206D69736D617463682C204C617337
:1006000074204C696E653A20004C696E65204E7509
:100610006D626572206973206E6F74204C61737413
:10062000204C696E65204E756D6265722B312C20F1
:100630004C617374204C696E653A20004D31313045
:100640000053657269616C20737461747573206DF9
:1006500069736D617463680A005344207265616454
:10066000206572726F720A00746F6F206D75636817
:1006700020696E6163746976652074696D65202DEB
:100680002063757272656E7420636F6D6D616E6448
:100690003A20002121204B494C4C20636175736541
:1006A000642062792000486F74656E642049646C30
:1006B000652054696D656F757400486F74656E646C
:1006C0002049646C652054696D656F75740A00700B
:1006D00061757365003D3D6F6E46696C616D656E59
:1006E0007452756E6F75743D3D004D36303000208C
:1006F00066696C616D656E745F72756E6F7574207E
:100700000066696C616D656E745F72756E6F75748D
:1007100020540046696C616D656E7452756E6F751C
:1007200074205400506F776572204F75746167654F
:10073000004D313030305300627573793A2070616A
:100740007573656420666F7220696E7075740A0037
:10075000627573793A2070617573656420666F7293
:1007600020757365720A00627573793A2070726F32
:1007700063657373696E670A0025533A2025530039
:100780002A2A2A6B696C6C2A2A2A00706F77657294
:100790006F6666004B494C4C45442E2000507269F0
:1007A0006E7465722068616C7465642E206B696C70
:1007B0006C28292063616C6C6564210A006563689C
:1007C0006F3A004572726F723A000A4D6561737537
:1007D00072656420706F696E74733A0A00357835FB
:1007E000206D6573682E205A206F66667365743AB3
:1007F00020002F2F616374696F6E3A006E6F746909
:100800006669636174696F6E200070726F6D7074D9
:100810005F00656E6400486F74656E6420746F6F6E
:1008200020636F6C640A0053656E64204D3130386C
:1008300020746F20726573756D650A00496E73656B
:1008400072742066696C616D656E7420616E6420DF
:1008500073656E64204D3130380A007061757365C0
:100860006400506175736500506F7765724F6666FE
:100870000A0057616974696E6720666F7220686547
:10088000617475702E0A004C656176696E67204749
:100890003236003F53706563696669656420582C81
:1008A0005920636F6F7264696E617465206F75742F
:1008B000206F6620626F756E64732E0A003F2852A7
:1008C0002965706561742076616C7565206E6F7442
:1008D00020706C61757369626C653B206D75737413
:1008E000206265206174206C6561737420312E0A6A
:1008F000003F2852296570656174206D75737420FE
:1009000062652073706563696669656420776865F0
:100910006E206E6F74207573696E6720616E204C57
:1009200043442E0A003F537065636966696564201D
:100930006E6F7A7A6C652074656D7065726174751E
:100940007265206E6F7420706C61757369626C657E
:100950002E0A003F537065636966696564206669A5
:100960006C616D656E742073697A65206E6F74209A
:10097000706C61757369626C652E0A003F53706517
:10098000636966696564207072696D65206C656E67
:10099000677468206E6F7420706C61757369626C27
:1009A000652E0A003F5072696D65206C656E677434
:1009B00068206D7573742062652073706563696665
:1009C000696564207768656E206E6F742075736941
:1009D0006E6720616E204C43442E0A003F537065C1
:1009E000636966696564206E6F7A7A6C65207369E5
:1009F0007A65206E6F7420706C61757369626C65C6
:100A00002E0A003F52657472616374696F6E204DE7
:100A1000756C7469706C696572206D757374206291
:100A200065207370656369666965642E0A003F53CB
:100A30007065636966696564205265747261637488
:100A4000696F6E204D756C7469706C696572206E8B
:100A50006F7420706C61757369626C652E0A003F5B
:100A6000537065636966696564206C61796572209D
:100A7000686569676874206E6F7420706C61757347
:100A800069626C652E0A0043292E0A003F53706587
:100A9000636966696564206265642074656D70656C
:100AA000726174757265206E6F7420706C617573FD
:100AB00069626C65202834302D004732362073740B
:100AC000617274696E672E2E2E0A004F46460A0028
:100AD0004661646520486569676874200042656402
:100AE000204C6576656C696E6720004661696C65AF
:100AF0006420746F20656E61626C652042656420BD
:100B00004C6576656C696E670A004D6573682042B6
:100B10006564204C6576656C20646174613A0A00F6
:100B2000496E76616C6964206D6573682E0A0020D9
:100B30006E6F7420656E74657265642E0A00507263
:100B40006F62696E6720506F696E740025532025AF
:100B5000692F256900206F6620004D424C204732E6
:100B60003920706F696E742000290A004A206F7561
:100B700074206F662072616E67652028302D002911
:100B80000A0049206F7574206F662072616E676578
:100B90002028302D004732384C30004D65736820D6
:100BA00070726F62696E6720646F6E65004D657369
:100BB000682070726F62696E6720646F6E652E0ABE
:100BC000005374617274206D6573682070726F6277
:100BD000696E672077697468202247323920533163
:100BE000222066697273742E0A004732395332002C
:100BF0004732384C300A473239533200686173202B
:100C00006E6F20646174612E0A004D657368204226
:100C10006564204C6576656C696E67200053206FB3
:100C20007574206F662072616E67652028302D35DF
:100C3000292E0A00651C621CA91CBA0E20204261E4
:100C4000636B6C6173682044697374616E636520C3
:100C5000286D6D293A2020202020202020002028E7
:100C600046312E30203D2066756C6C2C2046302E8F
:100C700030203D206E6F6E65290A002020436F7280
:100C800072656374696F6E20416D6F756E742F4667
:100C90006164652D6F75743A202020202046006124
:100CA00063746976653A0A00696E004261636B6C31
:100CB00061736820436F7272656374696F6E2000A0
:100CC00020204D36363600456E6473746F70206197
:100CD000646A7573746D656E740020440020204D45
:100CE00032303020540020204D323030205300204C
:100CF0002844697361626C6564293A0046696C61D5
:100D00006D656E742073657474696E67730020205E
:100D10004D32303120540020204D323031205800E7
:100D20004D617820416363656C65726174696F6EB3
:100D30002028756E6974732F7332290020204D327C
:100D4000303320540020204D3230332058004D6184
:100D500078206665656472617465732028756E69B4
:100D600074732F73290020520020204D323034201C
:100D70005000416363656C65726174696F6E202811
:100D8000756E6974732F7332292028503C70726914
:100D90006E742D616363656C3E20523C72657472A3
:100DA0006163742D616363656C3E20543C747261B1
:100DB00076656C2D616363656C3E290020540020CC
:100DC000530020204D323035204200416476616E60
:100DD0006365642028423C6D696E5F7365676D656D
:100DE0006E745F74696D655F75733E20533C6D6909
:100DF0006E5F66656564726174653E20543C6D6922
:100E00006E5F74726176656C5F666565647261744D
:100E1000653E20583C6D61785F6A65726B3E205973
:100E20003C6D61785F6A65726B3E205A3C6D6178FB
:100E30005F6A65726B3E20453C6D61785F6A6572E2
:100E40006B3E2900204C0020410020440020460039
:100E500020550020520020470020530020204D3212
:100E6000313700546F6F6C2D6368616E67696E6710
:100E70000020204D323138205400486F74656E6474
:100E8000206F66667365747300204400204900205B
:100E9000204D333031204500486F74656E6420501A
:100EA00049440020440020490020204D33303420A4
:100EB0005000426564205049440020450020204DE8
:100EC000393220540020204D3932205800537465A7
:100ED00070732070657220756E6974004E6F204DBE
:100EE0006F76652E0073706563696679696E672039
:100EF0004458435F4D4952524F5245445F4D4F4411
:100F0000452E0A005072696E746572206D75737497
:100F100020626520696E204458435F4455504C4917
:100F2000434154494F4E5F4D4F4445207072696FA5
:100F30007220746F200A002E0A002028302D3130D4
:100F400029002076616C7565206F7574206F6620AE
:100F500072616E676500416476616E6365204B0067
:100F600047323800203B00205500204C0020204D07
:100F700036303320540046696C616D656E74206CA8
:100F80006F61642F756E6C6F6164004D3234532550
:100F90006C6454256C64004739322E394525730042
:100FA00047314625640047315A25734636303000B4
:100FB0004731582573592573463330303000473157
:100FC00032004D313036502569532569005425696A
:100FD0002053004D313039532569005425695300A1
:100FE0004D3230305425694430004D323030542574
:100FF00069442573004739322E395A2573004D3420
:1010000032305325635A25730047323852305859CD
:101010000047315A257346363030004739322E3971
:101020005A2573004739322E394530004D31303959
:101030005325690054256953004D313930532569D2
:10104000004D343230205330205A30003D3D4F6E39
:10105000506F7765724C6F7373526573756D653D34
:101060003D00203B200020204D34313320530050E0
:101070006F7765722D6C6F7373207265636F766521
:101080007279004F4646004F4E00203B20486F7358
:10109000742068616E646C696E672000203B204D8F
:1010A0006F646520006D6D00203B2044697374619E
:1010B0006E6365200046696C616D656E74207275A3
:1010C0006E6F757420003B200020496E76616C695C
:1010D00064206578747275646572200047322F470A
:1010E000332062616420706172616D657465727332
:1010F0000A00536C6565702E2E2E004D65736820B6
:10110000706F696E74206F7574206F662072616EE7
:1011100067650A004D302053746F70004D312053C5
:10112000746F7000436C69636B20746F2052657339
:10113000756D652E2E2E00456E642066696C6520E7
:101140006C6973740A00426567696E2066696C6534
:10115000206C6973740A004E6F206D656469610AC2
:1011600000286E6F2066696C652900437572726590
:101170006E742066696C653A200043616E6E6F7410
:10118000206F70656E207375626469722000507202
:10119000696E742074696D653A20006F6B006F662C
:1011A0006600F604F104EA04E304D504444542551C
:1011B000473A004D31313320530050533A300A0042
:1011C00050533A310A0044656C6179656420706F50
:1011D0007765726F66660A0054656E6C6F672044AF
:1011E00033204F46462E00434F4E4649475F4558F1
:1011F000504F5254004D4541545041434B00434FD2
:101200004F4C45525F54454D5045524154555245FF
:10121000004348414D4245525F54454D504552416F
:101220005455524500424142595354455050494E3D
:10123000470041524353004D4F54494F4E5F4D4F6D
:1012400044455300544845524D414C5F50524F5411
:10125000454354494F4E00455854454E4445445F1C
:101260004D323000435553544F4D5F4649524D5710
:101270004152455F55504C4F4144004C464E5F57DC
:1012800052495445004C4F4E475F46494C454E41EC
:101290004D45004155544F5245504F52545F5344B1
:1012A0005F5354415455530053445F57524954457A
:1012B00000524550454154004D554C54495F564FDE
:1012C0004C554D45005344434152440050524F4DFC
:1012D00050545F535550504F525400484F53545F31
:1012E000414354494F4E5F434F4D4D414E4453008F
:1012F000454D455247454E43595F50415253455223
:1013000000434153455F4C494748545F4252494767
:1013100048544E45535300544F47474C455F4C4942
:101320004748545300534F4654574152455F504F1E
:10133000574552004255494C445F50455243454E33
:1013400054004C4556454C494E475F44415441007A
:101350005A5F50524F42450052554E4F555400412E
:1013600055544F4C4556454C005052494E545F4AD7
:101370004F420050524F4752455353004155544F2E
:101380005245504F52545F54454D50004155544FB3
:101390005245504F52545F504F5300564F4C554D8D
:1013A000455452494300454550524F4D0042494E25
:1013B0004152595F46494C455F5452414E53464550
:1013C000520053455249414C5F584F4E5F584F466B
:1013D00046004649524D574152455F4E414D453AB0
:1013E0004D61726C696E206275676669782D322E68
:1013F000312E782028536570203137203230323238
:101400002031333A30343A35322920534F55524344
:10141000455F434F44455F55524C3A676974687560
:10142000622E636F6D2F4D61726C696E4669726DCD
:10143000776172652F4D61726C696E2050524F5406
:101440004F434F4C5F56455253494F4E3A312E3021
:10145000204D414348494E455F545950453A5465E3
:101460006E6C6F67204433204558545255444552A2
:101470005F434F554E543A3220555549443A6365BF
:101480006465326132662D343161322D343734383F
:101490002D396231322D6335356336326633363756
:1014A00066660A002F2F005741524E494E472120B1
:1014B0004C6F77205A204A65726B206D6179206CE1
:1014C00065616420746F20756E77616E7465642049
:1014D0007061757365732E0A0020204D61783A2083
:1014E00000200020204D696E3A2000203B20002083
:1014F000204D323131205300536F667420656E6485
:1015000073746F70730046523A0020466C6F773ADE
:1015100020004261627973746570205A004D424C1C
:101520002041646A757374205A00496E76616C6953
:10153000642065787472756465720A00646973006A
:10154000656E0043290A0061626C656420286D693C
:101550006E2074656D702000436F6C642065787434
:1015600072756465732061726520005049442041A2
:1015700075746F74756E6500206661696C656421B1
:1015800020426164206865617465722069640A00A4
:10159000504944204175746F74756E65004D6573D4
:1015A0006820706F696E74206F7574206F6620728A
:1015B000616E67650A004D34323120696E636F7267
:1015C0007265637420706172616D657465722075F7
:1015D000736167650A004F666673657473204170B6
:1015E000706C696564004572723A20546F6F2066B2
:1015F00061722100546F6F206661722066726F6D98
:10160000207265666572656E636520706F696E74C1
:101610000A00454550524F4D204F4B0A004D38347B
:1016200000446F6E65207072696E74696E67206623
:10163000696C650A004D3737004D33310020204D6D
:10164000323036205800486F6D65206F66667365CE
:1016500074004361703A00526573756D696E67205E
:101660005344002569730025696D202569730025A1
:1016700069682025696D2025697300256964202526
:1016800069682025696D2025697300256979202501
:101690006964202569682025696D20256973000A21
:1016A00053746174733A2046696C616D656E742081
:1016B000757365643A20002C204C6F6E67657374F7
:1016C000206A6F623A2000546F74616C2074696DF7
:1016D000653A200053746174733A20002C204661EF
:1016E000696C65643A20002C2046696E69736865F0
:1016F000643A20005072696E74733A20005374612A
:1017000074733A200042656420436F6F6C696E67A2
:101710002E2E2E004265642048656174696E672E26
:101720002E2E003D3D4477696E20496E697420433A
:101730006F6D706C6574653D3D00202D2064342014
:101740000064333A2000202D206432200064313AB6
:101750002000202D206C656E20005650207265639D
:1017600065697665643A20002A2A2A4E6F7A7A6C77
:101770006554656D705374617475735B325D203DA3
:10178000003D3D48656174696E6720446F6E652059
:101790004368616E67652046696C616D656E743D76
:1017A0003D002020737461727470726F677265738C
:1017B0007320004D32320A4D3231003D3D77616970
:1017C0007477617920353D3D003D3D7761697477DF
:1017D000617920343D3D003D3D77616974776179E1
:1017E00020333D3D003D3D7761697477617920315B
:1017F0003D3D00436F6E6669726D20436F6E746984
:101800006E7565005061757365537461747573000E
:10181000524553554D45204F5054494F4E533A0071
:1018200048656174696E672E2E2E000000436C6956
:10183000636B20746F2068656174000000526573EB
:10184000756D696E672E2E2E0000005075726769E7
:101850006E672E2E2E000000496E73657274206133
:101860006E6420436C69636B000000436C69636BBA
:1018700020746F20636F6E74696E7565000000459B
:101880006A656374696E672E2E2E000000506C65C9
:1018900061736520776169742E2E2E0000005061FF
:1018A000726B696E672E2E2E0000002A2A2A496E5E
:1018B0006974696E672063617264206973204F4B9D
:1018C0002A2A2A003D3D6F6E5072696E7454696D0C
:1018D000657253746F707065643D3D003D3D6F6E81
:1018E00055736572436F6E6669726D526571756985
:1018F0007265643D3D005061757365204D6F646590
:1019000020537461747573004C6F6164696E672E47
:101910002E2E0000003D3D6F6E466163746F72793C
:1019200052657365743D3D00270A0A000027202791
:10193000002027002D0063616E63656C00507269A2
:101940006E742041626F7274656400554920416273
:101950006F7274656400726573756D65004D323425
:10196000005761726E696E673A20436C65616E2044
:10197000436972636C652072657175697265732065
:1019800058590A005761726E696E673A2052616455
:10199000697573204F7574206F662052616E67659C
:1019A0000A004E6F7A7A6C6520746F6F20636F6CDB
:1019B00064202D20536B697070696E6720776970A1
:1019C000650A003D3D6F6E5072696E7454696D65B5
:1019D000725061757365643D3D00486F6D696E6757
:1019E000204661696C65640050524553454E540071
:1019F0004F5554006F70656E005452494747455229
:101A00004544003A20004D4F54494F4E203A2000A3
:101A10004F46460A003A200066696C616D656E7437
:101A2000007A325F6D696E007A5F6D696E00795F72
:101A30006D696E00785F6D617800785F6D696E002A
:101A40005265706F7274696E6720656E6473746F2F
:101A500070207374617475730A0020746F6F206C4A
:101A60006F6E6720657874727573696F6E2070721F
:101A70006576656E7465640A0020636F6C6420652A
:101A80007874727573696F6E2070726576656E74A6
:101A900065640A00486F6D652025732573257320E2
:101AA00046697273740000004CC200000000000020
:101AB00000005761726E696E673A20486F6D696EFB
:101AC000672042756D702044697669736F72203C9F
:101AD00020310A0002020400000B440040044400CC
:101AE0008018440000A0400000A0400000004020FA
:101AF000746F6F206C6F6E67206578747275736990
:101B00006F6E2070726576656E7465640A0020637E
:101B10006F6C6420657874727573696F6E20707273
:101B20006576656E7465640A003D3D6F6E5072693E
:101B30006E7454696D6572537461727465643D3D71
:101B400000536176696E67204457494E204C4344E8
:101B50002073657474696E672066726F6D204545E9
:101B600050524F4D0A003D3D6F6E53657474696E5F
:101B7000677353746F7265643D3D00536574746997
:101B80006E67732053746F72656400290A002062C7
:101B9000797465733B2063726320005365747469C4
:101BA0006E67732053746F7265642028000A206981
:101BB0006E6974207A70726F62655F7A6F666673A1
:101BC0006574203D20003D3D6F6E436F6E66696712
:101BD00075726174696F6E53746F7265526561647A
:101BE0003D3D00454550524F4D20496E6974696135
:101BF0006C697A65640A0048617264636F64656445
:101C00002044656661756C742053657474696E67F1
:101C100073204C6F616465640020286D6D2900207D
:101C20003B204C6576656C696E67200020204D3442
:101C300032302053004D65736820426564204C6546
:101C400076656C696E6700204B0020204D3930307E
:101C50002054004C696E65617220416476616E6348
:101C6000650020590020580020204D343235204690
:101C7000004261636B6C61736820636F6D70656EA9
:101C8000736174696F6E0046696C616D656E742076
:101C900072756E6F75742073656E736F720020209D
:101CA000473239205334205A00205A00204A00205D
:101CB0002047323920533320490020204D31343918
:101CC0002043203B20556E69747320696E20436564
:101CD0006C736975730A0054656D70657261747513
:101CE000726520556E697473002020473231203BA5
:101CF000004C696E65617220556E697473004545CC
:101D000050524F4D206461746173697A6520657229
:101D1000726F722E0A0053657474696E6720566F75
:101D20006C756D65204F6E203A20005365747469A0
:101D30006E67205374616E646279204F6E203A2082
:101D40000053657474696E6720566F6C756D6520FD
:101D50003A200053657474696E6720526F74617421
:101D6000696F6E203A200053657474696E67205362
:101D700074616E6462792054696D65203A20005365
:101D8000657474696E67205374616E646279203A79
:101D9000200053657474696E6720427269676874C5
:101DA0006E657373203A20004C6F6164696E672022
:101DB0004457494E204C43442073657474696E67E0
:101DC0002066726F6D20454550524F4D0A004469A0
:101DD0007363617264696E67204457494E204C43B7
:101DE000442073657474696E672066726F6D204558
:101DF0004550524F4D202D2073657474696E677382
:101E00002076657273696F6E20696E636F7272659A
:101E100063740A0044697363617264696E67204485
:101E200057494E204C43442073657474696E672093
:101E300066726F6D20454550524F4D202D207369BD
:101E40007A6520696E636F72726563740A005374F9
:101E50006F7265642073657474696E677320726550
:101E60007472696576656400290A00206279746578
:101E7000733B2063726320002073746F726564206B
:101E800073657474696E67732072657472696576C0
:101E90006564202800454550524F4D204352432051
:101EA0004572726F7200202863616C63756C617497
:101EB000656429210A0020213D2000454550524FEC
:101EC0004D20435243206D69736D61746368202D0A
:101ED000202873746F7265642920002053697A6525
:101EE0003A2000496E6465783A20000000484300BB
:101EF00000484300002041000048420000484200E2
:101F000000A0420000A042000048443333B94233ED
:101F100033B942200300002003000064000000E801
:101F2000030000E8030000454550524F4D20566520
:101F30007273696F6E204572726F7200204D61720C
:101F40006C696E3D563837290A00454550524F4D51
:101F50002076657273696F6E206D69736D6174634D
:101F6000682028454550524F4D3D0024F404D920A7
:101F70001BC40C5C0E9804C4095F0265077101F470
:101F800005F900FB04B30048048700C10369005849
:101F900003550003034500BE023A0084023100539A
:101FA000022A002902250004022000E4011C00C8C6
:101FB000011900AF0117009801140084011300718A
:101FC0000110006101100051010E0043010D0036A7
:101FD000010B002B010B0020010B00150109000C67
:101FE00001090003010800FB000800F3000800EBF2
:101FF000000700E4000600DE000600D8000600D25C
:10200000000600CC000500C7000500C2000500BDA9
:10201000000400B9000400B5000400B1000400ADE4
:10202000000400A9000400A5000300A20003009F13
:102030000004009B00030098000300950002009339
:10204000000300900003008D0002008B0003008855
:102050000002008600020084000300810002007F6D
:102060000002007D0002007B000200790002007780
:10207000000100760002007400020072000100718D
:102080000002006F0002006D0001006C0002006A97
:1020900000010069000200670001006600010065A0
:1020A00000010064000200620001006100010060A4
:1020B0000001005F0002005D0001005C0001005BA8
:1020C0000001005A000100590001005800010057AA
:1020D00000010056000100550001005400010053AA
:1020E00000000053000100520001005100010050A7
:1020F0000001004F0001004E0000004E0001004DA5
:102100000001004C0001004B0000004B0001004AA0
:10211000000100490001004800000048000100479C
:102120000001004600000046000100450000004597
:102130000001004400010043000000430001004290
:102140000000004200010041000000410001004089
:102150000001003F0000003F0001003E0000003E83
:102160000001003D0000003D0001003C0000003C7B
:102170000000003C0001003B0000003B0001003A71
:102180000000003A00010039000000390001003869
:102190000000003800000038000100370000003760
:1021A0000001003600000036000000360001003556
:1021B000000000350000003500010034000000344C
:1021C0000000003400010033000000330000003341
:1021D0000001003200000032000000320001003136
:1021E000000000310000003100010030000000302C
:1021F000000000300001002F0000002F0000002F21
:102200000000002F0001002E0000002E0000002E14
:102210000001002D0000002D0000002D0000002D09
:102220000001002C0000002C0000002C0000002CFD
:102230000001002B0000002B0000002B0000002BF1
:102240000001002A0000002A0000002A0000002AE5
:1022500000010029000000290000002900000029D9
:1022600000000029000100280000002800000028CC
:1022700000000028000000280001002700000027BF
:1022800000000027000000270000002700010026B2
:1022900000000026000000260000002600000026A6
:1022A0000001002500000025000000250000002599
:1022B000000000250000002500010024000000248B
:1022C000000000240000002400000024000100237E
:1022D0000000002300000023000000230000002372
:1022E0000000002300000023000100220000002263
:1022F0000000002200000022000000220000002256
:102300000001002100000021000000210000002148
:102310000000002100000021000000210001002039
:10232000000000200000002000000020000000202D
:102330000000002000000020000000200001001F1D
:102340000000001F0000001F0000001F0000001F11
:102350000000001F0000001F0001001E0000001E02
:102360000000001E0000001E00000024F4D43050C5
:10237000C38E20C2A24017828B7011127A910D81F8
:102380006CD90AA861E108C7586607615143061E67
:102390004B5D05C145A7041A411104093D9803711D
:1023A0003931034036DB0265339102D43054028068
:1023B0002E1D02632CEE01752AC501B028A0011064
:1023C0002781018F2564012B244B01E0223401ACCD
:1023D000211F018D200D01801FFC00841EED009740
:1023E0001DDF00B81CD200E61BC600201BBC006429
:1023F0001AB200B219A8000A19A0006A189900D1EF
:1024000017910040178B00B516840031167E00B37B
:102410001579003A157300C7146F0058146A00EE5E
:102420001366008813630025135E00C7125B006CFF
:1024300012570015125400C111510070114F0021A4
:10244000114B00D61049008D104700461044000281
:10245000104200C00F4000800F3E00420F3C0006BB
:102460000F3B00CB0E3800930E37005C0E35002773
:102470000E3400F30D3200C10D3100900D300060BC
:102480000D2E00320D2D00050D2C00D90C2B00AEA9
:102490000C2900850C29005C0C2700350C27000E48
:1024A0000C2600E80B2400C40B2400A00B23007DA5
:1024B0000B23005A0B2100390B2100180B2000F8C8
:1024C0000A1F00D90A1E00BB0A1E009D0A1D0080BB
:1024D0000A1D00630A1C00470A1B002C0A1B00117E
:1024E0000A1A00F7091A00DD091900C4091900AB1E
:1024F000091900920917007B091800630917004C9D
:1025000009160036091600200916000A091500F5FB
:10251000081500E0081400CC081400B8081400A442
:10252000081400900813007D0812006B081300586F
:102530000812004608120034081100230811001286
:1025400008110001081100F0071000E0071000D08A
:10255000071000C0071000B0070F00A1071000917E
:10256000070E0083070F0074070F0065070E005762
:10257000070E0049070E003B070D002E070E002036
:10258000070D0013070D0006070D00F9060C00EDFE
:10259000060D00E0060C00D4060C00C8060C00BCBA
:1025A000060C00B0060C00A4060B0099060C008D6A
:1025B000060B0082060B0077060B006C060B006111
:1025C000060A0057060B004C060A0042060A0038AD
:1025D000060A002E060A0024060A001A060A00103F
:1025E00006090007060A00FD050900F4050900EBCD
:1025F000050900E2050900D9050900D0050900C751
:10260000050900BE050900B5050800AD050800A5CF
:102610000509009C050800940508008C0508008445
:102620000508007C050800740508006C05070065B6
:102630000508005D050700560508004E0507004720
:102640000507004005080038050700310507002A86
:10265000050700230507001C050600160507000FE7
:102660000507000805060002050700FB040600F543
:10267000040700EE040600E8040600E2040700DB9D
:10268000040600D5040600CF040600C9040600C3F2
:10269000040600BD040600B7040600B1040500AC42
:1026A000040600A6040600A00405009B040600958D
:1026B000040500900406008A0405008504050080D6
:1026C0000406007A04050075040500700405006B1B
:1026D00004050066040500610405005C040500575C
:1026E000040500520405004D04050048040500439C
:1026F0000405003E0404003A0405003504050030DA
:102700000404002C04050027040400230405001E13
:102710000404001A04040016040500110404000D4A
:10272000040400090405000404040000040400FC7F
:10273000030400F8030400F4030400F0030400ECB5
:10274000030400E8030400E4030400E0030400DCE5
:10275000030400D8030400D4030400D0030400CC15
:10276000030400C8030300C503030020436F756E14
:102770007420583A0023646566696E6520444546B6
:1027800041554C545F0000626564004B6420004B6F
:102790006920004B7020005049442074756E696EAA
:1027A0006720646F6E65002066696E697368656492
:1027B000212050757420746865206C617374204BFF
:1027C000702C204B6920616E64204B6420636F6E17
:1027D0007374616E74732066726F6D2062656C6FC6
:1027E0007720696E746F20436F6E666967757261DA
:1027F00074696F6E2E680A00504944204175746FE9
:1028000074756E6500206661696C65642120746969
:102810006D656F75740A00504944204175746F747A
:10282000756E65004175746F74756E6520666169BB
:102830006C6564212054696D656F75742E00206687
:1028400061696C6564212054656D70657261747591
:10285000726520746F6F20686967680A0050494488
:10286000204175746F74756E65005049442043793A
:10287000636C65730025532025692F256900204B63
:10288000643A2000204B693A2000204B703A200027
:1028900020436C617373696320504944200A00200F
:1028A0004E6F206F76657273686F6F740A002054E4
:1028B000753A2000204B753A2000206D61783A204F
:1028C00000206D696E3A200020643A200020626981
:1028D00061733A20002073746172740A0050494495
:1028E000204175746F74756E65004175746F7475F1
:1028F0006E65206661696C6564212054656D706544
:1029000072617475726520746F6F20686967682ED4
:1029100000206661696C6564212054656D70657284
:10292000617475726520746F6F20686967680A004A
:10293000504944204175746F74756E650000004500
:102940003200426564004531004500626564002C38
:102950002073797374656D2073746F707065642172
:10296000204865617465725F49443A20004572727F
:102970003A204D415854454D50004D415854454D15
:102980005020747269676765726564004865617498
:10299000696E67204661696C6564004865617469A9
:1029A0006E67206661696C6564004D313132205379
:1029B000687574646F776E004572723A204D494EA7
:1029C00054454D50004D494E54454D502074726948
:1029D00067676572656400202F0020400020424038
:1029E0003A0020403A00436F6F6C696E672E2E2EBE
:1029F0000048656174696E672E2E2E0045256320A0
:102A000025530020573A0020573A00496E76616CF2
:102A100069642065787472756465720A00486F7421
:102A2000656E6420746F6F20636F6C640A0041638D
:102A3000746976652045787472756465723A200011
:102A4000473132580000002100240027002A002DC1
:102A5000003000330001010000040107010A017C7D
:102A60003C3E5E2B3D3F2F5B5D3B2C2A225C0043AE
:102A7000616E6E6F74206F70656E2073756264692D
:102A80007220004D6564696120496E697420466159
:102A9000696C0053442063617264206F6B0A006F9D
:102AA00070656E526F6F74206661696C65640A00B0
:102AB000766F6C756D652E696E6974206661696CE0
:102AC00065640A004E6F20534420636172640A00FB
:102AD000534420636172642072656C656173656440
:102AE0000A000A4D3234004D3233202573002E0A7D
:102AF000006F70656E206661696C65642C204669A4
:102B00006C653A200046696C652073656C6563747A
:102B100065640A002053697A653A200046696C654D
:102B2000206F70656E65643A2000454E4420535511
:102B300042524F5554494E450A002220706F73008F
:102B40002220706172656E743A2200535542524FD2
:102B50005554494E452043414C4C20746172676581
:102B6000743A220053756263616C6C204F76657213
:102B7000666C6F77004578636565646564206D6198
:102B80007820535542524F5554494E452064657044
:102B900074683A002E0A0044656C6574696F6E2093
:102BA0006661696C65642C2046696C653A20004654
:102BB000696C652064656C657465643A004E6F7479
:102BC000205344207072696E74696E670A00534422
:102BD000207072696E74696E672062797465200076
:102BE00057726974696E6720746F2066696C653A04
:102BF0002000667265736800646F696E6700206606
:102C0000696C653A20004E6F7720002F6175746FF4
:102C100025632E670070012C0190012701B001226D
:102C200001C0011D01F00118011002130130020E54
:102C3000016002090190020401C002FF000003FAD2
:102C4000004003F5008003F000D003EB002004E611
:102C5000007004E100E004DC004005D700C005D2AC
:102C6000004006CD00D006C8008007C3003008BE73
:102C700000F008B900C009B400B00AAF00B00BAA58
:102C800000D00CA500000EA000500F9B00C01096B5
:102C9000005012910000148C00C0158700B01782FC
:102CA00000B0197D00D01B7800001E730040206E1C
:102CB0000090226900F024640040275F0090295AA8
:102CC00000E02B5500102E500020304B00103246F3
:102CD00000E033410090353C001037370070383247
:102CE00000A0392D00B03A2800A03B2300603C1E14
:102CF00000103D1900903D1400103E0F00703E0A78
:102D000000C03E0500003F0000403FFBFF803FF653
:102D1000FFC03FF1FF2020506C616E6E65724275FE
:102D20006666657242797465733A20002046726562
:102D300065204D656D6F72793A200020436F6D708C
:102D4000696C65643A205365702031372032303227
:102D5000320A00204C61737420557064617465649C
:102D60003A20323032322D30392D3134207C20411E
:102D70007574686F723A20496E73616E6974794137
:102D800075746F6D6174696F6E0A004D61726C6964
:102D90006E206275676669782D322E312E780A00B2
:102DA00020536F6674776172652052657365740A8B
:102DB00000205761746368646F672052657365749F
:102DC0000A002042726F776E206F7574205265730F
:102DD00065740A002045787465726E616C205265D6
:102DE0007365740A00506F77657255700A007374CA
:102DF0006172740A004739310A47315A350A473936
:102E0000300A4D38340A4D31303453300A4D3134A4
:102E1000305330004D31303031006572726F7220A6
:102E200077726974696E6720746F2066696C650AD1
:102E300000446F6E6520736176696E672066696C09
:102E4000652E0A004D323900456E6473746F7073DD
:102E5000002553202563202563202563202563005A
:102E6000205A3A0020593A0020583A00656E64739F
:102E7000746F7073206869743A2000000022002586
:102E80000028002B002E0031003400020100000554
:102E90000108010B01C23100001C260000F41900DA
:102EA00000D80F0000EB080000C00400007502000D
:102EB000004001000043616E6E6F7420656E7465A2
:102EC00072207375626469723A20004D3235205069
:102ED0000A4D323400526573756D650055492050B6
:102EE00061757365004E6F204D61746368203A0010
:102EF000436F6E73747261696E206D65736856619D
:102F00006C20006D65736856616C200079506E749A
:102F1000200078506E7420006D657368506F696E84
:102F2000742000446973706C6179427269676874D7
:102F30006E657373205365743A2000446973706C36
:102F400061794272696768746E657373204C43449B
:102F50003A20004D32320A4D3231005265667265B8
:102F600073680050675570005067446F776E004972
:102F7000732046696C652000497320446972200003
:102F8000476F557044697200486173204D656469EC
:102F9000610046696C656E616D652053656C6563A3
:102FA000746564004D3130303043004D3130303085
:102FB000002046696C616D656E7420526573706F98
:102FC0006E7365204E6F00526573756D652059658F
:102FD0007320647572696E67207072696E74000A7E
:102FE000204E6F2046696C616D656E7400496E7687
:102FF000616C6964204F7074696F6E004D353030BC
:103000000053746F72652053657474696E67730042
:103010004D3939390A4D323830503053313630005D
:10302000424C546F756368205265736574004D356A
:1030300030320A4D35303000496E697420454550B4
:10304000524F4D004D3530300053746F7265205330
:10305000657474696E677300496E4C616E6743688E
:103060006F696365000A202A2A2A726563646174A5
:103070002E646174615B305D203D004732380A4741
:1030800031204631303030205A313000556E737562
:1030900070706F72746564204F7074696F6E205326
:1030A000656C6563746564004D36303553300A478E
:1030B000323858004D36303553310A54300A4732D1
:1030C000380A4D36303553320A473238580A4731BC
:1030D00058300A4D3630355333004D363035533184
:1030E0000A54300A4732380A4D36303553320A47CF
:1030F0003238580A47315830004D36303553310A8E
:10310000473238580A47315830004D323131533048
:103110000A4739310A47315A302E3032350A473999
:10312000300A4D3231315331004D32313153300A92
:103130004739310A47315A2D302E3032350A473956
:10314000300A4D3231315331004732395332004762
:10315000323953310047323652323535004731204B
:103160004631303030205A302E30004732380A474E
:1031700031204631303030205A302E30005A204F26
:103180006666736574203A202573005A204F666680
:10319000736574203A202573004732385A0A473144
:1031A00046313530305A302E30004732380A4731F8
:1031B00046313530305A302E3000426564204C653F
:1031C00076656C204F7074696F6E2000526574755F
:1031D000726E203A20004D3834004731463130308D
:1031E000305A302E30004732380A473146313030BD
:1031F000305A302E30004D616E75616C53657454D9
:10320000656D70005A204F6666736574203A2025FC
:103210007300526F756E64696E6720746F207374EB
:10322000657000526571756573746564204F6666DC
:10323000736574200053746F7020547269676765FA
:103240007265640053746F70204E6F0053746F701A
:103250005072696E740048616E646C6520446174DC
:10326000612041646A7573742032205365747469F7
:103270006E672053637265656E200048616E646CF2
:10328000652044617461205072696E7446696C6592
:1032900020332053657474696E67205363726565CB
:1032A0006E200048616E646C65204461746120503A
:1032B00072696E7446696C65203220536574746956
:1032C0006E672053637265656E20004D3834004888
:1032D000616E646C652044617461205072696E7423
:1032E00046696C6520506F73740048616E646C654C
:1032F0002044617461205072696E7446696C652067
:1033000050726500426567696E537769746368003F
:103310003D3D20436865636B6B65793D3D0072659B
:10332000636461742E61646472203D3D0072656364
:103330006461742E646174615B305D203D3D007793
:10334000616974776179203D3D0020202A2A2A2A6C
:103350002A2A2A5254535F48616E646C6544617432
:10336000612A2A2A2A2A2A2A2A200073686F7700CB
:10337000627574746F6E00626567696E004469738C
:1033800061626C6552756E6F757400507572676519
:103390004D6F726500506175736564004C6F6164B8
:1033A0002046696C616D656E742054004C6F6164D9
:1033B0002046696C616D656E7400496E7365727448
:1033C0002066696C616D656E7420616E6420736542
:1033D0006E64204D3130380A00726573756D656416
:1033E000004469736D69737300526573756D696E1E
:1033F000670052656865617420446F6E65005265B0
:1034000068656174696E672E2E2E0052656865616D
:1034100074004865617465722054696D656F7574D8
:103420000053656E64204D31303820746F2068651C
:103430006174206E6F7A7A6C650A00436F6E7469EE
:103440006E7565004E6F7A7A6C65205061726B659F
:103450006400FFFFFF544845524D414C2052554EE9
:103460004157415900546865726D616C2052756E08
:103470006177617900000020002300260029002CDC
:10348000002F0032000001000003010601090105C0
:10349000050505070508080808020202020A0A08CD
:1034A00008040404040101010101010101030303F3
:1034B0000303030303040707070C0C0C0C0C0C0C90
:1034C0000C0202020206060606060606060B0B0B97
:1034D0000B0B0B0B0B0102102020080810204010D2
:1034E00020408002010201080402010102040810C8
:1034F00020408080402010080402018004020180E6
:10350000402010080402010804020101020408100E
:10351000204080010204081020408000000A0B02B5
:10352000090C0D0E08070304010000000000000054
:10353000000000000000000000000000000000008B
:103540000000000000000012111000000000000048
:10355000000000000000000000000000000000006B
:103560000020453A00205A3A0020593A00583A00C3
:1035700054656E6C6F672044332052656164792E08
:10358000005072696E74696E672E2E2E005072693B
:103590006E742050617573656400524553554D45F6
:1035A000204F5054494F4E533A0048656174696E3C
:1035B000672E2E2E000000436C69636B20746F2011
:1035C00068656174000000526573756D696E672EE1
:1035D0002E2E00000050757267696E672E2E2E0029
:1035E00000004C6F6164696E672E2E2E000000494A
:1035F0006E7365727420616E6420436C69636B0046
:103600000000436C69636B20746F20636F6E746994
:103610006E7565000000456A656374696E672E2EDD
:103620002E000000506C6561736520776169742E0F
:103630002E2E0000005061726B696E672E2E2E00D8
:10364000000050617573654D73673D006F6B0A0034
:10365000526573656E643A2000220A00556E6B6EE7
:103660006F776E20636F6D6D616E643A202200206B
:1036700042002050006F6B006E6F74696669636171
:1036800074696F6E20003E017E0111241FBECFEFD2
:10369000D1E2DEBFCDBF00E00CBF84B78093F21C47
:1036A00014BE0FB6F894A89580916000886180934D
:1036B0006000109260000FBE16E0A0E0B2E0E4E50A
:1036C000F2EA02E00BBF02C007900D92A834B107E6
:1036D000D9F72CE1A8E4B6E001C01D92A23FB207E1
:1036E000E1F71BE1C4E4DBE100E006C0219701093A
:1036F000802FFE010F94574DC334D10780E0080797
:10370000A9F70F94D1370D9418510C940000209113
:10371000AA13833021F425FD0CC024FD0CC030E039
:10372000A90102C0559547958A95E2F7CA018170B3
:10373000089581E0089580E008958091BA0784FD9E
:103740000BC08091BC0787FD07C09091BD079370A7
:1037500081E019F480E0089581E008950F931F93AC
:10376000CF93DF9300D01F92CDB7DEB79C0109E95C
:1037700011E190E1E9E7F2E0D80101900D929A950C
:10378000E1F7F9012081318142815381F80160859F
:103790007185828593850F94604DF80160877187EC
:1037A0008287938780E090E0A0EAB0E489839A83DF
:1037B000AB83BC83CE0101960E941A8F0F900F90AD
:1037C0000F900F90DF91CF911F910F9108952F923D
:1037D0003F924F925F926F927F928F929F92AF92A1
:1037E000BF92CF92DF92EF92FF921F93CF93DF931E
:1037F000CDB7DEB72C970FB6F894DEBF0FBECDBFA6
:103800007A011901DC012D913D914D915C912D833F
:103810003E834F835887FB014080518062807380D4
:103820008090790290907A02A0907B02B0907C0206
:10383000A50194016D817E818F8198850F946E46DC
:1038400081110EC011E0A301920160917D0270917F
:103850007E0280917F02909180020F946E468111CA
:1038600010E0D1012D913D914D915C9129873A87CE
:103870004B875C87F701C080D180E280F380209184
:103880000202309103024091040250910502C701E7
:10389000B6010F946E46882309F44EC0C09202020E
:1038A000D0920302E0920402F09205028091850218
:1038B00090918602A0918702B091880240917D028A
:1038C00050917E0260917F027091800280929911E6
:1038D00090929A11A0929B11B0929C1140939D11CD
:1038E00050939E1160939F117093A011C092A111EB
:1038F000D092A211E092A311F092A4118093A5118D
:103900009093A611A093A711B093A81120E030E0E6
:1039100040E05FE36091DD117091DE118091DF1175
:103920009091E0110F94D44669837A838B839C83B2
:10393000CE0101960E941A8F2D813E814F815885BC
:103940002093991130939A1140939B1150939C119D
:1039500040929D1150929E1160929F117092A01101
:10396000D1012D913D914D915C916091A511709186
:10397000A6118091A7119091A8110F94604D6093AA
:10398000A5117093A6118093A7119093A8111111FE
:103990002FC020E030E0A90169857A858B859C8560
:1039A0000F946E46811133C060E070E088EC92E4C1
:1039B00069837A838B839C83CE0101960E941A8F40
:1039C0002C960FB6F894DEBF0FBECDBFDF91CF911E
:1039D0001F91FF90EF90DF90CF90BF90AF909F909E
:1039E0008F907F906F905F904F903F902F900895B1
:1039F0002AEF3EE74AE25FE36091E1117091E21144
:103A00008091E3119091E4110F94D446D1CF60E0FE
:103A100070E080EA91E4CCCF80919A0790919B0767
:103A2000009731F04AE050E070E060E00D94894486
:103A300060E070E0CB0108950F931F93CF93DF9365
:103A400000D000D01F921F92CDB7DEB78B01FC01D2
:103A500023A5211102C00F94170D1D821E821F8203
:103A6000188620E030E040E05FE3609181027091D1
:103A7000820280918302909184020F94604D698349
:103A80007A838B839C839E012B5F3F4FAE014F5FF8
:103A90005F4F6DE772E089E792E00E94E71B1D82AD
:103AA0001E821F82188620E030E040E05FE3F801CC
:103AB00060857185828593850F94604D69837A83D3
:103AC0008B839C83B8016C5F7F4F9E012B5F3F4FC0
:103AD000AE014F5F5F4FC8010E94E71B28960FB6EB
:103AE000F894DEBF0FBECDBFDF91CF911F910F9134
:103AF00008950F931F93CF93DF93C82FD0E0FE015B
:103B0000EE0FFF1FE65CFD4F71836083CC0FDD1F5E
:103B1000CC0FDD1F8E01075E1D4F072E000C880B9A
:103B2000990B0F9475462AE037ED43E25CE30F945E
:103B3000D446C15FD74F288139814A815B810F9478
:103B4000D446F8016083718382839383DF91CF91A0
:103B50001F910F910895682F880F770B880B990B91
:103B60000D94B802682F70E090E080E00D94B802E8
:103B70009B01AC01485F5F4FBC016C5F7F4F0C94B1
:103B8000E71B2F923F924F925F926F927F928F929C
:103B90009F92AF92BF92CF92DF92EF92FF920F93DC
:103BA0001F93CF93DF93CDB7DEB7A6970FB6F894E8
:103BB000DEBF0FBECDBF8C011B015A8749874090E5
:103BC000790250907A0260907B0270907C02809023
:103BD0007D0290907E02A0907F02B0908002DB0177
:103BE0008D919D910D90BC91A02D8B8B9C8BAD8B5D
:103BF000BE8B9C01AD01C301B2010F945F4D6B01FF
:103C00007C01D10114968D919D910D90BC91A02DB8
:103C10008F8B988FA98FBA8F9C01AD01C501B4011C
:103C20000F945F4D6B8F7C8F8D8F9E8FA985BA858A
:103C30008D919D910D90BC91A02D8B879C87AD8718
:103C4000BE879C01AD01C301B2010F945F4D6F8F20
:103C500078A389A39AA3A985BA8514968D919D917D
:103C60000D90BC91A02D8F87988BA98BBA8B9C014E
:103C7000AD01C501B4010F945F4D6BA37CA38DA36F
:103C80009EA3A7019601C701B6010F94D4466B010C
:103C90007C012B8D3C8D4D8D5E8DCA01B9010F9439
:103CA000D4469B01AC01C701B6010F94604D4B0196
:103CB0005C012B893C894D895E896B857C858D856E
:103CC0009E850F945F4D2B013C012F89388D498DC6
:103CD0005A8D6F85788989899A890F945F4D6B0118
:103CE0007C01A3019201C301B2010F94D4462B01C0
:103CF0003C01A7019601C701B6010F94D4469B0170
:103D0000AC01C301B2010F94604D0F940E506B01D2
:103D10007C012F8D38A149A15AA1CA01B9010F9484
:103D2000D4462B013C012BA13CA14DA15EA1CA01AF
:103D3000B9010F94D4469B01AC01C301B2010F94A9
:103D4000604D9B01AC01C501B4010F94C04F181622
:103D5000B4F520E030E0A901C701B6010F94C04FCF
:103D600087FF2AC0C701B601905820E030E040EA42
:103D700050E40F94C04F181614F5A10169857A8597
:103D8000C8010E94C11DA6960FB6F894DEBF0FBEF3
:103D9000CDBFDF91CF911F910F91FF90EF90DF90FA
:103DA000CF90BF90AF909F908F907F906F905F90DB
:103DB0004F903F902F900895C701B601D6CF20E0D5
:103DC00030E040E050E4C501B4010F94C04F181634
:103DD00024F4B101C8010E941C1D19821A821B82A1
:103DE0001C82BE016F5F7F4FC1010E94B81D2DEC88
:103DF0003CEC4CEC5CE3C701B6010F94D4469B014C
:103E0000AC01F80160817181828193810F94D44665
:103E10006D837E838F839887D8019B968C919B9727
:103E20008823C9F02AE939E949E95FE314966D91DD
:103E30007D918D919C9117970F94D44669837A83D5
:103E40008B839C83BE016F5F7F4F89E991E10E9464
:103E5000B81DF80113A6BE016B5F7F4F89859A8557
:103E60000E94B81D90CF2F923F924F925F926F9217
:103E70007F928F929F92AF92BF92DF92EF92FF92CA
:103E80000F931F93CF93DF93CDB7DEB768970FB62D
:103E9000F894DEBF0FBECDBFFB015081342F350F2C
:103EA000353008F0D0C0E180022F0E0D053008F04B
:103EB000CAC0F12C852E912CF701E058F84FE08113
:103EC000F0E002C0F595E7955A95E2F7E0FFBBC038
:103ED00010E0A32EB12CF801E058F84FE081F0E09B
:103EE00002C0F595E7953A95E2F7E0FFACC0D22E17
:103EF000642F3C01660F770B072E000C880B990B83
:103F00000F9475461B012C01F401EE0FFF1FEE0FFD
:103F1000FF1FEC50F54EA2019101608171818281F9
:103F200093810F94604D6D877E878F87988BF50105
:103F3000EE0FFF1FEE0FFF1FEC50F54EA201910197
:103F400060817181828193810F945F4D69837A834F
:103F50008B839C836D2D660F770B072E000C880BCF
:103F6000990B0F9475464B015C01F701EE0FFF1F93
:103F7000EE0FFF1FE052F54EAC019B016081718195
:103F8000828193810F94604D698B7A8B8B8B9C8B94
:103F9000000F111F000F111FF801E052F54EA5018F
:103FA000940160817181828193810F945F4D6D8353
:103FB0007E838F839887F30180859185A285B38561
:103FC00089879A87AB87BC878D8B9E8BAF8BB88F89
:103FD00040E152E061E070E0CE0141960E949C70A9
:103FE00040E152E061E070E0CE0105960E949C70D5
:103FF00048EF51E06EEC7FEFCE010D960E949C7071
:1040000048EF51E06EEC7FEFCE0101960E949C706C
:10401000BE016F5E7F4FCE010D960E94858F882373
:1040200091F0BE016B5F7F4FCE0101960E94858F9C
:10403000882349F0AE014F5F5F4FBE01635F7F4F42
:10404000C3010E94C11D68960FB6F894DEBF0FBE73
:10405000CDBFDF91CF911F910F91FF90EF90DF9037
:10406000BF90AF909F908F907F906F905F904F9098
:104070003F902F90089580919A0790919B07009709
:1040800031F04AE050E070E060E00D945B4360E0A6
:1040900070E0CB0108950E943B2097FD0CC00E9468
:1040A0003B206F3F71058105910509F034F40E94B2
:1040B0003B20862F089580E008958FEF089580912A
:1040C0009A0790919B07892B41F00E944B2091E029
:1040D000811101C090E0892F089591E0FCCF0E94EA
:1040E0003B20CB0108950F931F93CF9380919A07A4
:1040F00090919B07009709F1FC018F01C1912C2F32
:104100002F7DA1F0C53431F0C53621F0C83511F04E
:10411000C83799F7F801108270E060E00F94FD4114
:10412000F801C083CF911F910F91089570E060E076
:10413000CF911F910F910D94FD4160E070E0CB0194
:10414000F1CF2FEB280F2A3108F047C0E22FF0E023
:104150008091BA079091BB07A091BC07B091BD07B1
:1041600004C0B695A795979587952A95D2F780FDB7
:1041700002C081700895E056F84FE081EE2341F1CE
:104180008091961690919716E80FF92FF11D808176
:1041900090ED980F9A3030F08E3251F48181805337
:1041A0008A3098F4F0939B07E0939A0781E0089592
:1041B0008D3211F08B3249F4818190ED980F9A3055
:1041C00088F38E3211F48281EACFF0E0E0E0EACFAA
:1041D00010929B0710929A07E9CF80E008950E9401
:1041E000A120882341F081E020919A0730919B071C
:1041F000232B09F480E00895CF92DF92EF92FF9293
:104200006A017B010E94EF20882331F0FF90EF903C
:10421000DF90CF900C947320C701B601FF90EF9010
:10422000DF90CF9008954F925F926F927F92AF92FE
:10423000BF92CF92DF92EF92FF920F931F93CF9393
:104240008BEBA82E82E0B82E99E9E92E91E1F92EA8
:1042500009E712E021EBC22E22E1D22EC0E0F501E7
:1042600081915F010E94EF20882309F4A9C00E9478
:1042700073202B013C018C2F0E94871B882309F49B
:1042800095C0F8012081318142815381C301B2017F
:104290000F94604DF7016083718382839383CF5FB6
:1042A000F4E0EF0EF11C0C5F1F4F84E0C80ED11C30
:1042B000C330A9F685E40E94EF20882309F48BC05F
:1042C0000E9473206B017C0183E00E94871B88237E
:1042D00071F02091850230918602409187025091C1
:1042E0008802C701B6010F94604D6B017C01C0923A
:1042F000A511D092A611E092A711F092A81140E06A
:1043000050E0BA0186E40E94FC2020E030E0A901E0
:104310000F94C04F181684F40E94732020E030E000
:1043200040E752E40F945A4E609375027093760200
:1043300080937702909378028091A91383FD28C01F
:1043400080918C09882321F1209185023091860289
:1043500040918702509188026091A5117091A61139
:104360008091A7119091A8110F945F4D2091990908
:1043700030919A0940919B0950919C090F94604D8E
:104380006093990970939A0980939B0990939C0973
:10439000CF911F910F91FF90EF90DF90CF90BF9042
:1043A000AF907F906F905F904F900895F6012081BD
:1043B000318142815381C301B2010F945F4D6ACFB5
:1043C000F80180819181A281B381F701808391837B
:1043D000A283B38364CF8091850290918602A091DD
:1043E0008702B09188028093A5119093A611A093A3
:1043F000A711B093A81183CFCF93DF93EB010E9455
:10440000EF20882321F0DF91CF910C946F20CE0113
:10441000DF91CF910895CF93DF93EB010E94EF20BE
:10442000882319F00E943B20EB01CE01DF91CF9150
:104430000895CF93C62F0E94EF20882319F0CF91C3
:104440000C944B208C2FCF910895CF93DF93C82FDE
:10445000D62F0E94EF20882321F0DF91CF910C947A
:104460005F208C2F0E94A120811101C08D2FDF9130
:10447000CF910895E3EDF3E187EBDF011D928A957B
:10448000E9F7089580917A11811104C00E943A22BF
:104490000C948DF98091131B82FF09C087FD07C022
:1044A00040E060E070E080E090E40D94B108089591
:1044B0008091D313882361F090918914891308C0E7
:1044C0008091131B84FF04C086E194E10C9484D393
:1044D00080E00895FC01238121110C94CFCF089531
:1044E000AC018091A81381110AC020910F02309174
:1044F00010022350310981E0421753070CF080E08D
:10450000089597E1899FF0011124E758F74E20E0C4
:1045100030E040E05FE364817581868197810F948C
:10452000604D0F94CC4ECB010C947022CF93DF934F
:10453000C0916A18D0916B18209729F16091661884
:104540007091671880916818909169180F94CC4EFB
:104550006E5F7F4F24976C177D07ACF47093D4087F
:104560006093D3080F94C612605A75418F4F9F4FC6
:104570006093D5087093D6088093D7089093D80895
:10458000DF91CF9108951092D5081092D60810921D
:10459000D7081092D808F4CF0F931F93CF93DF93CF
:1045A000082F10E097E1899FF0011124E758F74E9A
:1045B000C085D185209729F1648175818681978195
:1045C0000F94CC4E6E5F7F4F26976C177D07CCF40F
:1045D00086E0809FE001819FD00D1124C752D74F04
:1045E000798368830F94C612605E714B8F4F9F4F23
:1045F0006A837B838C839D83DF91CF911F910F9181
:10460000089586E0809FF001819FF00D1124E7520C
:10461000F74F1282138214821582EECF95E0899FA4
:10462000F0011124E350FE4E108211821282138297
:1046300014820C94CC22CF93DF9310929B0810929B
:104640009C0810929D0810929E08ECE4F2E184E62A
:10465000DF011D928A95E9F7C0E0D0E06D2F8C2F25
:104660000F94AC0ADF5FD530C9F7CF5FC530A9F72B
:10467000DF91CF9108959091AF139817A1F00E9408
:10468000357189E792E00E9458718091AF1391E0F3
:1046900089278093AF13882321F089E792E00E9455
:1046A000EB6F0C94A2890895EF92FF920F931F93E2
:1046B000CF93DF930CE412E1C5E07801D5E0F70178
:1046C00061917191819191917F0120E030E0A90188
:1046D0000F946E4681110EC0D15089F7C1500C5E07
:1046E0001F4FC111EACFDF91CF911F910F91FF9022
:1046F000EF90089581E0F7CFCF92DF92EF92FF9293
:104700000F931F93CF93DF93833009F452C0C82FC8
:10471000D0E08E01000F111F000F111FF801E95E9C
:10472000F74FC080D180E280F3802091230830E0F1
:1047300002C0359527958A95E2F720FD10C06627BF
:104740007727CB016C197D098E099F09DF91CF91E5
:104750001F910F91FF90EF90DF90CF90089560919F
:10476000210270E090E080E00F94734620E030E09A
:104770004FE753E40F945A4E9058F801E758F74F1B
:1047800020813181428153810F94D446CC0FDD1FAB
:10479000CC0FDD1FCF53DE4E288139814A815B81EA
:1047A0000F94D4460F94CC4E6C197D098E099F0945
:1047B000CDCF60E070E0CB01C9CF4F925F926F9296
:1047C0007F928F929F92AF92BF92FF920F931F930F
:1047D000CF93DF938C01C7E1D8E0F12C8F2D0E949D
:1047E0007C23F80141905190619071908F018990E4
:1047F0009990A990B990FE013497641975098609BA
:104800009709860E971EA81EB91E80829182A282E9
:10481000B382F394F3E0FF12E1CFDF91CF911F91C8
:104820000F91FF90BF90AF909F908F907F906F906F
:104830005F904F9008958F929F92AF92BF92CF92C8
:10484000DF92EF92FF920F931F93CF93DF93CDB739
:10485000DEB72C970FB6F894DEBF0FBECDBF182F72
:104860004A015B01CE0101967C0100E06C01802FC2
:104870000E947C23F70161937193819391937F014F
:104880000F5F0330A1F784E0189FF0011124E7586F
:10489000F74F80829182A282B382C6010E94DD23FB
:1048A0002C960FB6F894DEBF0FBECDBFDF91CF912F
:1048B0001F910F91FF90EF90DF90CF90BF90AF903E
:1048C0009F908F900895CF92DF92EF92FF920F9377
:1048D0001F93CF93DF93CDB7DEB72C970FB6F89425
:1048E000DEBF0FBECDBFC82ECE0101967C0110E009
:1048F000D82E0F2D812F0E947C23F7016193719395
:10490000819391937F011F5F1330A1F7C092210221
:104910008D2D902F0E94DD232C960FB6F894DEBFCC
:104920000FBECDBFDF91CF911F910F91FF90EF9000
:10493000DF90CF90089520917A0730917B07280F60
:10494000391F30937B0720937A072091EB08309131
:10495000EC08280F391F3093EC082093EB082091C6
:104960000D0830910E08820F931F90930E088093CC
:104970000D080F94C6126093ED087093EE088093B3
:10498000EF089093F0080895CF92DF92EF92FF9294
:104990006B017C0183E3C816D104E104F10470F0DB
:1049A00082E3C81AD108E108F10862E370E080E010
:1049B00090E00F9493120E9423DCECCFC701B60164
:1049C0000F949312FF90EF90DF90CF900C9423DC24
:1049D0000F931F930F94C61201E010E020E030E027
:1049E000611571058105910519F000E010E098014D
:1049F000DC01CB01800F911FA21FB31F80937C07A6
:104A000090937D07A0937E07B0937F0780918B09D9
:104A1000811117C01092E1091092E2091092E30986
:104A20001092E4091092E009999AA19A81E080938A
:104A30008B096AEF70E080E090E01F910F910C9479
:104A4000C4241F910F9108950F931F93CF930E9439
:104A50009D1B8823C1F185E40E94A120882361F079
:104A600080919A0790919B07892B41F10E946F20BA
:104A7000823010F40E94BDF10BEB12E0C0E0F801AF
:104A800021918F0121548091BA079091BB07A09189
:104A9000BC07B091BD0704C0B695A79597958795BB
:104AA0002A95D2F780FF03C08C2F0E940AF2CF5FB5
:104AB000C33029F7CF911F910F91089580E00E9494
:104AC00016E481E0D7CF60E08CED9EE00E942B9D44
:104AD0000E94E82480E00E940AF281E00E940AF22B
:104AE00082E00E940AF280E00E9416E481E0CF9109
:104AF0001F910F910C94BDF1CF93DF93EC01892BA3
:104B000039F00E94E824CC38D10514F0CCE8D0E08C
:104B1000D0936B18C0936A18DF91CF910C949622B2
:104B20001F93CF93DF93EC01162F892B11F00E9476
:104B3000E824E12FF0E087E1189FD0011124A75865
:104B4000B74EEE0FFF1FE95BFC4F808191810F97FD
:104B5000C817D9070CF4CE0119969C938E93189719
:104B6000812FDF91CF911F910C94CC228091BA13A9
:104B70000E949DF164E670E080E090E00C94C42413
:104B8000109278118091AC089091AD08A091AE0878
:104B9000B091AF088093A8089093A908A093AA08A1
:104BA000B093AB0808959091BD121092BD1292304F
:104BB000D9F09430E1F0913001F5882319F081307B
:104BC00021F0089590937911089582E080937911EE
:104BD00080917811882389F0E091BA13F0E0EF50CA
:104BE000F54F10820C94C02510928C1108958DE51C
:104BF00099E19093030B8093020B0895E4E0F1E0B8
:104C000080818E7F80838091050180958170809363
:104C100003010C94C0258091BE12813069F09091FF
:104C2000131B92FB882780F992FF07C097FB882708
:104C300080F991E08927089581E008959091131BF0
:104C400094FB882780F994FF06C081E090917A1C3C
:104C5000911101C080E008950E941E26882339F03A
:104C60008091131B82FB882780F991E089270895A2
:104C700080917B11811106C08091BE12823011F0AB
:104C80000C942C2681E0089581E00895CF93DF9362
:104C9000EC01E62F660FFF0BE55EFA4CE491E25063
:104CA000E13108F0B0C0F0E08827E65AF94D8F4FA7
:104CB0000D94574D6B2603270327032703279526BB
:104CC0007726B926B7269726DD26DB26BB260327BF
:104CD0000127FF26DF2682E1E1E9F2E0DE01019013
:104CE0000D928A95E1F7CE01DF91CF91089581E091
:104CF00020EB30E03983288321EB30E03B832A83AB
:104D00001D821C8223EB30E03F832E8324EB30E0B6
:104D1000398728871B861A861D861C8692E09E8707
:104D20008F8781E0888B198ADECF80E0E1CF81E038
:104D30008F5F20E930E03983288321E930E03B832D
:104D40002A8322E930E03D832C8328E930E03F8349
:104D50002E832AE930E0398728872CE930E03B8729
:104D60002A8726E930E03D872C8793E0D8CF80E082
:104D7000DFCF80E0DECF81E08F5F20EA30E0398353
:104D8000288321EA30E03B832A8322EA30E03D8316
:104D90002C8328EA30E03F832E832AEA30E03987EB
:104DA00028872CEA30E03B872A8726EA30E03D87D7
:104DB0002C8794E0B4CF80E0DFCF80E0DECF81E0CD
:104DC0008F5F20E231E03983288321E231E03B83A9
:104DD0002A8322E231E03D832C8328E231E03F83C5
:104DE0002E832AE231E0398728872CE231E03B87A5
:104DF0002A8726E231E03D872C8795E090CF80E03E
:104E0000DFCF80E0DECF82E1FE0111928A95E9F7E3
:104E10006ACF8F929F92AF92BF92CF92DF92EF9222
:104E2000FF920F93CF93DF931F92CDB7DEB75C0154
:104E30007B0149016B01C40ED51EF5018081918172
:104E40000F948C4C8983002311F0F7018083BE01FD
:104E50006F5F7F4FC4010F94DA01F501808191816A
:104E6000019691838083FFEFEF1AFF0AEC14FD0493
:104E700021F780E00F90DF91CF910F91FF90EF909D
:104E8000DF90CF90BF90AF909F908F9008959091BA
:104E9000D10095FD0CC09091D00095FF08C0809383
:104EA000D6008091D00080648093D0000895209136
:104EB000D3062F5F2F770FB607FC27C09091D4063B
:104EC000921328C09091D00095FF1EC09091D406F7
:104ED0004091D306941306C09091D1009F7D90938A
:104EE000D10012C0E92FF0E0ED52F94F32819F5FFF
:104EF0009F773093D6009093D4063091D0003064E1
:104F00003093D000491741F3D9CF9091D406921332
:104F100001C0FBCFE091D306F0E0ED52F94F828360
:104F20002093D3068091D10080628093D1000895B0
:104F30008091C7079091C8072FEF3FEF981751F066
:104F4000E92FF0E0E953F84F228130E09F5F9F7333
:104F50009093C807C90108951F920F920FB60F9240
:104F600011240BB60F922F938F939F93EF93FF9380
:104F70008091D4062091D306821306C08091D1007F
:104F80008F7D8093D10012C0E82FF0E0ED52F94FF1
:104F900092818F5F8F779093D6008093D406909103
:104FA000D00090649093D000281741F3FF91EF91C7
:104FB0009F918F912F910F900BBE0F900FBE0F906E
:104FC0001F9018951F920F920FB60F9211240BB6D7
:104FD0000F920F931F932F933F934F935F936F9372
:104FE0007F938F939F93AF93BF93CF93DF93EF9371
:104FF000FF93C091D6000091C807D091C70711E078
:105000001D0F1F739091D206913108F09FC0E92FB8
:10501000F0E08827E15FF74D8F4F0D94574D202822
:105020004F285E286D287428A6287828A6287C2872
:105030008028A628842888288C289328A6289E289B
:10504000C03229F028F5CA3011F0CD3031F5011702
:1050500031F0ED2FF0E0E953F84FC283D12FD09318
:10506000C707FF91EF91DF91CF91BF91AF919F91D2
:105070008F917F916F915F914F913F912F911F91F0
:105080000F910F900BBE0F900FBE0F901F901895B1
:10509000CD3481F081E0CE3471F080E10CC0CA33B0
:1050A00038F4C033A0F6C03291F2CD32B1F7CFCF91
:1050B000CD3499F782E08093D206C9CFC13359F03D
:1050C00018F4C03221F2E9CF88E0C433A1F38BE0B9
:1050D000C83389F3E2CF83E0EECF84E0C03359F3E5
:1050E00086E0C13341F3D9CF85E0C833B1F6E3CFD1
:1050F00087E0C23391F6DFCF89E0C13371F6DBCFB1
:105100008AE0C03351F6D7CF8CE0C73331F6D3CF26
:105110008DE0C63311F6CFCFC03209F498CF8EE0C0
:10512000C33549F2BACF80ED8C0F8A3008F08FCFAB
:105130009FE09093D2068093D10689CFCA3019F0B0
:10514000CD3009F084CF1092D20681CFCA3019F049
:10515000CD3009F07CCF8091DF1A8823A1F39730FE
:1051600089F038F4953079F71092500210928C1132
:10517000EACF9A3059F09F3031F78091D1060E94E2
:10518000D325E1CF81E08093E608DDCF81E08093F5
:10519000E508D9CF9091C10095FD0CC09091C00059
:1051A00095FF08C08093C6008091C0008064809302
:1051B000C000089520914F062F5F2F770FB607FC90
:1051C00027C090915006921328C09091C00095FF7F
:1051D0001EC09091500640914F06941306C09091C6
:1051E000C1009F7D9093C10012C0E92FF0E0E15B08
:1051F000F94F32819F5F9F773093C600909350069E
:105200003091C00030643093C000491741F3D9CFCA
:1052100090915006921301C0FBCFE0914F06F0E051
:10522000E15BF94F828320934F068091C100806239
:105230008093C1000895CF93DF93EC01FE01849128
:105240002196882319F00E94CA28F8CFDF91CF91C8
:105250000895CF92DF92EF92FF921F93CF93DF9347
:10526000CDB7DEB76C970FB6F894DEBF0FBECDBFDB
:105270000E94357183E50E94EF20882309F4A0C0C5
:10528000109159020E944B20809359021092A70856
:105290000E9413E5809159028230C1F034F487FFF7
:1052A00047C081E08093590243C08330D1F7123068
:1052B00009F446C084E09FE00E941B2985EE9EE031
:1052C0000E941B2981E0809359026CC088E50E94EE
:1052D000EF208823D1F00E9473206B017C0120E035
:1052E00030E042E852E40F94C04F181634F0C12C5D
:1052F000D12C82E8E82E82E4F82EC0925502D0929A
:105300005602E0925702F092580282E50E94EF2086
:10531000882331F00E946F209093C5078093C407C3
:105320008091BA13882321F060E080E00E948AE532
:1053300080E00E945C8710928E110E9413E532C0BB
:1053400081E08093A7080E9413E580E1E9E7F2E09D
:10535000DE01119601900D928A95E1F72DEC3CEC5F
:105360004CEC5DE369817A818B819C810F945F4D68
:1053700069837A838B839C83198A1A8A1B8A1C8A85
:105380001D8A1E8A1F8A188E198E1A8E1B8E1C8EDD
:105390009E012F5E3F4F40E065E772E0CE0101962F
:1053A0000E945D846C960FB6F894DEBF0FBECDBF31
:1053B000DF91CF911F91FF90EF90DF90CF900895F4
:1053C00087E50E94A120882309F47CCFEBCFCF93FF
:1053D000C62F0E941B298C2FCF910C9423D40E949E
:1053E000CA288FE29BE00C941B2988E698E00E9473
:1053F0001B2980918B09882371F0999AA1981092AA
:105400008B091092E1091092E2091092E3091092BF
:10541000E4091092E00908950F931F93CF938C0134
:10542000C62F82EF97E00E941B29C8010E941B290A
:10543000CC2331F08AE0CF911F910F910C94CA28B0
:10544000CF911F910F9108950F931F93CF938C01CC
:10545000C62F60E08AE098E00E940C2AC8010E94F2
:105460001B29CC2331F08AE0CF911F910F910C942E
:10547000CA28CF911F910F91089561E082E198E0D1
:105480000C94242AEF92FF920F931F93CF937C01E9
:105490008B01C42F60E08AE098E00E940C2AC701CB
:1054A0000E941B2980E20E94CA28C8010E941B2971
:1054B000CC2319F08C2F0E94CA288AE0CF911F912B
:1054C0000F91FF90EF900C94CA28DF92EF92FF9219
:1054D0000F931F93CF93DF93D82E7B018A01E901AD
:1054E0000E943D2AD092BD1240E0B70187E793E3C6
:1054F0000E94422A0115110531F040E0B80180E711
:1055000093E30E94422A209731F040E0BE0180E7F9
:1055100093E30E94422A61E08BE693E3DF91CF910F
:105520001F910F91FF90EF90DF900C94242AAF927F
:10553000BF92CF92DF92EF92FF920F931F93CF9380
:10554000DF938DED97E00E941B2960919B0870917D
:105550009C0880919D0890919E0845E00E9463D52B
:105560008AEC97E00E941B29C0E0D9E0D15021F0DD
:1055700080E20E94CA28FACF8C2F0E9423D4CF5FEA
:10558000C53099F78AE00E94CA280CE412E1C0E015
:1055900080E20E94CA288C2F0E9423D45801D5E0B3
:1055A00080E20E94CA28F501C080D180E280F380A9
:1055B000A7019601C701B6010F94525081112CC06A
:1055C00020E030E0A901C701B6010F94C04F87FD6C
:1055D00003C08BE20E94CA2845E0C701B6010E94C1
:1055E00063D5D15084E1A80EB11CD111D9CF8AE086
:1055F0000E94CA28CF5F0C5F1F4FC53049F68AE072
:10560000DF91CF911F910F91FF90EF90DF90CF909E
:10561000BF90AF900C94CA28F12C80E20E94CA2857
:10562000F3948DE3F8E0FF12F9CFDBCF811107C0CF
:1056300083E890E10E941B298AE00C94CA2887E83D
:1056400090E1F8CFCF936FE670E10F948B09C09192
:105650007A11C05D86E690E10E941B298C2F0E9482
:10566000CA2882E690E10E941B2980917A11CF918D
:105670000C94162B83EC97E00C941B298DEB97E090
:105680000C941B29811102C00C943E2B0895CF93DA
:1056900084E50E94EF20C091BA138823E9F00E94AC
:1056A0004B20C82F8230C4F00E943E2B8DE40E9414
:1056B000CA286091C1077091C20790E080E00F9402
:1056C0004E0289EC90E10E941B298C2F0E94AB1D99
:1056D0008AE00E94CA28CFEF8C2FCF9108950F93B4
:1056E0001F93CF93811116C0C42F8B010E943E2BB4
:1056F00086EC90E10E941B29C8010E941B29CC2343
:1057000049F08AE30E94CA288AE0CF911F910F9145
:105710000C94CA28CF911F910F910895AF92BF9218
:10572000CF92DF92EF92FF920F931F93CF93DF936D
:105730006091BA1370E084E50E94FC218230C0F0D1
:105740008FE30E94CA2884E50E94CA2882E49FE071
:105750000E941B2987E39FE0DF91CF911F910F915A
:10576000FF90EF90DF90CF90BF90AF900C941B29EB
:105770009927EC01CC0FDD1FCC0FDD1FFE01EF5E82
:10578000F64FA080B180C280D3808BE40E94EF20CE
:10579000882339F10E9473207B018C0120E030E0E6
:1057A000A9010F94C04F87FD0AC020E030E040E21D
:1057B00051E4B701C8010F946E461816A4F48FE3A4
:1057C0000E94CA288BE40E94CA2882E49FE00E94BB
:1057D0001B298AE39FE00E941B2987E39FE00E9428
:1057E0001B29750186019501A601B701C8010F9417
:1057F0006E46882351F00E943571CF5ED64FA701C7
:10580000B801488359836A837B838091BA0790915A
:10581000BB07A091BC07B091BD07892B8A2B8B2BAE
:10582000D9F50E943E2B86E59FE00E941B2980E26D
:105830000E94CA2880E30E94CA288AE30E94CA28DC
:1058400060911109709112098091130990911409C6
:1058500042E00E9463D580E20E94CA2881E30E9450
:10586000CA288AE30E94CA28609115097091160916
:10587000809117099091180942E00E9463D58AE04F
:10588000DF91CF911F910F91FF90EF90DF90CF901C
:10589000BF90AF900C94CA28DF91CF911F910F91C8
:1058A000FF90EF90DF90CF90BF90AF9008952F9230
:1058B0003F924F925F926F927F928F929F92AF92A0
:1058C000BF92CF92DF92EF92FF920F931F93CF93ED
:1058D000DF93CDB7DEB76D970FB6F894DEBF0FBE7E
:1058E000CDBF83E50E94A120182F3090AF138823ED
:1058F00019F00E945F20382E8091790290917A02EF
:10590000A0917B02B0917C028A8F9B8FAC8FBD8F60
:1059100080917D0290917E02A0917F02B0918002E1
:105920008E8B9F8BA88FB98F80918102909182027C
:10593000A0918302B09184028A8B9B8BAC8BBD8B30
:10594000112329F0311003C080E00E943B23809195
:10595000BA079091BB07A091BC07B091BD0725E1A4
:10596000B695A795979587952A95D1F74C015D0136
:10597000E1E08E229924AA24BB240E945423882388
:1059800009F4C5C083E40E94A120882309F49EC0C5
:105990000E9473202B013C018CE492E19987888757
:1059A0009F838E83B5E0BD8300E0212CE8ECEE8779
:1059B000F2ECFF871A861B8628EC2C8782E48D8701
:1059C000AE81BF81B98BA88B15E0E889F989C190B8
:1059D000D190E190F190F98BE88B2A853B854C853D
:1059E0005D85C701B6010F946E4687FF04C0CA8665
:1059F000DB86EC86FD86202F322D4E855F85C70124
:105A0000B6010F94C04F181624F40C2D2D2CEE86E1
:105A1000FF861150D1F6FD81F150FD838E819F816B
:105A200044969F838E83F111CBCF202F322D4E854C
:105A30005F856A857B858C859D850F94604D20E010
:105A400030E040E05FE30F94D446A30192010F944D
:105A5000604D2B013C012DEB37E346E855EB0F94ED
:105A6000C04F87FD0AC02DEB37E346E855E3C3017D
:105A7000B2010F946E4618164CF580E00E943B234D
:105A800010E0E884F98400E0D7016D917D918D915B
:105A90009D917D016D01B4E0CB1AD108A301920163
:105AA0000F945F4DF6016083718382839383602F2F
:105AB000812F0F94AC0A0F5F053031F71F5F888587
:105AC00099854496998788871530D9F689288A2838
:105AD0008B2851F00E945423882331F08AE09BE008
:105AE0000E941B290E94972A8AE50E94A1208823F0
:105AF00051F00E94732069837A838B839C83CE014B
:105B000001960F945B0E832D0E943B230CC0311035
:105B100004C089288A288B2839F30E943E2B80E212
:105B20009BE00E941B29332051F08091AF1381111B
:105B300006C00E943A2B8BEE9AE00E941B290E941D
:105B40003E2B8DED9AE00E941B298091AF130E949D
:105B5000162B0E943E2B80ED9AE00E941B29C090DC
:105B6000AB13D090AC13E090AD13F090AE1320E0E7
:105B700030E0A901C701B6010F94C04F18160CF010
:105B800051C042E0C701B6010E9463D50E9471C7AF
:105B90002A8D3B8D4C8D5D8D6091790270917A02DA
:105BA00080917B0290917C020F946E4681111FC000
:105BB0002E893F89488D598D60917D0270917E02BA
:105BC00080917F02909180020F946E4681110FC0E8
:105BD000209181023091820240918302509184028F
:105BE0006A897B898C899D890F946E4681110E94F8
:105BF000DB8F6D960FB6F894DEBF0FBECDBFDF9181
:105C0000CF911F910F91FF90EF90DF90CF90BF90B9
:105C1000AF909F908F907F906F905F904F903F904C
:105C20002F9008958BEC9AE00E941B29B1CFCF935F
:105C3000C82F82E0C11184E060E00F94AF090E9498
:105C40003E2B87E298E0CC2311F08CE398E0CF91D3
:105C50000C941B29CF92DF92EF92FF926A017B0195
:105C60000E941B2942E0C701B601FF90EF90DF9030
:105C7000CF900C9463D5CF92DF92EF92FF92CF93A7
:105C80008091BA07887809F059C08091BB0787FDD9
:105C900055C08091BC07867009F050C00E943E2B11
:105CA00085EB90E10E941B29E091BA13F0E0EF50E0
:105CB000F54F808181113CC083E890E10E941B294F
:105CC000E091BA1384E0E89FF0011124E455F74F06
:105CD000408151816281738188EA90E10E942A2E7D
:105CE00085EA90E10E941B29E091BA13F0E0EF549D
:105CF000F74FF0808CE990E10E941B296F2D70E036
:105D000090E080E00F94B8028AE890E10E941B299D
:105D10008091890781110FC083E890E10E941B29BF
:105D20008AE0CF91FF90EF90DF90CF900C94CA283B
:105D300087E890E1C3CF87E890E1F0CF88E40E9444
:105D4000A120882321F00E945F2080938907C090C2
:105D5000BA07D090BB07E090BC07F090BD0781E187
:105D6000F694E794D794C7948A95D1F781E0C82236
:105D7000DD24EE24FF2483E50E94A120C82FCD2836
:105D8000CE28CF2811F4882341F00E94C025CC23CF
:105D900021F00E945F208093F10A84E40E94A120F8
:105DA000882311F10E9473206093AC087093AD08B2
:105DB0008093AE089093AF0880E50E94A1208823CD
:105DC000C9F00E946F209C013327233031051CF05D
:105DD0002730310579F48093B108CF91FF90EF908F
:105DE000DF90CF900C94FE258CE40E94A1208111BD
:105DF000D9CFE2CFCF91FF90EF90DF90CF90089571
:105E0000FF920F931F93CF93DF93082FF62E41E05D
:105E100068E97EE00E946F2BC9E7D8E110E0F11637
:105E200019F08FEFF81235C0802F0E94422B8FE8B7
:105E30009EE00E941B29812F0E94AB1D4B855C8533
:105E40006D857E8582E796E30E942A2E2CEA35EC4A
:105E500047E25EE36F85788989899A890F945A4E63
:105E6000AB01BC018CE89EE00E942A2E2CEA35ECA6
:105E700047E25EE36B897C898D899E890F94D446C5
:105E8000AB01BC0189E89EE00E942A2E8AE00E94B4
:105E9000CA286796113031F4DF91CF911F910F918D
:105EA000FF90089511E0BBCFCF93DF93C82F6AE72F
:105EB0007EE00F948B098C2F0E94422B61E081E7DA
:105EC0009EE00E94E729C4E3D2E14C855D856E85A2
:105ED0007F8585E69CE10E942A2E488959896A8936
:105EE0007B8982E69CE10E942A2E89EA9CE10E943D
:105EF0001B296C897D898E899F8943E00E9463D527
:105F00008AE0DF91CF910C94CA280E942A2E8AE061
:105F10000C94CA28CF93DF93D82FC62F6DEC7EE068
:105F20000F948B094091C1115091C2116091C3111E
:105F30007091C41185EC9EE00E942A2E4091C511FB
:105F40005091C6116091C7117091C81182E69CE111
:105F50000E942A2E4091C9115091CA116091CB1113
:105F60007091CC1189EA9CE10E942A2E8AE00E945D
:105F7000CA28C7FF2CC08D2F0E94422B60E08DEBFA
:105F80009EE00E94E7294091CD115091CE11609181
:105F9000CF117091D0118AEB9EE00E94852FC7FF30
:105FA00018C08D2F0E94422B61E08DEB9EE00E9475
:105FB000E7294091D1115091D2116091D311709184
:105FC000D4118AEB9EE0DF91CF910C94852FCC23E6
:105FD00091F2C13031F3DF91CF9108952F923F922A
:105FE0004F925F926F927F928F929F92AF92BF92E9
:105FF000CF92DF92EF92FF920F931F93CF93DF9395
:1060000000D0CDB7DEB70E94472B87FDC5C0909169
:10601000BA0794FD21C09091BC0797FD1DC09091D7
:10602000BD079370C9F4682F81E00F900F900F9017
:10603000DF91CF911F910F91FF90EF90DF90CF9064
:10604000BF90AF909F908F907F906F905F904F9098
:106050003F902F900C948A2F9BEB292E92E0392EA3
:1060600029EAE22E21E1F22E19828D5F282F30E0FD
:10607000C901880F991F880F991FFC01EF53FE4E2D
:106080006F018C010B521E4E9C012C5D374F3B83E0
:106090002A83F10181911F010E94EF20882351F092
:1060A000F981F33031F10E947320F701608F718F15
:1060B000828F938FF981FF5FF98324E0E20EF11C58
:1060C000F43039F70F900F900F90DF91CF911F911F
:1060D0000F91FF90EF90DF90CF90BF90AF909F9087
:1060E0008F907F906F905F904F903F902F900C9487
:1060F000FF850E9473204B015C0120E030E040EA04
:1061000051E40F946E4687FF41C0A5019401F6014A
:1061100060817181828193810F945A4E2B013C01E1
:10612000AC019B016091FE0A7091FF0A8091000B07
:106130009091010B0F94D4466093FE0A7093FF0A6E
:106140008093000B9093010BA3019201F8016081F1
:106150007181828193810F94D446F80160837183A9
:1061600082839383EA81FB81608171818281938143
:106170000F947346A30192010F94D4460F94D34E0B
:10618000EA81FB816083718382839383F60180823D
:106190009182A282B3828ECF0F900F900F90DF91E9
:1061A000CF911F910F91FF90EF90DF90CF90BF9014
:1061B000AF909F908F907F906F905F904F903F90A7
:1061C0002F900895CF93DF9362EB7EE00F948B09BD
:1061D000C2E6D8E14B855C856D857E8589EA9EE0C7
:1061E0000E942A2E2CEA35EC47E25EE36F8578891F
:1061F00089899A890F945A4EAB01BC0186EA9EE0C8
:106200000E942A2E2CEA35EC47E25EE36B897C89FA
:106210008D899E890F94D446AB01BC0183EA9EE030
:10622000DF91CF910C94852FFF920F931F93CF9303
:10623000DF9363E67EE00F948B098CE59EE00E947D
:106240001B29C6EFD8E0488159816A817B8189E5A5
:106250009EE00E942A2E488559856A857B858FE6B7
:1062600096E30E942A2E4C815D816E817F818AEBAC
:106270009EE00E942A2E6C857D85072E000C880BDF
:10628000990B0F947546AB01BC0182E796E30E941F
:106290002A2E6E857F85072E000C880B990B0F9494
:1062A0007546AB01BC0186E59EE00E942A2E6889F6
:1062B0007989072E000C880B990B0F947546AB015A
:1062C000BC0183E59EE00E942A2E6A897B89072E05
:1062D000000C880B990B0F947546AB01BC0180E54F
:1062E0009EE00E942A2E6C898DE49EE00E94E729A0
:1062F0006D898AE49EE00E94E72909E119E0F8012E
:10630000F28087E49EE00E941B298F2D0E94B21D1F
:10631000F801618170E090E080E00F947346AB017A
:10632000BC0184E49EE00E942A2E4E895F89688D1C
:10633000798D89EA9CE1DF91CF911F910F91FF90B8
:106340000C94852FCF92DF92EF92FF92CF93DF9341
:1063500000D01F92CDB7DEB781E50E94A12088232F
:1063600009F468C08091BA130E943BD4811157C0D0
:1063700080E1E9E7F2E0A9E9B1E101900D928A95A7
:10638000E1F720910C0930910D0940910E095091CF
:106390000F09609181027091820280918302909135
:1063A00084020F94604D6093810270938202809307
:1063B000830290938402C0907002D0907102E090AA
:1063C0007202F0907302A70196010F94C04F181645
:1063D00044F4C0928102D0928202E0928302F09251
:1063E000840220E030E040E05FE36091DD117091D5
:1063F000DE118091DF119091E0110F94D4466983F2
:106400007A838B839C83CE0101960E944C880E94E4
:1064100035710E9457D485EA91E10E94FFD40F9014
:106420000F900F900F90DF91CF91FF90EF90DF9042
:10643000CF90089583E50E94EF208823F1F00E9419
:1064400073206B017C0120E030E0A9010F946E46BF
:1064500087FD03C120E030E048E453E4C701B60102
:106460000F94C04F18160CF4FCC0C092F608D092DE
:10647000F708E092F808F092F90882E40E94EF2011
:106480008823F9F00E9473206B017C0120E030E04A
:1064900040E251EC0F946E4687FDEAC020E030E008
:1064A00040E251E4C701B6010F94C04F18160CF436
:1064B000E6C0C092FE08D092FF08E0920009F09278
:1064C000010985E40E94EF208823F1F00E947320E7
:1064D0006B017C0120E030E0A9010F946E4687FD3E
:1064E000D5C020E030E048E453E4C701B6010F9482
:1064F000C04F18160CF4CEC0C092FA08D092FB0818
:10650000E092FC08F092FD0880E50E94EF208823CD
:1065100099F00E9473200F94CC4E693185E1780781
:1065200014F068E175E16A30710514F46AE070E016
:10653000709303096093020987E40E94EF20882387
:1065400089F00E9473200F94CC4E6536710514F0CB
:1065500064E670E077FF02C070E060E070930509C8
:106560006093040982E50E94EF20882399F00E943D
:1065700073200F94CC4E693185E1780714F068E1FF
:1065800075E16A30710514F46AE070E070930709F0
:106590006093060985E50E94EF20882399F00E9408
:1065A00073200F94CC4E693185E1780714F068E1CF
:1065B00075E16A30710514F46AE070E070930909BE
:1065C000609308098AE50E94EF20882351F00E9419
:1065D000732060930C0970930D0980930E099093BA
:1065E0000F09109219098CE40E94EF20882379F09A
:1065F0000E946F208230910550F480931A0991E037
:106600002091BA13281708F090E090931B0981E4B9
:106610000E94A120882321F00E945F2080931B0903
:1066200084E50E94A1208823F1F180919A0790913E
:106630009B07892BE1F10E946F208230910588F53C
:106640002091BA132817190661F18F5F80931909F9
:106650000E94EFE710921909E2CEC12CD12C7601ED
:1066600004CFC12CD12C38E4E32E33E4F32EFDCE3D
:10667000C12CD12C20E2E22E21ECF22E1ACFC12C1B
:10668000D12C90E2E92E91E4F92E13CFC12CD12C1C
:10669000760132CFC12CD12C88E4E82E83E4F82E89
:1066A0002BCF1092190981E00E941431B8CE0E94BC
:1066B000EFE7B5CECF93DF936BEC7DE00F948B09C2
:1066C0006091BD117091BE118091BF119091C01168
:1066D0000F947346AB01BC0182EC9DE00E942A2E10
:1066E0004091F5115091F6116091F7117091F811E8
:1066F0008FEB9DE00E942A2E4091F9115091FA11E2
:106700006091FB117091FC118CEB9DE00E942A2E90
:10671000C2EFDAE0488159816A817B8185E69CE19C
:106720000E942A2E4C815D816E817F8182E69CE1F0
:106730000E942A2E488559856A857B8589EA9CE1D5
:106740000E942A2E4C855D856E857F858AEB9EE0B2
:10675000DF91CF910C94852F62E77DE00F948B0938
:106760004091E9115091EA116091EB117091EC1197
:1067700089E69DE00E942A2E4091ED115091EE1184
:106780006091EF117091F01186E69DE00E942A2E33
:106790004091F1115091F2116091F3117091F41147
:1067A0008CEB9DE00C94852FCF93C82F6EE47DE099
:1067B0000F948B094091D5115091D6116091D7114A
:1067C0007091D81185E49DE00E942A2E4091D91144
:1067D0005091DA116091DB117091DC1182E69CE13D
:1067E0000E942A2E4091DD115091DE116091DF113F
:1067F0007091E01189EA9CE10E94852FC11102C0CD
:106800000E943E2B60E08CE39DE00E94E7294091CE
:10681000E1115091E2116091E3117091E4118AEB62
:106820009EE00E94852FC11102C00E943E2B61E0B4
:106830008CE39DE00E94E7294091E5115091E6111B
:106840006091E7117091E8118AEB9EE0CF910C9472
:10685000852F1F93CF93DF93182F60E27DE00F9475
:106860008B09C9EAD1E1688179818A819B810F9482
:106870007346AB01BC0187E19DE00E942A2E6C812A
:106880007D818E819F810F947346AB01BC0182E6AE
:106890009CE10E942A2E688579858A859B850F94C4
:1068A0007346AB01BC0189EA9CE10E94852F812FD0
:1068B0000E94422B60E08EE09DE00E94E7296C85FB
:1068C0007D858E859F850F947346AB01BC018AEB55
:1068D0009EE00E94852F812F0E94422B61E08EE076
:1068E0009DE00E94E729688979898A899B890F94AC
:1068F0007346AB01BC018AEB9EE0DF91CF911F9103
:106900000C94852FCF93DF93C82F811113C040E0E3
:106910006CEF7CE080E00E946F2B8091B9138111B5
:1069200004C08FEE9CE00E941B298AE00E94CA28C6
:106930000E943E2BD091B91386EE9CE00E941B2949
:106940008D2F0E94B21D8AE00E94CA288C2F0E94BF
:10695000422B8DED9CE00E941B2980E00E94AB1D24
:106960004091B1135091B2136091B3137091B4136D
:106970008AED9CE00E94852F8C2F0E94422B8DED8A
:106980009CE00E941B2981E00E94AB1D4091B51341
:106990005091B6136091B7137091B8138AED9CE0D3
:1069A000DF91CF910C94852F67EC7CE00F948B09DD
:1069B00080EC9CE00E941B29409197085091980818
:1069C0006091990870919A0889EA9CE10C94852F4E
:1069D000CF92DF92EF92FF920F931F93CF93DF93AB
:1069E0000BEB12E0C0E0D1E0F80181918F010E9431
:1069F000A120882399F00E94357180919A07909187
:106A00009B0740E050E0BA01892B21F00E947320DF
:106A1000AB01BC018C2F0E941B24D0E0CF5FC330A0
:106A200019F786E40E94A1208823E1F10E943571C4
:106A30000E9473206B017C0120E030E040E85FE3BE
:106A40000F94C04F18163CF120E030E0A901C701B7
:106A5000B6010F946E4687FF03C0C12CD12C76017E
:106A600020E030E04FE753E4C701B6010F94D4466D
:106A700020E030E040E05FE30F94604D0F94D34E90
:106A8000862FDF91CF911F910F91FF90EF90DF90B4
:106A9000CF900C946324C12CD12C80E8E82E8FE396
:106AA000F82EDECFDD2309F43EC08BEA9CE00E9485
:106AB0001B2980912102811104C088EA9CE00E9478
:106AC0001B298FE99CE00E941B296091210270E044
:106AD00090E080E00F94734620E030E04FE753E40D
:106AE0000F945A4EAB01BC018BE79CE00E942A2E0A
:106AF0008EE59CE00E941B298CE39CE00E941B29F0
:106B0000C9E7D8E004E31CE0499159916991799172
:106B1000F801859194910E94852F0E5F1F4FF8E038
:106B2000C538DF0789F7DF91CF911F910F91FF9053
:106B3000EF90DF90CF900895CF93DF93EB010E9409
:106B40001B29BE01DD0F880B990BDF91CF910D94AE
:106B5000B8020E949C358AE00C94CA289F92AF929A
:106B6000BF92CF92DF92EF92FF920F931F93CF933A
:106B7000DF9300D000D01F921F92CDB7DEB760E048
:106B800083E50E941922863028F08DE19CE00E9466
:106B90001B2947C0833009F4E1C1B0F4813021F1F1
:106BA000823009F453C08AE09CE00E941B290E94B5
:106BB00054238823A1F08091AF130E94162B0E94CA
:106BC000972A0E94DB8F2DC0843009F411C28530D2
:106BD00051F780E00E943B230E941B23F2CF8CEFF1
:106BE0009BE00E941B29EDCF0E941B2310920702FD
:106BF000109206028091BA079091BB07A091BC0742
:106C0000B091BD071DE0B695A795979587951A9504
:106C1000D1F780FD18C08AEE9BE09093030B809320
:106C2000020B28960FB6F894DEBF0FBECDBFDF91E2
:106C3000CF911F910F91FF90EF90DF90CF90BF9079
:106C4000AF909F90089580EF9BE0E7CF8091060280
:106C50009091070297FF03C081EC9BE098CF0097CB
:106C600009F096C01D821E821F8218868DEC9CEC56
:106C7000ACE4BEE389839A83AB83BC83BE016B5FC4
:106C80007F4FCE0101960E944F898091060290911C
:106C90000702893191050CF0A5C021E020935B0229
:106CA0009C012F5F3F4F309307022093060265E05F
:106CB0000F94214D382F80FF03C024E0291B922F11
:106CC00084E09802F0011124EC50F54E608171814E
:106CD0008281938124E03202F0011124E052F54ECA
:106CE0002081318142815381EDECCE2EECECDE2E01
:106CF000ECE4EE2EEEE3FE2ECD82DE82EF82F8860D
:106D000019821A821B821C82FE0131966F01E12CCE
:106D1000F12C00EA10E40E94758819821A821B8205
:106D20001C82B601CE0105960E944F890091060291
:106D30001091070289E1F82EE12C0931110514F4B4
:106D4000F02EE12E6F2D7E2D8AE59BE00E949C3572
:106D500069E170E085E59BE00E94A93510161106F7
:106D60000CF02FCF1F9289E18F93EF92FF928EE369
:106D70009BE09F938F938CE49BE09F938F931F9254
:106D80000F94E5050FB6F894DEBF0FBECDBF19CF47
:106D9000815065E00F94214D80FF03C024E0291B42
:106DA000922F25E09202F0011124E80FF11D87FDDA
:106DB000FA95EE0FFF1FEE0FFF1FE45BFD4E809173
:106DC000810290918202A0918302B091840280831B
:106DD0009183A283B38360E080E00F94AC0A1092A9
:106DE0005B0253CF80E090E0A0EAB0E480938102A0
:106DF00090938202A0938302B093840285E792E08D
:106E00000E944C880E9435718FEF9FEF909307028C
:106E1000809306028DEA9BE00E941B2960E08BE9CB
:106E20009BE00E942B9D85E99BE00E94EDBE81E0E6
:106E30000E943B230E945423882309F471C010E070
:106E400000E0E12C54E0B52E65E0C62E72E8D72EA6
:106E5000F12CF02FF170AF2E9E2C9F0C8B2D8F19E3
:106E6000A11001C08F2DF801C89EE00DF11D112465
:106E7000EE0FFF1FEE0FFF1FE45BFD4E20E030E042
:106E80004AE754E460817181828193810F94D446F2
:106E90000F94CC4E70936E1A60936D1AC092611A63
:106EA000D092641A892D90E08058974F880F991FCF
:106EB000092E000CAA0BBB0B8093651A9093661ADF
:106EC000A093671AB093681A81E19AE10E946B9BC4
:106ED000F39425E0F212C0CFE20E0F5F1F4F89E15D
:106EE000E812B6CF83E090E090936E1A80936D1A0B
:106EF000F092611AD092641A85E490E1A0E0B0E0CB
:106F00008093651A9093661AA093671AB093681AD3
:106F100081E19AE10E946B9B81E00E943B2306CFB6
:106F200082E090E090936E1A80936D1A85E08093D2
:106F3000611A82E88093641A85E490E1A0E0B0E0F1
:106F40008093651A9093661AA093671AB093681A93
:106F500081E19AE10E946B9B80E0DFCF89E40E948F
:106F6000EF20882371F00E946F20182F853068F081
:106F700064E070E082E89BE00E949C358FE79BE034
:106F800006CE8AE40E94EF294CCE8AE40E94EF20CC
:106F90008823B9F30E946F20082F853048F064E001
:106FA00070E08CE69BE00E949C3589E69BE0EFCD8B
:106FB0008AE50E94EF208823C9F00E94732025E013
:106FC0001202F0011124E00FF11D07FDFA95EE0FFA
:106FD000FF1FEE0FFF1FE45BFD4E60837183828312
:106FE0009383602F812F0F94AC0AEBCD8AE5CACF33
:106FF0008AE50E94EF208823C9F30E9473206093E2
:107000009B0870939C0880939D0890939E08D9CD0F
:107010002F923F924F925F926F927F928F929F92A8
:10702000AF92BF92CF92DF92EF92FF920F931F9396
:10703000CF93DF93CDB7DEB7CB58D1090FB6F89415
:10704000DEBF0FBECDBF8AEB9AE00E941B2987E00E
:107050000E946CA181116EC084E50E94EF208823FC
:1070600029F00E946F2060E00E948AE580E090E0B5
:10707000A0E8BFE389839A83AB83BC838D839E831F
:10708000AF83B8878DEC9CECACE4BEE389879A872C
:10709000AB87BC8780E090E0A0E2B1E48D879E875B
:1070A000AF87B88B8CE390E09A8B898B8DEC90E066
:1070B0009C8B8B8B8DEC9CECACECBEE38D8B9E8B18
:1070C000AF8BB88F80E090E0A0EEBFE3898F9A8FFE
:1070D000AB8FBC8F1BA61CA64AE959E969E97EE380
:1070E0008FE40E94FC206D8F7E8F8F8F98A360E0CD
:1070F00083E40E94252289A360E08BE40E9425227C
:107100008AA382E40E94EF20882381F10E946F20ED
:10711000009761F19C01285231092536310520F193
:107120006CE870E08CE89AE00E949C3587E89AE071
:107130000E941B29C557DF4F0FB6F894DEBF0FBE64
:10714000CDBFDF91CF911F910F91FF90EF90DF9016
:10715000CF90BF90AF909F908F907F906F905F90F7
:107160004F903F902F9008959A8B898B8CE40E94CA
:10717000EF208823E1F00E9473206B017C01C98617
:10718000DA86EB86FC8620E030E0A9010F94C04F40
:1071900087FD0AC020E030E040E050E4C701B601BE
:1071A0000F946E4618161CF48FE59AE0C1CF81E566
:1071B0000E94A120882331F180919A0790919B072A
:1071C000892BE9F00E9473206B017C01CD82DE8265
:1071D000EF82F8862DEC3CEC4CE45DE30F94C04F5D
:1071E00087FD0AC020E030E040E751E4C701B60166
:1071F0000F946E46181634F48EE29AE099CF83E02D
:107200009AE096CF83E50E94EF208823E9F00E9460
:1072100073206B017C01CD8ADE8AEF8AF88E2DEC1B
:107220003CEC4CEC5DE30F94C04F87FD0AC020E0BE
:1072300030E040E050E4C701B6010F946E461816E6
:107240001CF48CED99E074CF80E50E94A120882386
:1072500041F180919A0790919B07892B19F484EA58
:1072600099E066CF8BA58F5F8BA70E9473206B017F
:107270007C01CD86DE86EF86F88A20E030E0A90129
:107280000F94C04F87FD0AC020E030E048EC51E485
:10729000C701B6010F946E4618161CF48CE799E0EE
:1072A00047CF86E40E94EF208823E9F00E947320F4
:1072B0006B017C01C98EDA8EEB8EFC8E20E030E013
:1072C00040E85FE30F94C04F87FD0AC020E030E044
:1072D00040E850E4C701B6010F946E4618161CF43E
:1072E00083E599E025CFC98CDA8CEB8CFC8C8D88FA
:1072F0009E88AF88B88CA7019601C701B6010F948C
:10730000D4469B01AC0160E070E084E490E40F940B
:107310005A4E29813A814B815C810F94D4462B01CE
:107320003C01A5019401C501B4010F94D446A70105
:1073300096010F94D4462CEE31E548EB5DE30F94B3
:107340005A4E9B01AC01C301B2010F94D44669832C
:107350007A838B839C8388E40E94EF20882379F0D2
:107360000E946F20009759F09C01255A3109283856
:10737000310518F085E299E0DBCE9C8B8B8B85E59F
:107380000E94A1208823C9F00F94C61261157105CF
:107390008105910511F00F94F44180919A07909125
:1073A0009B07892B09F10E947320609385077093D6
:1073B0008607809387079093880782E50E94A12023
:1073C0008823B9F080919A0790919B07892BA1F0AF
:1073D0000E946F20AD969FAF8EAFAD97181619061D
:1073E0008CF08DEB98E0A4CE60E070E088E492E44D
:1073F000DCCF81EF98E09CCE2AE130E0AD963FAF44
:107400002EAFAD9789E50E94EF20882399F10E9465
:1074100073202091B5123091B6124091B71250915D
:10742000B8120F945F4D6B017C0188E50E94EF203C
:10743000882349F10E9473202091B1123091B21239
:107440004091B3125091B4120F945F4D6BA37CA383
:107450008DA39EA3CFA2D8A6E9A6FAA6BE01695D18
:107460007F4FCE0183960E94858F811115C083E9DD
:1074700098E05ECEC0907D02D0907E02E0907F02C8
:10748000F0908002D2CF6091790270917A0280915F
:107490007B0290917C02DACF8091BA079091BB0772
:1074A000A091BC07B091BD0753E0B695A7959795FD
:1074B00087955A95D1F780959095A095B095817054
:1074C0000E943B2380E090E0A0EAB0E48DA79EA755
:1074D000AFA7B8ABCE018D960F94370D3091B9138D
:1074E000CA57DF4F3883C658D0401092B9130E9454
:1074F000097282E798E00E941B2989899A898A315A
:1075000091050CF04AC06091BA138B899C890E9446
:10751000902541E061E08091BA130E94BED88111AC
:1075200045C06FEF87E898E00E942B9D8CA58111E4
:1075300004C0CE0101960F94170D80E090E0A0EA00
:10754000B0E48093A1119093A211A093A311B093E2
:10755000A4111DA61EA61FA618AABE01635D7F4F1B
:1075600089E991E10E94B81DCA57DF4FB881C6581A
:10757000D040B093B9130E9409728AA18111DACD6B
:1075800010926B1810926A180E9496228091BA137A
:1075900060E090E00E949025CDCD0E947C2561E0C6
:1075A00081E00E9435D78111AECFBBCF109285020A
:1075B00010928602109287021092880285E892E06B
:1075C0000E9498848BA5882309F452C020E030E003
:1075D00040E751E46091E1117091E2118091E31173
:1075E0009091E4110F945A4E6DA77EA78FA798AB88
:1075F00080E1E9E7F2E0A9E9B1E101900D928A9515
:10760000E1F72D853E854F8558896091A5117091D0
:10761000A6118091A7119091A8110F94604D6093CD
:10762000A5117093A6118093A7119093A811CE0174
:107630008D960E941A8F2D853E854F8558896091C1
:10764000A5117091A6118091A7119091A8110F9486
:107650005F4D6093A5117093A6118093A71190932D
:10766000A8118CA5811104C0CE0101960F94170DAD
:10767000E0E8F7E085E0DF011D928A95E9F780E117
:10768000E9E7F2E0A9E9B1E101900D928A95E1F70D
:1076900089859A85AB85BC858093A1119093A211B1
:1076A000A093A311B093A4111DA61EA61FA618AAED
:1076B000BE01635D7F4F89E991E10E94B81DBE0163
:1076C000635E7F4F89E991E10E94B81DE1E5F0E03A
:1076D000EC0FFD1F3496C657DF4FF983E883CA5875
:1076E000D04089A1882309F4CDC38091790290917B
:1076F0007A02A0917B02B0917C02EF968CAF9DAF95
:10770000AEAFBFAFEF9780917D0290917E02A091C6
:107710007F02B0918002EB968CAF9DAFAEAFBFAF52
:10772000EB97A4EFBAE1AF96BFAFAEAFAF97312CF6
:10773000212CBFEFA496BFAFA497EFEFA896EFAFB1
:10774000A897FFEFC158DF4FF883CF57D0402FE401
:10775000C058DF4F2883C058D04033ECCF57DF4F9D
:107760003883C158D04007E481E090E0022C02C089
:10777000880F991F0A94E2F7C957DF4F99838883CE
:10778000C758D040A0E8B7E0E396BFAFAEAFE397ED
:10779000E0EEFAE1E196FFAFEEAFE19710E0C757F8
:1077A000DF4F2882C958D040E396AEADBFADE39716
:1077B0008D91E396BFAFAEAFE39790E0C957DF4F2F
:1077C000E881F981C758D0408E239F23892B09F087
:1077D000FAC0AF96AEADBFADAF97CD90DD90ED9056
:1077E000FC90E196AEADBFADE1978D919D910D906E
:1077F000BC91A02DE7968CAF9DAFAEAFBFAFE79722
:10780000A7019601EF966CAD7DAD8EAD9FADEF9764
:107810000F945F4D2B013C01E7962CAD3DAD4EAD75
:107820005FADE797EB966CAD7DAD8EAD9FADEB9701
:107830000F945F4D4B015C01A3019201C301B201A2
:107840000F94D4462B013C01A5019401C501B4015C
:107850000F94D4469B01AC01C301B2010F94604D5B
:107860000F940E504B015C01A70196016BA17CA106
:107870008DA19EA10F945F4D6B017C01E7962CAD0D
:107880003DAD4EAD5FADE7976FA178A589A59AA5EF
:107890000F945F4D2B013C01A7019601C701B60172
:1078A0000F94D4466B017C01A3019201C301B20184
:1078B0000F94D4469B01AC01C701B6010F94604DF3
:1078C0000F940E5020E030E040E751E40F945A4E00
:1078D000A50194010F94604D6B017C018090850798
:1078E00090908607A0908707B090880720E030E04E
:1078F00040E85FE3C501B4010F94C04F1816F4F4DB
:10790000C501B4010F94CC4E4B015C0160E070E006
:10791000CB01181419041A041B0434F40F94A54164
:10792000A50194010F94D44C0F9475469B01AC01B2
:10793000B601C7010F94604D6B017C019601A70150
:10794000C158DF4F6881CF57D040C058DF4F788192
:10795000C058D040CF57DF4F8881C158D040902FBA
:107960000F94C04F18167CF5A4961FAFA497C75765
:10797000DF4FB881C958D040A896BFAFA897CE575F
:10798000DF4FC882C258D040CD57DF4FD882C3588E
:10799000D040CC57DF4FE882C458D040CB57DF4FA0
:1079A000F882C558D040C158DF4FC882CF57D04069
:1079B000C058DF4FD882C058D040CF57DF4FE88241
:1079C000C158D0400F2D1F5FE196EEADFFADE1979E
:1079D0003496E196FFAFEEAFE197153009F0E4CEB3
:1079E000FFEF2F1A3F0AAF962EAD3FADAF972C5F3A
:1079F0003F4FAF963FAF2EAFAF9735E02316310420
:107A000009F0B2CEA496AFADA4978A2F90E0A896C5
:107A1000BFADA897EB2FF0E0DC01A058B84F41E0D4
:107A200050E0A8960FACA89702C0440F551F0A94C7
:107A3000E2F72C91242B2C93A8962FADA8976A9649
:107A40002FAF6A97A4963FADA4976B963FAF6B9705
:107A5000CE57DF4F4881C258D040CD57DF4F5881B5
:107A6000C358D040CC57DF4F6881C458D040CB5763
:107A7000DF4F7881C558D0406F964CAF5DAF6EAF89
:107A80007FAF6F972F3F09F4E2C13F3F09F4DFC199
:107A9000EE0FFF1FEE0FFF1FEC50F54E108101811E
:107AA00032802380412F502F632D722D65964CAF6D
:107AB0005DAF6EAF7FAF6597880F991F880F991FD5
:107AC000FC01E052F54EC080D180E280F3806996DF
:107AD000CCAEDDAEEEAEFFAE6997C657DF4F688124
:107AE0007981CA58D040CE018F5A9F4F0E94858F0E
:107AF000882309F4B0C120E030E040EA50E4612F6F
:107B0000702F832D922D0F94604D4B015C01CB01A2
:107B1000D50121968CAF9DAFAEAFBFAF2197259613
:107B2000CCAEDDAEEEAEFFAE2597A8968FADA89792
:107B30008111E2C1A4969FADA4979111B2C120E03A
:107B400030E040EA50E4C701B6010F94604D6B018C
:107B50007C01A496AFADA497AA2309F4C4C1A4964E
:107B6000EFADA497E4300CF0BEC122ED422E23E528
:107B7000522E2BE7622E21E4722E21968CAC9DAC06
:107B8000AEACBFAC219725968CAD9DADAEADBFAD73
:107B90002597A7968CAF9DAFAEAFBFAFA7979C01BF
:107BA000AD0169966CAD7DAD8EAD9FAD69970F94BB
:107BB0005F4DAB966CAF7DAF8EAF9FAFAB97A5011E
:107BC000940165966CAD7DAD8EAD9FAD65970F94BC
:107BD0005F4D2D966CAF7DAF8EAF9FAF2D97AB965F
:107BE0008CAD9DADAEADBFADAB9761968CAF9DAF8B
:107BF000AEAFBFAF6197A50194016091790270911A
:107C00007A0280917B0290917C020F945F4D4B0130
:107C10005C01A7962CAD3DAD4EAD5FADA7976091D1
:107C20007D0270917E0280917F02909180020F947C
:107C30005F4DA7966CAF7DAF8EAF9FAFA797812F9B
:107C4000902FA32DB22D8DA79EA7AFA7B8ABC9AA21
:107C5000DAAAEBAAFCAAC984DA84EB84FC84CDAA54
:107C6000DEAAEFAAF8AE2DEC3CEC4CEC5CE3C301D1
:107C7000B2010F94D44629813A814B815C810F94E3
:107C8000D44620918502309186024091870250911E
:107C900088020F94604D69AF7AAF8BAF9CAFA5019E
:107CA0009401C501B4010F94D4464B015C01A79621
:107CB0002CAD3DAD4EAD5FADA797CA01B9010F9494
:107CC000D4469B01AC01C501B4010F94604D20E086
:107CD00030E040E050E40F94C04F1816ACF420E0C0
:107CE00030E040E05FE3C701B6010F94604D299694
:107CF0006CAF7DAF8EAF9FAF2997BE01635C7F4FA6
:107D0000CE0101960E941C1D89859A85AB85BC8594
:107D100029968CAF9DAFAEAFBFAF2997A3961CAE8F
:107D20001DAE1EAE1FAEA397BE01615A7F4FCE019E
:107D3000CD960E94B81D8CA58823C1F02AE939E9A7
:107D400049E95FE36D817E818F8198850F94D446E8
:107D5000A3966CAF7DAF8EAF9FAFA397BE01615A64
:107D60007F4F89E991E10E94B81D1CA6E090D911CE
:107D7000F090DA110091DB111091DC11A090D51177
:107D8000B090D611C090D711D090D8119501A6010E
:107D9000B701C8010F94C04F181614F4750186017D
:107DA0008090750290907602A0907702B090780251
:107DB0002DEC3CEC4CEC5DE3B701C8010F94D446CC
:107DC00060937502709376028093770290937802A5
:107DD00040E0BE01675B7F4FCE018D960F94431448
:107DE00080E1E9E7F2E0A9E9B1E101900D928A951D
:107DF000E1F78092750290927602A0927702B0929B
:107E0000780220E04FEFBE01675A7F4FCE01019606
:107E10000E94331F20E041E0BE01675A7F4FCE0130
:107E200001960E94331F2FEF40E0BE01675A7F4F3B
:107E3000CE0101960E94331F21E040E0BE01675A47
:107E40007F4FCE0101960E94331F0E9435718091B1
:107E5000BF128093C012AD96AEADBFADAD97119776
:107E6000AD96BFAFAEAFAD97AB2B09F45ACB6A96C8
:107E70008FAD6A9787FD55CB6B968FAD6B9787FF5C
:107E800030CC4FCB8BA19CA1ADA1BEA1EF968CAF06
:107E90009DAFAEAFBFAFEF978FA198A5A9A5BAA52B
:107EA0003ACC812F902FA32DB22D21968CAF9DAF70
:107EB000AEAFBFAF219720E030E040EA50E4C70109
:107EC000B6010F945F4D25966CAF7DAF8EAF9FAF1F
:107ED0002597A496BFADA497B4300CF430CE182DDE
:107EE000092D3A2C2B2C92ED492E93E5592E9BEF20
:107EF000692E90E4792E41CEA896FFADA897F43074
:107F00000CF452C0A4962FADA49724300CF120E0BD
:107F100030E040EA50E4612F702F832D922D0F94B2
:107F20005F4D21966CAF7DAF8EAF9FAF219720E064
:107F300030E040EA50E4C701B6010F945F4D6B0199
:107F40007C01A4968FADA49784300CF40ECECBCFD9
:107F5000812F902FA32DB22D21968CAF9DAFAEAF68
:107F6000BFAF219720E030E040EA50E4C701B601FE
:107F70000F94604D25966CAF7DAF8EAF9FAF259768
:107F8000A4963FADA4973111D2CF20E030E040EA73
:107F900050E4612F702F832D922D0F945F4D162F7B
:107FA000072F382E292E9FCFA4969FADA49791110D
:107FB0000DC020E030E040E251E4B401C5010F946F
:107FC0005F4D162F072F382E292ECFCDA496AFAD9B
:107FD000A497A4309CF020E030E040E251E4B401EA
:107FE000C5010F945F4D21966CAF7DAF8EAF9FAFF3
:107FF0002197182D092D3A2C2B2CB7CD182D092D92
:108000003A2C2B2C82ED482E83E5582E8BEF682ED0
:1080100081E4782EB2CD5F926F927F928F929F9281
:10802000AF92BF92CF92DF92EF92FF920F931F9386
:10803000CF93DF931F92CDB7DEB77C0139018B015F
:108040005B01A40EB51ED12CC12CA016B10609F4FB
:1080500050C0F70180809180F80151908F015982C2
:10806000C4010F948C4C5816B9F1652DC4010F94BE
:10807000944CFFEFCF1ADF0AC6018F779927892B1F
:1080800021F162E070E080E090E00F949312C4016F
:108090000F948C4C99818917F9F00E943E2B8BEF3D
:1080A00094E00E941B2981E00F90DF91CF911F91F6
:1080B0000F91FF90EF90DF90CF90BF90AF909F9087
:1080C0008F907F906F905F90089562E070E080E005
:1080D00090E00E94C424DBCFBE016F5F7F4FC301DD
:1080E0000F94DA01F7018081918101969183808359
:1080F000ACCF80E0D9CF0E941B298AE00C94CA281B
:108100002F923F924F925F926F927F928F929F92A7
:10811000AF92BF92CF92DF92EF92FF920F931F9395
:10812000CF93DF93CDB7DEB7C659D1090FB6F89418
:10813000DEBF0FBECDBF0E9458228823F1F180918F
:10814000BA079091BB07A091BC07B091BD07AC01E5
:10815000BD01E2E17695679557954795EA95D1F788
:1081600040FF45C08CE490E10E947B408EEF8093FD
:108170000A081092090881E09AE590936E1A80939C
:108180006D1A8CE490E09093701A80936F1A87E0D8
:108190008093611A82E88093641A84E890E0A0E0FA
:1081A000B0E08093651A9093661AA093671AB09313
:1081B000681A81E19AE10E946B9BCA56DF4F0FB6A5
:1081C000F894DEBF0FBECDBFDF91CF911F910F910D
:1081D000FF90EF90DF90CF90BF90AF909F908F90E7
:1081E0007F906F905F904F903F902F90089562E046
:1081F000B695A795979587956A95D1F780FF07C0A3
:108200000E943A220E948DF90E94BBA3D6CF2090F3
:108210007F1430908014409081145090821480918B
:10822000881481FF05C09091A91398609093A913B9
:1082300082FB882780F98093A81381E490E10E9453
:10824000EDBE80910F14909110149E012F5F3F4F4F
:108250003901009799F09F938F9389E390E19F9361
:108260008F933F932F930F940546C3010E94BFBE87
:108270000F900F900F900F900F900F9000910B1494
:1082800010910C14043B110514F404EB10E01F9240
:108290001F9284E390E19F938F937F926F920F944C
:1082A0000546C3010E94BFBE1F930F938CE290E16D
:1082B0009F938F937F926F920F940546C3010E9404
:1082C000BFBE00910D1410910E140FB6F894DEBFCE
:1082D0000FBECDBF043B110514F404EB10E01F9258
:1082E00081E08F9384E390E19F938F937F926F92CD
:1082F0000F940546C3010E94BFBE1F930F938CE2EB
:1083000090E19F938F937F926F920F940546C301E4
:108310000E94BFBE9091DC13CF56DF4F9883C159A6
:10832000D040E091DD13CE56DF4FE883C259D040F4
:10833000F091DE13CD56DF4FF883C359D040209122
:10834000DF13CC56DF4F2883C459D0402091E61369
:108350003091E7134091E8135091E913692F7E2F74
:108360008F2FCC56DF4F9881C459D0400F94604D69
:108370004B015C0184E290E10E94EDBE8091881483
:108380000FB6F894DEBF0FBECDBF6401750180FD4E
:1083900014C0CF56DF4FC880C159D040CE56DF4FF2
:1083A000D880C259D040CD56DF4FE880C359D04065
:1083B000CC56DF4FF880C459D0408E010F571F4F65
:1083C00023E041E0B601C7010F943B419F938F9397
:1083D0008BE190E19F938F937F926F920F9405466C
:1083E000C3010E94BFBE0F900F900F900F900F908F
:1083F0000F909601A701B401C5010F94C04F181644
:10840000DCF423E041E0B401C5010F943B419F93AC
:108410008F9381E190E19F938F937F926F920F945E
:108420000546C3010E94BFBE0F900F900F900F90A2
:108430000F900F906401750189E090E10E94EDBEFC
:1084400087E08093F00A8093F10860911214709194
:10845000131480911414909115148E010F571F4F0F
:1084600021E041E00F943B419F938F9380918814CA
:1084700083FB882780F9CB56DF4F8883C559D040CE
:10848000CA56DF4F1882C659D040CB56DF4F88817D
:108490009981C559D040C0969F938F938EEF9FE0EE
:1084A0009F938F937F926F920F940546C3010E9412
:1084B000BFBE21E041E0B601C7010F943B419F934D
:1084C0008F9385EF9FE09F938F937F926F920F948E
:1084D0000546C3010E94BFBE43E0A42E44E1B42E72
:1084E0000FB6F894DEBF0FBECDBFF12CE12C5AEED3
:1084F000C52E5FE0D52EF501619171918191919129
:108500005F018E010F571F4F23E041E00F943B4165
:108510009F938F93FF92EF92DF92CF927F926F9211
:108520000F940546C3010E94BFBE0FB6F894DEBF8C
:108530000FBECDBFEA94EF2809F054C18091881492
:1085400084FD15C0809102141F928F9380EE9FE0EE
:108550009F938F937F926F920F940546C3010E9461
:10856000BFBE0F900F900F900F900F900F908BE069
:10857000C82E84E1D82E10E000E09BEDA92E9FE0EC
:10858000B92E23ED822E2FE0922EF601E190F1908C
:108590006F01E114F104D9F01F930F93BF92AF92D2
:1085A0007F926F920F940546C3010E94BFBEFF9257
:1085B000EF929F928F927F926F920F940546C30124
:1085C0000E94BFBE0FB6F894DEBF0FBECDBF013014
:1085D000110509F00BC1809102141F928F938DEC4D
:1085E0009FE09F938F937F926F920F940546C301F4
:1085F0000E94BFBE809111140F900F900F900F90AA
:108600000F900F908823A1F01F928F931F921F92BB
:1086100082EC9FE09F938F937F926F920F94054619
:10862000C3010E94BFBE0FB6F894DEBF0FBECDBF20
:108630008EEB9FE00E94EDBE6091D8137091D9132C
:108640008091DA139091DB138E010F581F4F23E0B6
:1086500041E00F943B41F82EE92E6091D4137091C4
:10866000D5138091D6139091D713005F1F4F23E04D
:1086700041E00F943B41EF92FF929F938F9380EBE9
:108680009FE09F938F937F926F920F940546C30153
:108690000E94BFBE23E041E0CF56DF4F6881C15941
:1086A000D040CE56DF4F7881C259D040CD56DF4FF3
:1086B0008881C359D040CC56DF4F9881C459D040EF
:1086C0000F943B419F938F9386EA9FE09F938F93F4
:1086D0007F926F920F940546C3010E94BFBE8091A6
:1086E000E5138F938091E4138F9380EA9FE09F932B
:1086F0008F937F926F920F940546C3010E94BFBE75
:108700006091E0137091E1138091E2139091E31373
:1087100023E041E00F943B419F938F9387E99FE0D3
:108720009F938F937F926F920F940546C3010E948F
:10873000BFBE8CE0EAEEF3E1A7ECB3E101900D924D
:108740008A95E1F78CE0E6EFF3E1ABEBB3E1019062
:108750000D928A95E1F780E00E94B18681E00E9447
:10876000B18682E00E94B186809187148093AA131B
:1087700081E080937A110E94422286E194E19F93E6
:108780008F9387EE9AE29F938F937F926F920F94CD
:1087900005460FB6F894DEBF0FBECDBFC3010E94E1
:1087A000BFBE809186148F93809185148F938091A2
:1087B00084148F93809183148F935F924F923F9292
:1087C0002F928BE89FE09F938F937F926F920F94ED
:1087D0000546C3010E94BFBE0FB6F894DEBF0FBEB0
:1087E000CDBFEBCCEE24E394F12C85CE01E010E07C
:1087F000CCCE0F931F93CF93DF93082F41E066E712
:108800007FE00E946F2BC7E8D8E010E0802F0E9425
:10881000422B8DE69FE00E941B29812F0E94AB1DF9
:108820004C815D816E817F818AE69FE00E942A2EC5
:10883000488159816A817B8187E69FE00E942A2EC8
:1088400084E69FE00E941B2989E19CE10E947B4015
:108850002896113029F4DF91CF911F910F9108953F
:1088600011E0D4CFCF93DF93EC0160E08CEF97E081
:108870000E940C2ACE01DF91CF910C947B40CF93C4
:10888000DF93CDB7DEB7A8970FB6F894DEBF0FBE63
:10889000CDBF8C017B01942E0E94BFDA011511051A
:1088A00009F4C8C00E943E2BC8010E947B40E1141D
:1088B000F10421F496E8E92E97E2F92E80910B0855
:1088C00080FD89C0816080930B08CDB6DEB680E85C
:1088D00097E00E947B4081E09AE590936E1A809326
:1088E0006D1A88E590E09093701A80936F1A87E074
:1088F0008093611A82E88093641A84E890E0A0E093
:10890000B0E08093651A9093661AA093671AB093AB
:10891000681A81E19AE10E946B9BC8010F94BB45E4
:108920005C01C7010F94BB458A0D9B1D03962DB7B3
:108930003EB7281B390B0FB6F8943EBF0FBE2DBFB4
:108940008DB79EB701965C01FF92EF921F930F9334
:1089500089E797E09F938F93BF92AF920F9405465C
:108960008AE289838A838B838C83D501CE01059625
:10897000EDB7FEB738960FB6F894FEBF0FBEEDBF49
:10898000BE016F5F7F4FFC01E61BF70B2D9121119C
:108990000BC0E60FF71F8AE29F01261B370B283218
:1089A000310534F48193F8CFFC012193CF01EBCF53
:1089B00020E630E140E050E081E19AE10F94F701D8
:1089C0006AE070E080E090E00E94089B0FB6F894A7
:1089D000DEBE0FBECDBE0E943A2B8DE997E00E940D
:1089E0001B2961E08BE897E00E940C2A89EE93E056
:1089F000019739F000C00000EEE5F9E03197F0F79B
:108A0000F7CFF89489EE93E0019739F000C00000A9
:108A1000E6EEF3E03197F0F7F7CF0E94BFDA992046
:108A200031F00E94FFF10E94F529A895FECF0E9427
:108A3000B7F1F9CFE114F10421F486E8E82E87E2DA
:108A4000F82E04E917E03ACF8091BF129091C0123E
:108A50002FEF3FEF981751F0E92FF0E0E154FD4E72
:108A6000228130E09F5F9F779093C012C9010895E3
:108A70002F923F924F925F926F927F928F929F922E
:108A8000AF92BF92CF92DF92EF92FF920F931F931C
:108A9000CF93DF93CDB7DEB764970FB6F894DEBF00
:108AA0000FBECDBFB82E80919816843008F0C0C19B
:108AB00021E6D22E80919816843008F0F8C080917B
:108AC000BF129091C012891B8F7709F4F0C00E94E9
:108AD000244597FF0BC00E943A2B81E496E00E9448
:108AE0001B298091BF128093C012E4CF8A3019F005
:108AF0008D3009F0D3C01092A71380914513909147
:108B00004613FC01EF5BFC4E1682892B19F40E9480
:108B100023DCD0CF109246131092451307E413E1E3
:108B2000F8018191803209F446C08E3409F0A1C069
:108B30006CE376E0C8010F94EB457C01892B41F092
:108B40006EE470E0C80104960F94AE50009709F4EB
:108B5000C8014AE050E070E060E001960F945B438A
:108B60002B013C018091411390914213A09143133A
:108B7000B09144130196A11DB11D481659066A060D
:108B80007B0629F060E089E096E0EF2851F16AE287
:108B900070E0C8010F94DD509C01009729F1982FD7
:108BA000901BF12C992349F09150F801E90FF11D28
:108BB0008081F826F7CF8F01B3CF4AE050E070E014
:108BC00060E0C90101960F945B432F2D30E050E027
:108BD00040E0621773078407950751F060E08AEE62
:108BE00095E00F94470C66CF60E080EC95E0F9CFFC
:108BF0004092411350924213609243137092441377
:108C00008091E6098130E1F467E470E0C8010F94D7
:108C1000AE500097A9F04AE050E070E060E00196A5
:108C20000F945B43643071058105910548F48FE131
:108C300095E00E941B2960E085E195E00E942B9D54
:108C4000809147138B3309F435CF80919816843087
:108C500008F030CF80919A168D9DC001112467E4F1
:108C600073E18556994E0F94B95080E00F941E0C15
:108C700021CF8091131B80FFC3CF64E47EE2C80143
:108C80000F94EB45009731F0FC01838180538A30CB
:108C900008F0B6CF60E086E995E0A3CF25E433E1A4
:108CA00047E453E167EA73E10E94A6AF03CF8091E6
:108CB000131B83FDBDC082FFBBC087FDB9C01A82F4
:108CC000198201E6F02E84E0E82E99E6D92E8091F3
:108CD0009816843008F0ACC00E94DEAF8111A8C0A5
:108CE00041E050E0BE016D5E7F4F87E79CE10E944E
:108CF00022CE0B8910E0019711F00FEF1FEF80914A
:108D00007F1C9091801CA091811CB091821C80934B
:108D10000F1B9093101BA093111BB093121B0E946A
:108D2000DEAF0F3F100749F4811107C00E943A2BB4
:108D300089E596E00E941B29CACF40919A16242FFC
:108D400030E00A3061F00D3051F0882309F462C040
:108D500089819A81009719F001969A8389831092EC
:108D6000550789819A81F29EF001F39EF00D11243E
:108D7000E856F94EE80FF91F1382892B59F50E9426
:108D800023DC0E94DEAF882309F4A1CF87E79CE1B2
:108D90000E94CFCF80910A1B882391F1815080934C
:108DA0000A1B8D9DC001112462E08F5D964F0E94C9
:108DB000F5FAE0910A1B24E0E29FF0011124E35E42
:108DC000F64F60817181828193810E942AAC0E945A
:108DD000E0C77DCF1A82198281E00F941E0C80912A
:108DE0000F1B9091101BA091111BB091121B80932F
:108DF0001C1290931D12A0931E12B0931F12C1CF8C
:108E00000E94D8CF8091131B88608093131BE0923F
:108E1000E6095DCF4F9DA00111244556594E9E0194
:108E20002F5F3F4F65E577E0802F0E94A6AF4FCFC1
:108E30000F94C6126B017C01B11004C080917B11AC
:108E4000882351F0C092ED08D092EE08E092EF082E
:108E5000F092F008BB24B39480919C0790919D07F9
:108E6000A0919E07B0919F070097A105B105B1F0B1
:108E70004091ED085091EE086091EF087091F00874
:108E8000840F951FA61FB71FA7019601281B390B3A
:108E90004A0B5B0BDA01C901B7FFC3C190910B19F3
:108EA00080910C199813D2C14091090250910A0285
:108EB00060910B0270910C02452B462B472B29F039
:108EC000981709F4CCC110926B070E940B26182F3B
:108ED000811103C00E943826182F0F94C6124B012F
:108EE0005C0180915A071817D1F081E090E0A0E072
:108EF000B0E081149104A104B10419F080E090E085
:108F0000DC01880D991DAA1DBB1D80937C079093E1
:108F10007D07A0937E07B0937F0710935A07111126
:108F20002FC08091560790915707A0915807B09194
:108F30005907A5019401281B390B4A0B5B0BDA0179
:108F4000C901B7FD1DC0D501C4018C53964FAF4F69
:108F5000BF4F8093560790935707A0935807B0933D
:108F600059078091D008811109C00E940B268111F8
:108F700005C00E943826882309F4A2C10E94E82473
:108F80000F94C6124B015C0110918C11012F11112D
:108F900008C080910B1990910C1901E0981301C041
:108FA00000E020E030E04CE053E460917D187091E7
:108FB0007E1880917F18909180180F94C04F87FD84
:108FC00003C0002309F4E7C1111108C090910B19E7
:108FD00080910C1911E0981301C010E020E030E0FE
:108FE0004CE053E460919418709195188091961814
:108FF000909197180F94C04F87FD03C0112309F477
:10900000CAC180E091E040915F0750916007609194
:10901000610770916207452B462B472B09F490E0BE
:10902000981789F0882309F4B8C1D501C401805884
:10903000904BAD4EBF4F80935F0790936007A09316
:109040006107B0936207409085025090860260905D
:1090500087027090880220915B0730915C074091F5
:109060005D0750915E07C301B2010F946E468823DD
:1090700019F180915F0790916007A0916107B0910D
:10908000620740925B0750925C0760925D077092A6
:109090005E07892B8A2B8B2B09F456C0D501C4019E
:1090A0008058904BAD4EBF4F80935F079093600701
:1090B000A0936107B093620780915F07909160076A
:1090C000A0916107B09162070097A105B105E1F198
:1090D000881A990AAA0ABB0AB7FC36C010925F0721
:1090E0001092600710926107109262078AEB96E077
:1090F0000E941B2960E086EA96E00E942B9D8091E9
:10910000811890918218181619062CF460E090E0EE
:1091100080E00E94902580919818909199181816D7
:1091200019062CF461E090E080E00E949025809187
:109130006A1890916B181816190634F410926B186F
:1091400010926A180E9496228091F2089091F3087A
:10915000A091F408B091F5080097A105B10531F18F
:1091600046015701881A990AAA0ABB0AD501C40107
:10917000B7FD1CC08091E6098330C0F08FEF9FEFF0
:10918000DC018093F2089093F308A093F408B09365
:10919000F50880E1E9E7F2E0A9E9B1E101900D927B
:1091A0008A95E1F70E94CD8A0E9435718091670708
:1091B00090916807A0916907B0916A07A70196018D
:1091C000281B390B4A0B5B0BDA01C901B7FD63C2DF
:1091D00030910B1990910C1920910002809153024B
:1091E000391709F4DEC0E0910C1935E6E39FF00170
:1091F0001124E858F44F9081899FC0011124880FF1
:10920000892F881F990B9195281709F409C180931C
:1092100000020F94C612009100020111C5C060E067
:10922000BDC10E943A2B83E996E00E941B29609100
:1092300096167091971688E696E00E948EF840E0A8
:1092400070E060E090E080E00E943F44C092ED0852
:10925000D092EE08E092EF08F092F00825CEB1101F
:1092600032CE0F94C6120091ED081091EE082091B5
:10927000EF083091F0088090090290900A02A090C7
:109280000B02B0900C02080D191D2A1D3B1D601B1E
:10929000710B820B930B97FD16CE80916B0781119A
:1092A00014CE81E080936B0780E00E94CCF181E0D6
:1092B0000E94CCF182E00E94CCF10E94B7F105CE71
:1092C0008091B01381115ACE8091D108811156CE70
:1092D0008091D208811152CE80918118909182188C
:1092E000181619060CF44ACE80918318811146CEC7
:1092F0008091981890919918181619060CF43ECE82
:1093000080919A1881113ACE80916A1890916B18C9
:10931000181619060CF432CE80916C1881112ECEDD
:1093200020E030E048E452E460917D1870917E18AE
:1093300080917F18909180180F94C04F87FF1ECEA8
:1093400020E030E048E452E4609194187091951860
:1093500080919618909197180F94C04F87FF0ECE6A
:1093600080917C0790917D07A0917E07B0917F0747
:109370000097A105B10561F0881A990AAA0ABB0AEB
:1093800030E3831A35E7930AA108B108B7FCF8CD9A
:109390000E94F529F5CD81E035CE80E090E0DC013A
:1093A0004ACE9091B01328CF10E061E00F3F110535
:1093B00009F4F4C069E0CE0101960E94462689892D
:1093C000882309F4E6C0E981FA819F858889911193
:1093D000A3C0608190E023E030E0A901481B590B55
:1093E000440F551F042E01C0220F0A94EAF720955E
:1093F000262362E070E001C0660F4A95EAF7262B4B
:109400002083FC013396EE0FFF1F41E050E04C0F2C
:109410005D1FE40FF51F0190F081E02D11830083A3
:1094200080911009882309F429C18090130290903B
:109430001402E091BA1327E1E29FF0011124E758EA
:10944000F74EC401029720853185281739070CF49F
:1094500015C110910C19612C712C00E01C8A8091AF
:109460000B19811709F49EC0812F90E035E6389FD3
:10947000F001399FF00D1124E85DF44F45895689BC
:109480006789708D452B462B472B81F4418D528D7A
:10949000638D748D452B462B472B41F4458D568D9E
:1094A000678D70A1452B462B472B99F145E6489FC8
:1094B0009001499F300D1124C901885D944F5C01D2
:1094C000FC0161A172A183A194A10F9473461B01B9
:1094D0002C01F50165A176A187A190A50F94734693
:1094E0009B01AC01C201B1010F945A4EF5012181DB
:1094F0003281438154810F94D4462B015C01930146
:10950000402F5C890F94C04F18161CF432010A2DAD
:10951000BC8A1F5F1F70A3CF2A89211181CFAFEFB3
:10952000B0E0923029F0AD85BE850D90BC91A02DA4
:10953000608190E023E030E0A901481B590B440F03
:10954000551F042E01C0220F0A94EAF72095262306
:1095500062E070E001C0660F4A95EAF7262B20838F
:109560000396880F991FE1E0F0E0EC0FFD1F8E0FCE
:109570009F1FFC01A080B18098010F94064D2FEF32
:1095800030E040E050E00F94B24CF501318320838D
:1095900047CF61E00F37110508F441CE89E00F9401
:1095A00065123ECF20913602309137024091380249
:1095B00050913902B301802F9C890F94D4462B011E
:1095C0003C01B401092C000C880B990B0F947546D3
:1095D0009B01AC01C301B2010F94604D69837A8392
:1095E0008B839C834091110250911202B401CE01F1
:1095F00001960E949C7049805A806B807C8080908C
:10960000630790906407A0906507B0906607A50176
:109610009401C301B2010F946E4687FF1CC020E085
:1096200037ED43EA5CE3C301B2010F94D4462B014A
:109630003C0128E431EE4AE75FE3C501B4010F9431
:10964000D4469B01AC01C301B2010F94604D698304
:109650007A838B839C8369817A818B819C816093DF
:1096600063077093640780936507909366070F9470
:10967000CC4ECB016091BA130E949025F4E6CF0E38
:10968000D11CE11CF11CC0926707D0926807E092E0
:109690006907F0926A070E9423DC8091E60988231B
:1096A00009F46AC28091BA1390E0FC01EF50F54FC3
:1096B0002081222309F4D2C08F54974FFC0180816E
:1096C000882309F4CBC0809178118111C7C08091A3
:1096D0007B11811105C00E940B26882309F4BEC0AE
:1096E000F894E091BA13F0E0EF54F74F908197307F
:1096F00009F090C080910301817090916C079827C8
:1097000080936C078091B008892B8093B00860919A
:10971000A8087091A9088091AA089091AB08789444
:1097200020E030E0A9010F946E4687FF97C081E0EA
:109730008093781180917B1181118EC080911C09DA
:1097400081118AC080911B09811181C085ED96E04D
:109750000E947B4084E08093220B81E09AE5909305
:109760006E1A80936D1A8EE490E09093701A809335
:109770006F1A87E08093611A82E88093641A84E804
:1097800090E0A0E0B0E08093651A9093661AA093F1
:10979000671AB093681A81E19AE10E946B9B0E945C
:1097A0003D2A01E00093BD1240E363E177E087E7E3
:1097B00093E30E94422A61E08BE693E30E94242A0D
:1097C00010918907102760E08BE598E071F460E064
:1097D00081E097E00E940C2A80E30E94CA288AE078
:1097E0000E94CA2860E08FEC96E00E940C2A8FEE5F
:1097F00096E00E941B2980E30E94CA288AE00E940A
:10980000CA28112349F18AEE96E09093030B8093C6
:10981000020B22C0992309F47ACF8091030121E041
:10982000923009F420E08170281371CF8091AC0848
:109830009091AD08A091AE08B091AF088093A808B0
:109840009093A908A093AA08B093AB0860CF0E9498
:10985000EFE7882309F47ACF0E9435718091131BBA
:1098600082FF53C087FD51C080917A11882309F48B
:109870004AC0359B48C080916D078F5F80936D070C
:10988000833008F442C08090810290908202A090C0
:109890008302B090840220E030E040E050E4C50153
:1098A000B4010F94604D6B017C0120E030E448E18D
:1098B00054E40F946E4687FD07C0C12C80E4D82E77
:1098C00088E1E82E84E4F82EA5019401C701B601D1
:1098D0000F945F4D6B017C0120E030E0A9010F94F3
:1098E0006E4687FF03C0C12CD12C760140E0C70132
:1098F000B6010F94B1080E94BFDA40E070E060E06A
:1099000084E297E0A1CC10926D0790910901892F14
:1099100080958170109101028117C9F02091131B6D
:1099200020642093131B8093010290FD3EC164EFDD
:1099300071E080E090E00E94C4240E9405D08091F4
:10994000131B84FD55C1111132C10E9473A40F94E1
:10995000C6126B017C01109108021123F1F0809175
:109960008D118823D1F040916E0750916F0760915F
:1099700070077091710746015701841A950AA60A6B
:10998000B70AB501A40177FD1AC0833009F42BC1D1
:109990000CF01AC181300CF01FC1212F30E0A8EE6D
:1099A000B3E00F94064DC60ED71EE81EF91EC092F6
:1099B0006E07D0926F07E0927007F0927107809166
:1099C000BE12813009F073C00F94C6126B017C0186
:1099D0008091760790917707A0917807B0917907E9
:1099E000A7019601281B390B4A0B5B0BDA01C90151
:1099F000B7FD3AC0D701C601805F984DAF4FBF4F4A
:109A00008093760790937707A0937807B0937907B0
:109A10008090380890903908A0903A08B0903B08A0
:109A20000E94D791AB01BC0140933808509339088C
:109A300060933A0870933B08809191099091920944
:109A4000A0919309B091940988199909AA09BB09B1
:109A5000840F951FA61FB71F8093910990939209B9
:109A6000A0939309B0939409809172079091730722
:109A7000A0917407B091750746015701881A990A99
:109A8000AA0ABB0AD501C401B7FD11C020E8C20E65
:109A90002EEED21E26E3E21EF11CC0927207D09277
:109AA0007307E0927407F09275070E94966F0E9408
:109AB000A4B180919907882381F10F94C6126B019C
:109AC0007C018091950790919607A0919707B0919E
:109AD000980746015701881A990AAA0ABB0AD501B4
:109AE000C401B7FD1AC02091990730E0A8EEB3E099
:109AF0000F94064DC60ED71EE81EF91EC09295079C
:109B0000D0929607E0929707F09298078091BA1347
:109B10000E9453D68AE00E94CA2880919407882325
:109B200059F10F94C6126B017C01809190079091BE
:109B30009107A0919207B0919307A7019601281B66
:109B4000390B4A0B5B0BDA01C901B7FD15C0209137
:109B5000940730E0A8EEB3E00F94064DC60ED71E72
:109B6000E81EF91EC0929007D0929107E0929207EA
:109B7000F09293070E94A9C764960FB6F894DEBFCF
:109B80000FBECDBFDF91CF911F910F91FF90EF904E
:109B9000DF90CF90BF90AF909F908F907F906F900D
:109BA0005F904F903F902F9008950E94E8CF123021
:109BB00008F0CDCE0E9473A4CACE81E397E09093C3
:109BC000030B8093020BC3CE843009F0E6CE0E94D3
:109BD0003E2B88E397E004C00E943E2B87E697E087
:109BE0000E941B29DACE0E943E2B80E597E0F8CF39
:109BF000123018F40E94F6AEAACE123009F0A7CEA9
:109C00000E940FD4882379F081E00E9401F947EB8C
:109C100050E063ED73E188E19BE10E9422CE88E190
:109C20009BE10E94CFCF0E9458228111C6CF0E9493
:109C30003A220E948DF981E08093091B0E94BBD3D8
:109C400086CE1F93CF93DF93D82F162F8091A91321
:109C500083FD15C0C091BA1387E1C89FF00111249C
:109C6000E758F74E808591850E947022882339F04D
:109C70006C2F80910F02909110020E949025612F0D
:109C80008BE00F94AF09DD2349F040E061E0809163
:109C9000BA13DF91CF911F910C94BED88091A81375
:109CA00091E089278093500217E180915002882328
:109CB000F9F0C091BA131C9FE0011124C758D74E88
:109CC00020E030E040E05FE36C817D818E819F8108
:109CD0000F94604D0F94CC4E28853985621B730B11
:109CE00077FF03C07195619571096430710544F483
:109CF000109250028091A91383FF06C081E019C021
:109D000080E00E943845D1CFE091BA1387E1E89F07
:109D1000F0011124E758F74E808591850E9470224A
:109D2000882361F30E943E2B86E198E00E941B2964
:109D300080E0DF91CF911F9108956F927F928F9273
:109D40009F92AF92BF92CF92DF92EF92FF920F93CA
:109D50001F93CF93DF93CDB7DEB764970FB6F89418
:109D6000DEBF0FBECDBF0E94472B082F87FDC7C0A7
:109D70008AE50E94EF20882309F4D6C040E050E035
:109D8000BA018AE50E94FC206B017C0163E085E05A
:109D90000F94AF091091BA13A02E002E000CBB082F
:109DA0001A151B0421F060E0802F0E948AE52091A3
:109DB000810230918202409183025091840260E0DE
:109DC00070E888E194E40F945F4D3B014C019601EB
:109DD000A7010F94C04F181614F063017401C60157
:109DE000D7018D839E83AF83B88720E030E0A9013F
:109DF000B601C7010F946E46882321F0CE01059667
:109E00000E94AE1B80E090E0A8E4B2E489879A87C4
:109E1000AB87BC871D861E861F86188A8CE40E942D
:109E2000EF20882309F487C00E9473206B017C0116
:109E300020E030E0A901C701B6010F94C04F87FFB1
:109E400004C0F7FAF094F7F8F094C98ADA8AEB8A3A
:109E5000FC8A87E18A9DF0018B9DF00D1124E75863
:109E6000F74EE084F18486E0E816F104C4F020E0C7
:109E700030E040E05FE364817581868197810F94D3
:109E8000604D0F94CC4E6E197F0977FF03C071951A
:109E900061957109FF24F394663071050CF4F12C7F
:109EA00063E080E00E94214E811152C063E089E0AE
:109EB0000F94AF096D817E818F8198856B017C0144
:109EC000F7FAF094F7F8F094C982DA82EB82FC8218
:109ED00020E030E0A9010F946E46882321F0CE01E6
:109EE00001960E94AE1B8091BA13811721F060E0A9
:109EF000812F0E948AE560E089E00F94AF096496A3
:109F00000FB6F894DEBF0FBECDBFDF91CF911F918A
:109F10000F91FF90EF90DF90CF90BF90AF909F9008
:109F20008F907F906F900895C12CD12C80EAE82EFD
:109F300090E4F92E2BCFE091BA1388E0E89FF0016E
:109F40001124E957F74FC480D580E680F78070CFA1
:109F5000E02E03E02F2DAE01475F5F4FBE016F5E25
:109F60007F4FCE010D960F94D90EA4CF4F925F92E2
:109F70006F927F92AF92BF92CF92DF92EF92FF9259
:109F80001F93CF93DF9300D000D01F921F92CDB7C5
:109F9000DEB75C01E62EF42E642F80E00E94214E95
:109FA000182F81111BC0EE2021F060E089E00F9492
:109FB000AF09812F28960FB6F894DEBF0FBECDBF34
:109FC000DF91CF911F91FF90EF90DF90CF90BF90E6
:109FD000AF907F906F905F904F900895EE2021F0AA
:109FE0006F2D83E00F94AF0980E090E0A0E7B2E42A
:109FF0008D839E83AF83B88780E090E0A0E5B1ECCD
:10A0000089839A83AB83BC83BE016B5F7F4FCE0194
:10A0100001960E946E8968E873E180E090E00E94FA
:10A02000C424C12CD12C88ECE82E81E4F82ECD82FA
:10A03000DE82EF82F88680E090E0A8EAB1E48983CE
:10A040009A83AB83BC83BE016B5F7F4FCE010196C9
:10A050000E946E894090ED115090EE116090EF11CA
:10A060007090F011C092ED11D092EE11E092EF11CC
:10A07000F092F01180E090E0A0E2B1E48D839E8345
:10A08000AF83B887F50180819181A281B3818983F3
:10A090009A83AB83BC83BE016B5F7F4FCE01019679
:10A0A0000E946E894092ED115092EE116092EF1174
:10A0B0007092F0110E94B6257CCF4F925F926F9202
:10A0C0007F928F929F92AF92BF92CF92DF92EF9248
:10A0D000FF921F93CF93DF9300D000D01F921F9267
:10A0E000CDB7DEB70E94472BD82E87FDF0C08AE59A
:10A0F0000E94EF20812C912C40EAA42E40E4B42E43
:10A10000882341F040E050E0BA018AE50E94FC203B
:10A110004B015C0164E083E00F94AF091091BA1326
:10A12000ED2C0D2C000CFF081E151F0421F060E023
:10A130008D2D0E948AE520E030E0A901C501B4011F
:10A140000F94C04F181684F580E090E0A0EAB0E4C8
:10A150008D839E83AF83B8872091810230918202E4
:10A160004091830250918402C501B4010F94604D67
:10A170002B013C0120E030E848E154E40F946E46A6
:10A1800087FD07C0412C30E8532E38E1632E34E4BC
:10A19000732E49825A826B827C82BE016B5F7F4F35
:10A1A000CE0101960E944F8984E50E94EF20811123
:10A1B00029C027E8C22E28E0D22EF12CE12C809174
:10A1C000BA138E151F0421F060E08E2D0E948AE5DF
:10A1D000F60180819181A281B381B05889839A83ED
:10A1E000AB83BC8344E061E0CE0101960E94B64F90
:10A1F000F8E0CF0ED11CEA94EF2849F1EE24E39465
:10A20000F12CDDCF85E50E94A120882309F475C0DB
:10A210000E9473206B017C0120E030E0A901C7019E
:10A22000B6010F94C04F87FF04C0F7FAF094F7F817
:10A23000F094F7FAF094F7F8F094C982DA82EB829E
:10A24000FC8244E061E0CE0101960E94B64F20E01E
:10A2500030E0A901C501B4010F94C04F18165CF598
:10A2600080E090E0A0EAB0E48D839E83AF83B8875E
:10A27000A501940160918102709182028091830214
:10A28000909184020F945F4D6B017C0120E030E0DF
:10A29000A9010F94C04F18161CF0C12CD12C7601C7
:10A2A000C982DA82EB82FC82BE016B5F7F4FCE01F6
:10A2B00001960E944F898091BA13811721F060E0C6
:10A2C000812F0E948AE560E089E00F94AF0928960B
:10A2D0000FB6F894DEBF0FBECDBFDF91CF911F91B7
:10A2E000FF90EF90DF90CF90BF90AF909F908F90B6
:10A2F0007F906F905F904F900895F70183E0EE0F8D
:10A30000FF1F8A95E1F7E957F74FC080D180E280BF
:10A31000F38082CF2F923F924F925F926F927F9203
:10A320008F929F92AF92BF92CF92DF92EF92FF9265
:10A330000F931F93CF93DF9300D000D000D01F92D4
:10A34000CDB7DEB74C017B01498759010A8761E02F
:10A350008BE598E00E940C2A41EE53E362E678E038
:10A3600085E00F94240A90917B1181E0890F8093FE
:10A370007B118091131B82FB222720F9288782FF03
:10A3800008C087FDC7C08B7F8093131B9E5F90938F
:10A390007B110E94EC9C80E1E9E7F2E0ACE7B1E1DF
:10A3A00001900D928A95E1F787E00E944287782E0E
:10A3B00060E070E080E090E471103FC02090810286
:10A3C00030908202409083025090840220E030E07E
:10A3D00040E050E4C201B1010F94604D6B018C016B
:10A3E00020E030E848E154E40F94C04F18162CF4F4
:10A3F000C12C80E8D82E08E114E4F7016084F185CF
:10A40000FD83F701F285FE83F701F385FF83960153
:10A41000A801662D7D818E819F2F0F94C04F181645
:10A4200024F06C2CDD820E831F83A2019101662D26
:10A430007D818E819F810F945F4D2885222349F075
:10A4400020917A11222329F041E0711040E00F940D
:10A45000B1080E94357120E030E0A901F40160816B
:10A460007181828193810F946E468823A1F080913F
:10A47000BA130E94812281110EC080E090E0A0E713
:10A48000B2E489839A83AB83BC83BE016F5F7F4F45
:10A49000C4010E946E89711004C0B70180E00E945F
:10A4A00024920091BA1310918E116A8580E00E9467
:10A4B0009D8720E030E0A901F501608171818281F2
:10A4C00093810F946E46882329F042E06985C50187
:10A4D0000E94B64F602F812F0E949D870E94B62553
:10A4E00081E02A960FB6F894DEBF0FBECDBFDF9194
:10A4F000CF911F910F91FF90EF90DF90CF90BF9081
:10A50000AF909F908F907F906F905F904F903F9013
:10A510002F90089518863DCF8F929F92AF92BF9251
:10A52000CF92DF92EF92FF920F931F93CF93DF931F
:10A53000CDB7DEB7A0970FB6F894DEBF0FBECDBF84
:10A540000E94472BF82E87FD1BC18091BA0790917E
:10A55000BB07A091BC07B091BD0723E1B695A795B5
:10A56000979587952A95D1F71091BA1380FD1F2DE5
:10A5700061E081E00F94AF090E941B9B811104C030
:10A5800080E69FE00E94EDBEB090BA138F2D0F2C95
:10A59000000C990BB816190641F0809159028230CF
:10A5A00024F460E08F2D0E948AE585E40E94EF206C
:10A5B000882309F4F8C00E9473206B017C0120E01D
:10A5C00030E0A9010F94C04F87FF04C0F7FAF09460
:10A5D000F7F8F094F7FAF094F7F8F094C98EDA8E61
:10A5E000EB8EFC8E8CE0E3EAF2E0DE011196019046
:10A5F0000D928A95E1F788E50E94EF20882351F0BB
:10A6000040E050E0BA0188E50E94FC2069837A832B
:10A610008B839C8389E50E94EF20882351F040E0E2
:10A6200050E0BA0189E50E94FC206D837E838F8310
:10A6300098878AE50E94EF20882351F040E050E09F
:10A64000BA018AE50E94FC2069877A878B879C87FC
:10A65000E091BA1388E0E89FF0011124E957F74F21
:10A66000C080D180E280F38085E50E94EF208823BE
:10A6700021F00E9473206B017C0120E030E0A901F1
:10A68000C701B6010F94C04F87FF04C0F7FAF094DA
:10A69000F7F8F094F7FAF094F7F8F094CD8EDE8E98
:10A6A000EF8EF8A262E070E082E40E94FC21A82E06
:10A6B00080917B1181115CC0012F9E01235E3F4F71
:10A6C00041E0BE016F5F7F4FCE0149960E948A51E3
:10A6D000882309F44DC0612F81E00F94131A70E0B4
:10A6E00060E082E50E94FC214C0180E090E0A8E45B
:10A6F000B2E48D8B9E8BAF8BB88FE091BA1388E05C
:10A70000E89FF0011124E957F74FC480D580E68017
:10A71000F7808CE40E94EF20882321F00E947320B0
:10A720006B017C0120E030E0A901C701B6010F9464
:10A73000C04F87FF04C0F7FAF094F7F8F094C98A85
:10A74000DA8AEB8AFC8A1D861E861F86188A80910B
:10A750007B11882369F0E12E84012A2DAE014B5E26
:10A760005F4FBE016F5E7F4FCE010D960F94E60FD7
:10A770008091BA138B1521F060E08B2D0E948AE541
:10A78000A0960FB6F894DEBF0FBECDBFDF91CF917C
:10A790001F910F91FF90EF90DF90CF90BF90AF90FF
:10A7A0009F908F900895C12CD12CE12C80E4F82E3D
:10A7B00011CFCF92DF92EF92FF920F931F93CF931F
:10A7C000DF93CDB7DEB76C970FB6F894DEBF0FBE40
:10A7D000CDBF8CE40E94EF20882309F4B2C00E9410
:10A7E00073206B017C0120E030E0A9010F94C04F81
:10A7F00087FF04C0F7FAF094F7F8F094F7FAF094B2
:10A80000F7F8F094C98EDA8EEB8EFC8E8CE0E3EADA
:10A81000F2E0DE01119601900D928A95E1F788E54C
:10A820000E94EF208823A1F040E050E0BA0188E5C3
:10A830000E94FC202091B1123091B2124091B312CB
:10A840005091B4120F945F4D69837A838B839C83FC
:10A8500089E50E94EF208823A1F040E050E0BA0192
:10A8600089E50E94FC202091B5123091B6124091EA
:10A87000B7125091B8120F945F4D6D837E838F8312
:10A8800098878AE50E94EF20882351F040E050E04D
:10A89000BA018AE50E94FC2069877A878B879C87AA
:10A8A00061E080E00F94AF091D861E861F86188A1E
:10A8B00080917B11811136C00FEF9E01235F3F4FC6
:10A8C00040E0BE016F5F7F4FCE0149960E948A51E2
:10A8D000882341F16FEF80E00F94131A898D9A8DD0
:10A8E000AB8DBC8DB0588D8B9E8BAF8BB88F198A7A
:10A8F0001A8A1B8A1C8A1D861E861F86188A8091CA
:10A900007B11882379F0EE24EA9410E000E020E047
:10A91000AE014B5E5F4FBE016F5E7F4FCE010D9665
:10A920000F94E60F6C960FB6F894DEBF0FBECDBF46
:10A93000DF91CF911F910F91FF90EF90DF90CF901B
:10A940000895C12CD12CE12C80E4F82E57CFCF9262
:10A95000DF92EF92FF92CF93DF936B017C01D42FB4
:10A96000C0918D1183E080938D1181E080938C11D3
:10A97000C114D104E104F10431F00F94C612C60EE3
:10A98000D71EE81EF91E80918C11882389F0C1140E
:10A99000D104E104F10421F48D2F0E943845F3CF56
:10A9A0000F94C6126C197D098E099F0997FDF4CF8B
:10A9B00010928C11C0938D11DF91CF91FF90EF9089
:10A9C000DF90CF9008951F920F920FB60F9211242F
:10A9D0000BB60F922F938F939F93EF93FF938091DA
:10A9E000500620914F06821306C08091C1008F7DD2
:10A9F0008093C10012C0E82FF0E0E15BF94F928133
:10AA00008F5F8F779093C600809350069091C0001F
:10AA100090649093C000281741F3FF91EF919F91AC
:10AA20008F912F910F900BBE0F900FBE0F901F9024
:10AA300018951F920F920FB60F9211240BB60F921A
:10AA40000F931F932F933F934F935F936F937F9336
:10AA50008F939F93AF93BF93CF93DF93EF93FF9326
:10AA6000C091C6000091C012D091BF1211E01D0F1D
:10AA70001F7790914E06913108F09FC0E92FF0E0CA
:10AA80008827EA5BFA4A8F4F0D94574D57558655E4
:10AA90009555A455AB55DD55AF55DD55B355B75557
:10AAA000DD55BB55BF55C355CA55DD55D555C032CB
:10AAB00029F028F5CA3011F0CD3031F5011731F009
:10AAC000ED2FF0E0E154FD4EC283D12FD093BF12A1
:10AAD000FF91EF91DF91CF91BF91AF919F918F91B6
:10AAE0007F916F915F914F913F912F911F910F91A6
:10AAF0000F900BBE0F900FBE0F901F901895CD3486
:10AB000081F081E0CE3471F080E10CC0CA3338F4BA
:10AB1000C033A0F6C03291F2CD32B1F7CFCFCD34F1
:10AB200099F782E080934E06C9CFC13359F018F4EB
:10AB3000C03221F2E9CF88E0C433A1F38BE0C833FF
:10AB400089F3E2CF83E0EECF84E0C03359F386E0AF
:10AB5000C13341F3D9CF85E0C833B1F6E3CF87E005
:10AB6000C23391F6DFCF89E0C13371F6DBCF8AE0E3
:10AB7000C03351F6D7CF8CE0C73331F6D3CF8DE059
:10AB8000C63311F6CFCFC03209F498CF8EE0C3356B
:10AB900049F2BACF80ED8C0F8A3008F08FCF9FE05A
:10ABA00090934E068093D10689CFCA3019F0CD30EC
:10ABB00009F084CF10924E0681CFCA3019F0CD3003
:10ABC00009F07CCF8091DF1A8823A1F3973089F0B8
:10ABD00038F4953079F71092500210928C11EACF28
:10ABE0009A3059F09F3031F78091D1060E94D325D9
:10ABF000E1CF81E08093E608DDCF81E08093E50836
:10AC0000D9CF8EBD0DB407FEFDCF08958FEF8EBD59
:10AC10000DB407FEFDCF8EB50895909164009B7F23
:10AC200090936400982F906A96959CBD80FD03C018
:10AC300091E0863009F490E09DBD08952F923F92F7
:10AC40004F925F926F927F928F929F92AF92BF923C
:10AC5000CF92DF92EF92FF920F931F93CF93DF93E8
:10AC6000CDB7DEB7CC54D1090FB6F894DEBF0FBE16
:10AC7000CDBF2D968FAF2D9720918D112C962FAF94
:10AC80002C9781E080938D118091C3078D3409F456
:10AC90006CC5843511F40C94506B873409F0AFC146
:10ACA0008091C1079091C2078A31910509F4A9C228
:10ACB00008F097C18430910508F04EC12091E60953
:10ACC0008230910508F4FFC1233008F402C211E07C
:10ACD000029709F010E00E94132119821A821B8248
:10ACE0001C821D821E821F82188682E50E94EF2030
:10ACF000882309F405C20E9473206B017C0120E0C7
:10AD000030E0A9010F946E46882309F408C14090F1
:10AD1000790250907A0260907B0270907C02809160
:10AD20007D0290917E02A0917F02B09180022796D1
:10AD30008CAF9DAFAEAFBFAF279780909911909029
:10AD40009A11A0909B11B0909C1180919D119091AF
:10AD50009E11A0919F11B091A0112B968CAF9DAF29
:10AD6000AEAFBFAF2B97A5019401C301B2010F9401
:10AD70006E46811111C02B962CAD3DAD4EAD5FAD31
:10AD80002B9727966CAD7DAD8EAD9FAD27970F9419
:10AD90006E46882309F4C3C0A3019201C501B40122
:10ADA0000F945F4D20E030E040E05FE30F94D44625
:10ADB00023966CAF7DAF8EAF9FAF239727962CADB8
:10ADC0003DAD4EAD5FAD27972B966CAD7DAD8EAD95
:10ADD0009FAD2B970F945F4D20E030E040E05FE3A4
:10ADE0000F94D4462B013C0120E030E0A901C701BB
:10ADF000B6010F946E46881F8827881F181709F41C
:10AE000076C180E090E0A0E8BFEB27968CAF9DAFC5
:10AE1000AEAFBFAF279723962CAD3DAD4EAD5FAD26
:10AE20002397CA01B9010F94D4464B015C01A301D9
:10AE30009201C301B2010F94D4469B01AC01C5013C
:10AE4000B4010F94604D0F940E504B015C01AC01A6
:10AE50009B01C701B6010F945F4D2B966CAF7DAF80
:10AE60008EAF9FAF2B97A5019401C701B6010F9438
:10AE7000604D9B01AC012B966CAD7DAD8EAD9FAD51
:10AE80002B970F94D4466B017C0120E030E0A901A0
:10AE90000F94C04F87FD30C1C701B6010F940E500B
:10AEA0006B017C01C301B2019058A50194010F947C
:10AEB0005A4E27962CAD3DAD4EAD5FAD27970F9402
:10AEC000D446A70196010F94D44623962CAD3DADF0
:10AED0004EAD5FAD23970F94604D69837A838B836A
:10AEE0009C83A501940123966CAD7DAD8EAD9FAD85
:10AEF00023970F945A4E27962CAD3DAD4EAD5FADC6
:10AF000027970F94D446A70196010F94D446A30126
:10AF100092010F94604D6D837E838F83988720E02C
:10AF200030E0A90169817A818B819C810F946E4602
:10AF30008111FAC020E030E0A9016D817E818F810E
:10AF400098850F946E468111EFC00E943A2B8CEDCC
:10AF500090E10E941B29BDC08C30910509F4F7C017
:10AF60008531910509F4B5C0049709F048C080E522
:10AF70000E94EF20C12CD12C7601882321F00E9461
:10AF80000C1D6B017C0183E50E94EF20882361F09A
:10AF90000E94732020E030E04AE754E40F94D44646
:10AFA0000F94D34E6B017C010E9435718091211862
:10AFB000811105C060E082EF90E10E942B9D0F940B
:10AFC000C612C60ED71EE81EF91E0F94C6126C19C3
:10AFD0007D098E099F0997FF7CC080E00E9438455B
:10AFE000F4CF8232910509F4BBC260F48C31910533
:10AFF00009F423C108F408C14D9709F4AEC20F94B7
:10B00000510667C08A35910509F437C300F58A9760
:10B01000B1F78091E609833008F45BC089E40E94AF
:10B02000EF20082F10E0882319F00E946F20182FBE
:10B030008AE40E94EF20F82E882309F4BDC20E9402
:10B040006F200111BCC2853008F4C2C2BAC28B3570
:10B05000910509F415C38C35910589F68091C007D7
:10B06000882309F411C38930A1F54BEBA42E42E0EB
:10B07000B42E59E7C52E52E0D52EE12C00E010E0A9
:10B08000F50181915F010E94EF20F82E882369F07D
:10B09000133011F0E82EF02E0E947320D6016D932C
:10B0A0007D938D939C9313970F2D1F5FB4E0CB0E70
:10B0B000D11C143029F7EE2009F445C30E94A2895F
:10B0C0000E94DB8F06C0233020F00E9413210E94D3
:10B0D000CD8A2D96FFAD2D97F11102C00F94080671
:10B0E0002C962FAD2C9720938D110C94986180E0B5
:10B0F00090E0A0E8BFE389CEC12CD12C7601D2CE5E
:10B1000089E40E94EF20882331F00E947320698334
:10B110007A838B839C838AE40E94EF20882309F43E
:10B12000FECE0E947320F7CE412FBE016F5F7F4F8E
:10B1300089E991E10F9443140F94C6126093ED08CE
:10B140007093EE088093EF089093F008C2CF84E0EC
:10B150000E946CA18111BDCF70E060E080E50E948B
:10B160000B228BAF66E070E083E50E940B228FAB71
:10B1700063E070E084E50E940B228C8F40E050E099
:10B1800060ED70E482E50E94FC2069837A838B8302
:10B190009C838091BC0787FD04C08091BD078370AC
:10B1A00069F160E088E50E942522F82E60E089E5DB
:10B1B0000E94252200E0811102E01091AF13812F3F
:10B1C0000E943B2360E085E40E94252291E08927CC
:10B1D00080935B020F299E01245E3F4FAE014F5FBB
:10B1E0005F4FBE01695C7F4FCE01CB960E94DB9220
:10B1F00010925B02812F0E943B236BCFFF24F394BC
:10B20000DBCF0E94083865CF87E00E946CA18111D6
:10B2100060CF8CE0EFEAF2E0DE01119601900D9232
:10B220008A95E1F770E060E080E50E940B22BE01A4
:10B230006F5F7F4F0E9424924CCFD0908E11C090B0
:10B24000590287E00E944287811111C08091BA079C
:10B250009091BB07A091BC07B091BD07EEE0B695F9
:10B26000A79597958795EA95D1F780FD32CF0E94F3
:10B27000357110925B026091AF138CE40E9425221D
:10B28000B82E80E00E943B230F94C6126093ED0815
:10B290007093EE088093EF089093F008A090BA1393
:10B2A00061E080E00E948AE510928E110E9413E511
:10B2B0008091750290917602A0917702B091780208
:10B2C00080938C0790938D07A0938E07B0938F0780
:10B2D000809151029091520290938B0780938A073C
:10B2E00084E690E0909352028093510281E0809333
:10B2F0009E090E94BE918091BA079091BB07A091D0
:10B30000BC07B091BD07A7FB112710F92B2F2170A7
:10B31000B1FB882780F9121303C0811709F418C103
:10B32000922E082F82E50E94EF20F82E60E070E058
:10B3300080EA90E4F1100E9473206BAF7CAF8DAF78
:10B340009EAF20E030E0A9010F946E46882359F0AB
:10B35000F11005C0111103C0992009F49CC0CE0161
:10B36000CB960F94370D112309F490C0992009F45E
:10B370006FC01092790210927A0210927B021092A2
:10B380007C0210927D0210927E0210927F02109237
:10B3900080020E94A2898091BA13EE24E394F12CDA
:10B3A000811103C0EE24EA94FE2C8EED9BE6ADE8FD
:10B3B000B2E48FAB98AFA9AFBAAFEBEDFAE165910C
:10B3C00075918591949120E030E040EC5FE30F941B
:10B3D000D446905869837A838B839C83E7EDFAE1A6
:10B3E000659175918591949120E030E040EC5FE3A8
:10B3F0000F94D4462B013C01B701FF0C880B990B2D
:10B400000F9475469B01AC01C301B2010F94D44661
:10B410006C8F7D8F8E8F9F8FAE01495C5F4FBE0119
:10B420006F5F7F4FCE014C960E942D890E94C9917B
:10B430001092790210927A0210927B0210927C0292
:10B4400010927D0210927E0210927F021092800272
:10B4500081E08093BA1380E00E94A68980917902EE
:10B4600090917A02A0917B02B0917C02809332028B
:10B4700090933302A0933402B09335021092BA1322
:10B4800080E00E94A68981E00E945C87992019F0E3
:10B4900081E00E94A689002349F01092E8081092EA
:10B4A000E7081092EA0882E00E94A6890E94A28919
:10B4B00080915902823024F181E08093BA1380E0B8
:10B4C0000E94A6898091790290917A02A0917B02D4
:10B4D000B0917C028093320290933302A0933402A5
:10B4E000B09335021092BA1380E00E94A68981E0E1
:10B4F0000E945C87C0925902D0928E110E9413E57F
:10B5000080919D0980939E09BB2019F081E00E94E3
:10B510003B2380918C0790918D07A0918E07B0916D
:10B520008F078093750290937602A0937702B09371
:10B53000780280918A0790918B07909352028093B2
:10B54000510260E08A2D0E948AE50E94DB8FC1CD06
:10B550009924939411E001E0E5CE0E94AE35B9CD77
:10B560000E9435718CE40E94A120182F882321F0BD
:10B570001092E8081092E7088AE50E94EF20082F51
:10B58000882311F40C94716B61E083E50E942522FD
:10B59000182F70E060E08AE50E94FC21813091055F
:10B5A00029F0029731F00093EA0893CD1093E80850
:10B5B000FACF1093E708F7CF80E0002349F0153069
:10B5C00028F08BEF90E10E941B2983CDF1103BCD39
:10B5D00090E1E9E7F2E0A9E9B1E101900D929A95D5
:10B5E000E1F7002391F094E0199FF0011124EC5051
:10B5F000F54E40815181628173814093991150933E
:10B600009A1160939B1170939C11FF2091F0A4E01C
:10B610008A9FF0011124E052F54E80819181A28130
:10B62000B38180939D1190939E11A0939F11B0932D
:10B63000A01140E050E0BA0186E40E94FC206B01BA
:10B640007C0120E030E0A9010F94C04F18168CF463
:10B6500020E030E040E752E4C701B6010F945A4EB3
:10B6600069837A838B839C83CE0101960E941A8F13
:10B6700030CD60E070E0CB01F3CF1092AA1329CD5A
:10B680008FE08093AA1325CD3BEBC32E32E0D32E5F
:10B69000F12CE12C00E010E0F60181916F010E9495
:10B6A000EF20382E882309F447C00E9473204B01F5
:10B6B0005C01133059F0F701EF54FD4E20813181C8
:10B6C000428153810F945F4D4B015C01F701E758B4
:10B6D000FD4F2081318142815381C501B4010F9416
:10B6E0005F4D2B013C012DEB37E346E855EB0F9402
:10B6F000C04F87FD0AC02DEB37E346E855E3C30191
:10B70000B2010F946E461816BCF4133021F1A70154
:10B7100045545C4E5A01A3019201D5016D917D9172
:10B720008D919C910F94604DF501608371838283AC
:10B730009383812F0E94B1861F5FF4E0EF0EF11C0E
:10B74000143009F0A9CF002309F4BACC85E892E0BF
:10B750000E949884B5CC8092850290928602A09235
:10B760008702B0928802032DE7CF8091C1079091A4
:10B77000C2078937910511F40C940C6408F0D5C107
:10B780008E34910509F4B7C508F0FBC08A319105E4
:10B7900009F447C408F093C08431910509F4EDC35E
:10B7A00008F06EC08131910509F4E4C308F042C08D
:10B7B000029708F024CC80E50E94EF20C12CD12C08
:10B7C0007601882321F00E940C1D6B017C0183E52A
:10B7D0000E94EF20882361F00E94732020E030E077
:10B7E0004AE754E40F94D4460F94D34E6B017C0186
:10B7F0000E9435718091BE079091BF07009709F4B0
:10B80000B4C30E94BCA18091C1079091C2076CE1B2
:10B8100071E1892B11F464E171E130E020E04BE348
:10B8200054E382E00E94652A40E0C701B6010E940D
:10B83000A7544FCC429709F0E2CB83E50E94EF205A
:10B84000882309F477C60F94C6126093ED087093AD
:10B85000EE088093EF089093F0080E94732020E098
:10B8600030E04AE754E40F94D4460F94D34E6093EB
:10B87000090270930A0280930B0290930C0229CC68
:10B880008731910509F4B3C380F48531910509F43A
:10B89000ABC3469709F0B3CB8091131B82FF02C064
:10B8A00087FF17CC0E94E8CF14CC8831910509F4AA
:10B8B000B5C3499709F0A3CB0E94D9530ACC803273
:10B8C000910509F43AC4B0F58D31910509F41EC40F
:10B8D00070F48B31910509F4B3C34C9709F08FCB09
:10B8E0008091BE079091BF070E94AEF8F2CB8E31D7
:10B8F000910509F412C44F9709F081CB0E94D791AA
:10B900006C8F7D8F8E8F9F8FBE016F5F7F4FCE01BB
:10B910004C960E944BAB60E0CE0101960E9434A190
:10B920000E943E2BBE016F5F7F4F8EE891E10E9427
:10B930008EF8CFCB8B34910509F4D5C4B0F48132A5
:10B94000910509F425C48934910509F058CB80E5A7
:10B950000E94EF20882309F4BCCB0E944B2085363F
:10B9600008F084E680930C08B4CB8C34910509F47C
:10B97000BEC48D34910509F042CB81E00E94FCA346
:10B98000A8CB8C36910509F4A4CB08F068C08535A6
:10B99000910509F40DC608F040C08235910509F4FF
:10B9A000B9C590F58035910509F479C581359105C2
:10B9B00009F025CB0E9446711092B0130E94BFDAA5
:10B9C00081E00E94FCA368EE73E080E090E00E94BA
:10B9D000C42460E088ED91E10E942B9D84E40E94E4
:10B9E000EF20182F811171C510E060E083E50E94FF
:10B9F0002522882309F488C581E08093E00986EC3C
:10BA000091E10E941B2965CB8335910509F48AC514
:10BA10008435910509F411CFF2CA8936910509F4EC
:10BA200073C460F48C35910509F4E7C58836910537
:10BA300009F0E5CA80E00E94A4AA4BCB8A369105A2
:10BA400009F490C48B36910509F0D9CA60E080E50D
:10BA50000E94192281113DCB1092B0133ACB82374C
:10BA6000910509F4CEC5A0F58F36910509F4A0C45F
:10BA7000C8F48D36910509F442C48E36910509F05B
:10BA8000BECA8EE40E94EF20882309F422CB0E94D4
:10BA90003B20609341137093421380934313909320
:10BAA000441317CB8037910509F413CB81379105E7
:10BAB00009F0A5CA83E50E94EF20882309F4B9C4E0
:10BAC0000E944B208D3308F0AFC48093080201CB55
:10BAD0008637910509F461C6C0F48337910509F4EE
:10BAE00098C58537910509F08ACA8091BE07909163
:10BAF000BF07009709F44DC6FC012081222309F4F9
:10BB000048C661E00E9434A1E4CA8737910509F470
:10BB10007FC68837910509F072CA81E080939E093B
:10BB200080939D090E94BE91D4CA8D3921E092076D
:10BB300011F40C94336B08F007C1893D910511F4A1
:10BB40000C94DD6608F05AC0893C910509F4D6C60C
:10BB500030F58B39910509F47BC460F48D3791057C
:10BB600009F4AACE8C38910509F049CA80E00E94F8
:10BB70005DAAAFCA8E3B910509F465C4883C910566
:10BB800009F03DCA8091BA0783FD4EC68091BC077B
:10BB90008C7009F049C681E00E9482349ACA8D3CBB
:10BBA000910509F470C7A8F48B3C910509F4E8C627
:10BBB0008C3C910509F023CA8091BB0787FD1BC708
:10BBC0008091BC078E7009F016C781E00E94AC33EB
:10BBD00080CA8E3C910511F40C94DA65833D910581
:10BBE00009F00DCA83E50E94A120882311F40C946A
:10BBF0000D660E945F2080935A026BCA8E3251E01C
:10BC0000950711F40C94626808F071C08D3D9105A0
:10BC100011F40C94306708F04AC08A3D910511F484
:10BC20000C94E1668C3D910509F0E9C982E40E941B
:10BC3000A120882341F0809151029091520290936B
:10BC40000E0280930D0282E50E94A120882341F01C
:10BC500080910D0290910E029093520280935102B6
:10BC600083E50E94EF20882331F00E946F2090939B
:10BC70005202809351028091BA079091BB07A09124
:10BC8000BC07B091BD07892B8A2B8B2B09F021CAE9
:10BC9000609151027091520286E095E10E949C35BC
:10BCA00085E20E94CA288AE00E94CA2812CA82320B
:10BCB000B1E09B0711F40C9463678D32914009F059
:10BCC0009EC96FEF85E40E941922082F9091BA0750
:10BCD00093FF02C00C94CF679091BB07917811F04D
:10BCE0000C94CF67682F81E00E94002FF2C9803941
:10BCF000F1E09F0711F40C94EA68D0F48F3241E030
:10BD0000940711F40C94A8688033914009F077C926
:10BD10008091BA0783FF02C00C9425688091BB070D
:10BD2000817811F00C94256881E00E94E230D1C93D
:10BD30008A39A1E09A0709F4CCC98C39914009F0FD
:10BD40005EC90E943B2EC5C98835E2E09E0711F40A
:10BD50000C94666A08F08EC0853F21E0920711F4CA
:10BD60000C94356A08F061C0893A51E0950711F4E6
:10BD70000C948C6908F04CC0843AB1E09B0711F434
:10BD80000C94EE68853A914009F039C988E50E9423
:10BD9000A120C82E89E40E94A120A82E882311F496
:10BDA0000C94F2680E946F20182F89E50E94A12050
:10BDB000F82E8AE40E94A120E82E882311F40C9426
:10BDC0001D690E946F20082F8AE50E94A120D82EAD
:10BDD000B12C811104C081E50E94A120B82EA110D0
:10BDE00001C0E12C8E2D90E0C11001C0F12C8F0D0F
:10BDF000911D019731F4D1100C944869B1100C9445
:10BE000048690E943A2B86EB95E10E941B2961C983
:10BE10008C3AF1E09F0711F40C949069843F9140B3
:10BE200009F0EDC80E946D9D54C9883F41E0940718
:10BE300011F40C943D6A98F4863FA1E09A0711F43E
:10BE40000C94396A873F914009F0D9C861E083E5D5
:10BE50000E94252291E089270E9405F43AC98C307E
:10BE6000E2E09E0711F40C94506A8F34924009F47A
:10BE700068CFC5C88C3623E0920709F42AC908F5B3
:10BE80008A3952E0950711F40C94F76A68F48B35FF
:10BE9000B2E09B0711F40C946A6A8D35924009F068
:10BEA000AEC80E94292915C98D3BF2E09F0711F405
:10BEB0000C941B6B8E3B924009F0A1C80E945D5010
:10BEC00008C9873E43E0940711F40C94236BB8F43F
:10BED0008438A3E09A0711F40C941F6B803A9340C6
:10BEE00009F08DC82091BE073091BF079091131BB8
:10BEF00092609093131BC9010E94AEF8EAC8883E75
:10BF0000E3E09E0711F40C94456B893E934009F0E1
:10BF100076C80E9435718091131B877F8B7F809339
:10BF2000131B8091091B81110C94496B0E943A22CA
:10BF30000E948DF90E94D7916D337105810591059D
:10BF400020F089E396E10E94EDBE85E396E10E9430
:10BF5000EDBE84EE80930C0881E296E10E941B29DD
:10BF60008DE196E10E94EDBEB4C884E291E10E94A9
:10BF700089A349CC0E942425ACC88091131B84FF5F
:10BF80002CC086E491E10E941B2960E08CE40E94B1
:10BF90002522182F8091131B84FF1AC083E39BE195
:10BFA0000E946FD08BE1E3E3FBE1DE01119601908B
:10BFB0000D928A95E1F730E020E0412F70E060E0DB
:10BFC000CE0101960E9498F9CE0101960E946A2244
:10BFD00087E391E10E941B297CC80E943E2B87E5E4
:10BFE00091E10E941B2975C80E9405D072C8E0919A
:10BFF000BE07F091BF078191882331F08032D9F7D5
:10C00000DF0111971C92F7CF60E08091BE079091FD
:10C01000BF070E94F5FA10920C085BC80E9438AC6A
:10C0200058C88091131B84FF54C883E50E94EF20F9
:10C03000882309F44EC80E943B200E942AAC49C8BC
:10C040008091BA079091BB07A091BC07B091BD0742
:10C0500022E0B695A795979587952A95D1F780FF09
:10C060002CC08BE691E10E941B2980917A1C8823C9
:10C07000F9F0BE016F5F7F4F87E79CE10E941BCF05
:10C08000CE0101960E9477C7CE0101960E94B5D0DD
:10C090008091B418882339F080E20E94CA2884EB8A
:10C0A00098E10E9477C78AE00E94CA280C946958D8
:10C0B00081E691E10E941B29F6CF83E50E94EF20E3
:10C0C000882301F10E944B20182F8C3308F08CE359
:10C0D000809394070F94C6126B017C01212F30E0EE
:10C0E000A8EEB3E00F94064DC60ED71EE81EF91E4B
:10C0F000C0929007D0929107E0929207F092930736
:10C100000C9469580E94A9C70C9469588091131B1C
:10C110008E7F8093131B0C9469588091131B84FDB0
:10C1200002C00C9469580F94920A8091BE079091B6
:10C13000BF070E9428F90C9469588091131B82FF55
:10C1400003C087FF0E9435718091131B84FD02C0DC
:10C150000C94695860E080E50E942522182F682F12
:10C160008091BE079091BF070E94F5FA83E50E9477
:10C17000EF20882321F00E943B200E942AAC0E94DD
:10C18000E0C711110C9469580E94359C0C946958B1
:10C190000091BE071091BF07D12CC12C01151105CC
:10C1A000C1F0F80101900020E9F731979F01201BB1
:10C1B000310B6901D801CD01801B910B82179307C8
:10C1C00044F48D918F32B9F7CD010197FC011082B3
:10C1D000F2CF8BE1E3E3FBE1DE015C9601900D928F
:10C1E0008A95E1F7F12CE12CEC14FD040CF05DC014
:10C1F000F801EE0DFF1D8081811103C0FFEFEF1AE2
:10C20000FF0A5801AE0CBF1CD5018C91882309F49C
:10C210004CC0BFEFEB1AFB0AF801EE0DFF1D7F01CA
:10C22000E01AF10A81918111FACFCE014C960E9459
:10C230006FD08BE1FE017C96DE01119601900D928C
:10C240008A95E1F7B501CE0101960E947AC8CE0128
:10C2500001960E946A228FE20E94CA288091B41837
:10C26000882361F184EB98E10E9477C78091131BCA
:10C2700085FF1BC019821C8221E0A501BE01645EFE
:10C280007F4FCE0101960E94E3D081111AC08AE04F
:10C290000E94CA280E943E2BB5018AE791E10E94C4
:10C2A000D0ACCE0101960E946A228AE00E94CA2880
:10C2B000CE014C960E946A220C94695887EA98E154
:10C2C000D3CFCE014C960E94CFCF8BE1FE013196A9
:10C2D000DE015C9601900D928A95E1F7CE01019600
:10C2E0000E946A2281CF0E94359C0C9469580E945A
:10C2F000EC9C0C9469580E9407AF0C94695881E03B
:10C300000E94A4AA0C9469580E94472B182F87FDFD
:10C310000AC08BE991E10E941B29812F0E9453D60C
:10C320008AE00E94CA282C96EFAD2C97E0938D11DD
:10C33000C45BDF4F0FB6F894DEBF0FBECDBFDF91F9
:10C34000CF911F910F91FF90EF90DF90CF90BF9012
:10C35000AF909F908F907F906F905F904F903F90A5
:10C360002F90089560E080E50E94192281110C94BD
:10C3700069588091BA070FEF10E080FF07C0E09185
:10C38000BA13F0E0E055FC4E6081062F83E50E9471
:10C39000EF20882349F00E943B208B016F3F7105FD
:10C3A00019F010F00FEF10E00093B0130C946958DF
:10C3B00083E50E94EF20882321F00E944B20809388
:10C3C000A9130E943E2B8CEA91E10E941B298091C7
:10C3D000A913882331F110E000E020E08091A91337
:10C3E00090E0002E02C0959587950A94E2F780FFB1
:10C3F00012C0FF24F394F20E222319F08CE20E9463
:10C40000CA28F801EE0FFF1FEE55FE4E859194915C
:10C410000E941B292F2D0F5F1F4F05301105F1F6CC
:10C4200042CE8EE991E146CE8CE3809308020C94D3
:10C4300069580E943E2B6091080283EB91E10E94B3
:10C440009FB10C94695881E00E945DAA0C946958D0
:10C4500083E50E94EF20882311F40C9469580E9410
:10C460004B20182F8C3308F08CE3809399070F949E
:10C47000C6126B017C01212F30E0A8EEB3E00F94CF
:10C48000064DC60ED71EE81EF91EC0929507D09223
:10C490009607E0929707F09298070C94695883E505
:10C4A0000E94A120882369F080918B09882331F0B4
:10C4B00080EC91E10E941B290C9469588AEB91E170
:10C4C000F9CF0E94E8240C9469580E943B206B012C
:10C4D0006230710508F488CA0F94C6124B015C01E2
:10C4E000960121503109A8EEB3E00F94064D860E57
:10C4F000971EA81EB91E8092E1099092E209A092AF
:10C50000E309B092E40971CA111179CA0E94F529B0
:10C510000C9469588091AA138F7D80618093AA132F
:10C520000C9469588091AA138F7E80628093AA131D
:10C530000C9469580E949D1B8823B1F10E943571AB
:10C5400085E40E94A120882351F080919A07909160
:10C550009B07892B31F10E946F200E949DF18BEB8C
:10C56000E82E82E0F82E10E0D7012D917D012154B4
:10C570008091BA079091BB07A091BC07B091BD070D
:10C5800004C0B695A795979587952A95D2F780FF11
:10C5900003C0812F0E94CCF11F5F133029F70C9448
:10C5A00069580E94B7F1DBCF0E9446710C9469581C
:10C5B00083E50E94A120882311F40C9469580F94FC
:10C5C000C6126093ED087093EE088093EF08909385
:10C5D000F0080E94732020E030E04AE754E40F9412
:10C5E000D4460F94D34E60939C0770939D0780931D
:10C5F0009E0790939F070C9469580E94EE2F0C940D
:10C6000069580F942D0A81E399E10E9424E40C9467
:10C61000695882ED93E10E941B2960E082EC93E16E
:10C620000E9483B160E08DEA93E10E9483B161E0F2
:10C6300086EA93E10E9483B161E08BE993E10E9475
:10C6400083B160E08CE893E10E9483B161E08CE704
:10C6500093E10E9483B160E083E793E10E9483B19C
:10C6600061E089E693E10E9483B160E08FE593E1A8
:10C670000E9483B161E088E593E10E9483B160E0AC
:10C6800080E593E10E9483B161E082E493E10E943E
:10C6900083B161E084E393E10E9483B161E085E2CC
:10C6A00093E10E9483B160E087E193E10E9483B14E
:10C6B00060E081E093E10E9483B161E080EF92E16C
:10C6C0000E9483B161E08BED92E10E9483B161E051
:10C6D0008CEC92E10E9483B161E085EC92E10E94D2
:10C6E00083B160E088EB92E10E9483B160E081EB6E
:10C6F00092E10E9483B161E088EA92E10E9483B1F5
:10C7000061E083E992E10E9483B161E085E892E112
:10C710000E9483B160E08BE792E10E9483B160E008
:10C7200084E692E10E9483B161E087E592E10E9494
:10C7300083B161E084E492E10E9483B160E087E329
:10C7400092E10E9483B161E082E392E10E9483B1B1
:10C7500061E085E292E10E9483B160E081E192E1D3
:10C760000E9483B160E08EEF91E10E9483B160E0AE
:10C7700086E19BE10E949CB1682F617085EF91E199
:10C780000E9483B160E087EE91E10E9483B10C9436
:10C7900069580F94FF090C9469580091BE071091D5
:10C7A000BF0794E0F12C40E0915009F1D8018C9141
:10C7B000282F2B7F2134A1F411962C912133B9F429
:10C7C000813419F1853409F441E098012E5F3F4F1F
:10C7D00089012F5F3F4FD8018C918032C9F3E4CF9C
:10C7E000803529F4F801818180538A3070F341113A
:10C7F0000E943E2BFF2021F084EA94E10E941B2935
:10C80000C8010E94AD860C946958FF24F394DDCFD3
:10C810000E943C910C94695810929E0910929D09B7
:10C820000E94BE910C9469580E94472B182F87FFD5
:10C8300002C00C946958F090B91384E40E94EF2070
:10C84000082F882309F456C00E9473206B017C01D5
:10C8500020E030E0A9010F946E46882309F44CC013
:10C86000B4E01B02F0011124EF54FC4EC082D182CF
:10C87000E282F38220E030E0A9016091B11370916F
:10C88000B2138091B3139091B4130F946E4681113B
:10C890000CC080E090E0A0EEBFE38093B1139093D2
:10C8A000B213A093B313B093B41320E030E0A90106
:10C8B0006091B5137091B6138091B7139091B8132E
:10C8C0000F946E4681110CC080E090E0A0EEBFE3B3
:10C8D0008093B5139093B613A093B713B093B81386
:10C8E000602F83E50E9425228093B9130E9409726C
:10C8F0000C9469580F2DF4CF80E0F6CF8091BA07E1
:10C9000084FD0DC08091BC07887849F48091BD07F3
:10C91000837029F481E00E9429340C9469580E94A4
:10C92000472B87FF02C00C9469581BEBC12E12E005
:10C93000D12EF12C03E0E02EE80EF60181916F017B
:10C940000E94EF208823B1F0F3E00E2DFF120F2D8F
:10C950000E94732024E0029F8001112407551E4E7F
:10C960000F94D34ED8016D937D938D939C93139721
:10C970000E94DE70F394B4E0FB12DFCF0C94695890
:10C980008091BA0784FD0DC08091BC07887849F476
:10C990008091BD07837029F481E00E94D4330C9408
:10C9A00069580E94472B87FF02C00C946958ABEB73
:10C9B000EA2EA2E0FA2E00E0B3E0DB2ED80EF7015B
:10C9C00081917F010E94EF20882381F01D2D03308B
:10C9D00009F0102F0E94732024E0129FF00111240F
:10C9E000EB52FE4E60837183828393830F5F04302A
:10C9F00031F70C94695883E50E94EF20882391F069
:10CA00000E9473206093E9117093EA118093EB11F7
:10CA10009093EC116093F1117093F2118093F311E4
:10CA20009093F41180E50E94EF20882351F00E943A
:10CA300073206093E9117093EA118093EB11909346
:10CA4000EC1182E50E94EF20882351F00E947320B0
:10CA50006093ED117093EE118093EF119093F011AC
:10CA600084E50E94EF20882311F40C9469580E94F9
:10CA700073206093F1117093F2118093F3119093EE
:10CA8000F4110C9469588091BA07827169F480910D
:10CA9000BC078C7849F48091BD07837029F481E04C
:10CAA0000E945A330C94695882E40E94EF20882334
:10CAB00051F00E940C1D6093BD117093BE118093C4
:10CAC000BF119093C01183E50E94EF20882351F09D
:10CAD0000E9473206093F5117093F6118093F71103
:10CAE0009093F81184E50E94EF20882351F00E9472
:10CAF00073206093F9117093FA118093FB11909356
:10CB0000FC1188E50E94EF20882351F00E947320D9
:10CB10006093F20A7093F30A8093F40A9093F50AF3
:10CB200089E50E94EF20882351F00E9473206093D2
:10CB3000F60A7093F70A8093F80A9093F90A8AE547
:10CB40000E94EF20182F882351F00E9473206093D9
:10CB5000FA0A7093FB0A8093FC0A9093FD0A85E41D
:10CB60000E94EF20882351F00E9473206093FE0AF8
:10CB70007093FF0A8093000B9093010B112311F423
:10CB80000C9469582DEC3CEC4CEC5DE36091FA0A96
:10CB90007091FB0A8091FC0A9091FD0A0F946E46F9
:10CBA000181614F40C94695887EA94E10E941B2922
:10CBB0000C9469588091BA079091BB07A091BC076B
:10CBC000B091BD07EBEBCE2EE2E0DE2EF7ECEF2EC0
:10CBD000F3E1FF2E10E0892B8A2B8B2B29F481E0C7
:10CBE0000E949DBE0C946958D6018D916D010E94E2
:10CBF000EF20882351F00E947320F7016083718336
:10CC000082839383812F0E94B1861F5FF4E0EF0E31
:10CC1000F11C133049F70C94605868EF74E181E01F
:10CC20000F948B0910915A02105D8FEE94E10E94CF
:10CC30001B29812F0E94CA288BEE94E10E941B2998
:10CC400080915A020E94162B4090B1125090B2125D
:10CC50006090B3127090B41220915C0230915D022A
:10CC600040915E0250915F02C301B2010F94604D8A
:10CC700023966CAF7DAF8EAF9FAF23978090B51298
:10CC80009090B612A090B712B090B81220916002A6
:10CC9000309161024091620250916302C501B4017A
:10CCA0000F94604D27966CAF7DAF8EAF9FAF2797E7
:10CCB000C090B912D090BA12E090BB12F090BC12A2
:10CCC00020916402309165024091660250916702A2
:10CCD000C701B6010F94604D2B966CAF7DAF8EAF40
:10CCE0009FAF2B97209168023091690240916A02B0
:10CCF00050916B02C301B2010F94604D2B013C01B6
:10CD000020916C0230916D0240916E0250916F0241
:10CD1000C501B4010F94604D4B015C01209170027C
:10CD2000309171024091720250917302C701B601B5
:10CD30000F94604D6B017C0183EE94E10E941B29EE
:10CD400023964CAD5DAD6EAD7FAD239785E69CE13E
:10CD50000E942A2E27964CAD5DAD6EAD7FAD279714
:10CD600082E69CE10E942A2E2B964CAD5DAD6EAD05
:10CD70007FAD2B9789EA9CE10E942A2E81EE94E1F7
:10CD80000E941B2989ED94E10E941B29B301A20195
:10CD900085E69CE10E942A2EB501A40182E69CE171
:10CDA0000E942A2EB701A60189EA9CE10E942A2E40
:10CDB0008AE00E94CA280C9469580E94A2310C94FF
:10CDC00069588091BA079091BB07A091BC07B091B8
:10CDD000BD07892B8A2B8B2B29F481E00E94542FCD
:10CDE0000C9469580E94472B182F87FF02C00C949F
:10CDF000695888E50E94EF20882361F00E94732023
:10CE00002CE01202F0011124EC5CFD4E6083718372
:10CE10008283938389E50E94EF20882361F00E943A
:10CE200073204CE01402F0011124EC5CFD4E64838D
:10CE30007583868397838AE50E94EF20882311F407
:10CE40000C9469580E9473205CE01502F0011124D3
:10CE5000EC5CFD4E60877187828793870C946958DC
:10CE60000E94472B082F87FF02C00C94695883E566
:10CE70000E94EF20882341F00E946F20BC01802F88
:10CE80000E94791D0C9469580E943E2B002E000CC4
:10CE9000110B85E40E94CA2880E3800F0E94CA28F3
:10CEA000000F111FF801E65CFD4F608171818AE07F
:10CEB00095E10E949C3585E20E94CA288AE00E9482
:10CEC000CA280C9469588AE50E94EF208823D9F17A
:10CED0000E94732020E030E040E050EC0F946E465A
:10CEE000C12CD12CE12C60ECF62E87FD13C00E94E2
:10CEF000732020E030E040E050E40F94C04FC12C9C
:10CF0000D12CE12C50E4F52E181624F00E94732049
:10CF10006B017C018090C9119090CA11A090CB1137
:10CF2000B090CC1184E00E944287811111C0A5010C
:10CF30009401C701B6010F94D4460F94CC4ECB0197
:10CF40000E949B2405C083E50E94EF208111C0CF81
:10CF50008091BC0787FD1CC08091BD078370C1F420
:10CF60000E943E2B40919B0850919C0860919D0827
:10CF700070919E088DE195E10E94852F60910D08CA
:10CF800070910E0882E195E10E94A9350C946958D0
:10CF900082E50E94A1208111E3CF0C9469588F3F54
:10CFA00051F082304CF00E943A2B8AE295E10E94C7
:10CFB0001B290C94695800E080E50E94EF2088232B
:10CFC00061F00E947320A7E10A02F0011124EC57DE
:10CFD000F74E608371838283938389E40E94EF20FC
:10CFE0008823B9F00E947320B7E10B02900111244D
:10CFF000F901EC57F74E7F012CEA35EC47E25EE38E
:10D000000F94D446D70114966D937D938D939C9382
:10D01000179784E40E94EF20882311F40C94695838
:10D020000E947320B7E10B02800111240C57174EA8
:10D030002CEA35EC47E25EE30F945A4EF801608724
:10D040007187828793870C94695880E50E94EF204E
:10D05000882351F00E94732060936D1870936E18AE
:10D0600080936F189093701889E40E94EF208823B2
:10D0700081F00E9473202CEA35EC47E25EE30F94C6
:10D08000D4466093711870937218809373189093BC
:10D09000741884E40E94EF20882311F40C946958DA
:10D0A0000E9473202CEA35EC47E25EE30F945A4E5F
:10D0B000609375187093761880937718909378180A
:10D0C0000C94695883E50E94A120182F882369F0E9
:10D0D0000E946F209C019093100280930F0291E0B8
:10D0E000232B09F090E09093A81380E50E94A120E3
:10D0F000882361F020910F0230911002232B11F050
:10D100000E945F208093A8130C94695811110C940D
:10D1100069580E943E2B88E595E10E941B29809169
:10D12000A813882391F080E495E10E941B29609167
:10D130000F027091100287E495E10E949C3583E410
:10D1400095E10E941B290C9469588CE395E1EDCF81
:10D1500070E060E085E40E94FC21182F8F3F91F081
:10D160002CF044EBE42EF12C82307CF080E995E148
:10D170000E941B2988E795E10E941B290F94AB04AC
:10D180000C94695836E4E32EF12C83E40E94EF20DE
:10D1900005E0882319F00E946F20082F83E50E9484
:10D1A000EF20882319F00E946F207C0160E085E564
:10D1B0000E942522D82E60E08BE695E10E942B9DEF
:10D1C0002D2D402F612FC7010E94B6DE0F94FF095D
:10D1D0000C9469580E9435710C9469580E94572C20
:10D1E0000C946958C11003C01FEF0C94D55E0E94C7
:10D1F00073202091B1123091B2124091B31250912C
:10D20000B4120F945F4D20E030E040E251E40F94FF
:10D210005F4D20E030E842E752E40F94604D23E395
:10D2200030E247E05CE30F94D4460F94CC4E162FC7
:10D23000653010F40C94D55ED7CFF11003C00FEF1A
:10D240000C94E45E0E9473202091B5123091B612C6
:10D250004091B7125091B8120F945F4D20E030E02A
:10D2600040E251E40F945F4D20E030E04AE752E4A1
:10D270000F94604D2FE632E143E05CE30F94D44617
:10D280000F94CC4E062F653010F40C94E45ED7CF8B
:10D2900017FD02C007FF08C00E943A2B8DE995E1F7
:10D2A0000E941B290C9469580E947320A12F110F12
:10D2B000BB0B002E000C110B20E030E0A901BB20BD
:10D2C00091F025E02A9FF0012B9FF00D1124E00F33
:10D2D000F11FEE0FFF1FEE0FFF1FE45BFD4E2081DD
:10D2E000318142815381E5E0FE2EFA9EF001FB9EE2
:10D2F000F00D11240E0F1F1F000F111F000F111F23
:10D30000045B1D4E0F94604DD8016D937D938D93FA
:10D310009C9313970C9469580E94E8340C946958B4
:10D3200087E00E946CA181110C94695866EAC62EB0
:10D330006AE1D62EE9E7F2E02196FFAFEEAF219742
:10D34000AE014F5F5F4F1A017A0110E000E0F60175
:10D3500065917591859194912196AEADBFAD219760
:10D360008D909D90AD90BD902196BFAFAEAF2197AF
:10D37000A50194010F945F4D2B013C01F701408200
:10D3800051826282738220E030E040EA51EC0F94D7
:10D39000C04F87FD0AC020E030E040EA51E4C301FD
:10D3A000B2010F946E46181684F4F801EE5AFB4C45
:10D3B000E4911E1654F4B7FAB094B7F8B094D701BC
:10D3C0008D929D92AD92BC921397F70181909190AE
:10D3D000A190B1907F0120E030E040EA51ECC5011E
:10D3E000B4010F94C04F87FD33C020E030E040EA25
:10D3F00051E4C501B4010F946E4618164CF10F5F4D
:10D400001F4FF4E0CF0ED11C0330110509F09FCF60
:10D4100057ECE52E53E1F52E10E0F1018191919149
:10D42000A191B1911F01F70181939193A193B193C0
:10D430007F01812F0E94B1861F5F133071F70E9418
:10D44000DB8F60E086ED95E10E942B9D0C9469587E
:10D450000E943A2B84EF95E10E941B2961E086EE41
:10D4600095E10E942B9D0C9469580E9492F70C94B0
:10D4700069580E943BF50C94695881E08093A30899
:10D480000E947B6F1092A308882311F40C946958B2
:10D490000E943E2B82E196E10E941B290C94695860
:10D4A0001091131B12FF0AC017FD08C00E941E2610
:10D4B00080FB17F91093131B0C94695814FD02C0DC
:10D4C0000C9469580F94920A0C9469580E948C52DB
:10D4D0000C9469588091BB0783FD09C08091BC07FB
:10D4E000887129F481E00E94F9430C9469580E94E4
:10D4F000472B082F87FF02C00C94695885E50E94CE
:10D50000EF20882359F10E9473204B015C01E02E2B
:10D51000002E000CFF0820E030E0A9010F94C04F5E
:10D5200087FF04C0B7FAB094B7F8B09420E030E0B9
:10D5300048E453E4C501B4010F94C04F970143E0A0
:10D54000220F331F4A95E1F72957374F1816D4F1A8
:10D55000D9018D929D92AD92BC9213978CE40E945A
:10D56000EF20882311F40C9469580E9473206B01FA
:10D570007C01002E000C110B20E030E0A9010F947B
:10D58000C04F87FF04C0F7FAF094F7F8F09420E05A
:10D5900030E048E453E4C701B6010F94C04F98014E
:10D5A00093E0220F331F9A95E1F72957374F18164A
:10D5B0009CF0D9011496CD92DD92ED92FC921797D2
:10D5C0000C94695880E090E0A8E4B3E4F90180830A
:10D5D0009183A283B383C2CF80E090E0A8E4B3E458
:10D5E000F90184839583A683B7830C94695880914D
:10D5F000BA079091BB07A091BC07B091BD07892BDA
:10D600008A2B8B2B29F481E00E94D4340C94695826
:10D610008AE50E94EF20882311F40C9469580E9437
:10D62000732060939708709398088093990890935B
:10D630009A080C9469580E949D4E0C9469580E9457
:10D640008E2B0C94695883E08093E6091092611840
:10D6500060E083E50E94252281110C9469580F94A3
:10D6600094090C94695883E50E94A120882341F015
:10D670000E945F2080937A110E9442220C94695884
:10D6800081E00E94222B0C9469580E9480400C94E7
:10D6900069580E94BBD381110C9469580C94965F11
:10D6A0001091C1070F94C6126093ED087093EE08B5
:10D6B0008093EF089093F008812F012E000C990BB6
:10D6C0002091BA132817190651F060E083E50E94F3
:10D6D0002522682F812F0E948AE50C94695881E0E9
:10D6E000F8CF11110C94D35A0C9469582F923F9291
:10D6F0004F925F926F927F928F929F92AF92BF9262
:10D70000CF92DF92EF92FF920F931F93CF93DF930D
:10D71000CDB7DEB766970FB6F894DEBF0FBECDBFAC
:10D72000DC01CD90DD90ED90FC90139714962D9137
:10D730003D914D915C9117972B873C874D875E8774
:10D7400020E030E040E251E4C701B6010F945F4DA4
:10D7500023E330E247E05CE30F94D4460F94CC4ED1
:10D7600064300CF41EC163E0662E660F7708F30187
:10D77000EE0FFF1FEE0FFF1FEC50F54E80809180E3
:10D78000A280B380F3013196FA83E98320E030E090
:10D7900040E251E46B857C858D859E850F945F4DBD
:10D7A0002FE632E143E05CE30F94D4460F94CC4E75
:10D7B00064300CF4FAC063E0062F660F110BF80119
:10D7C000EE0FFF1FEE0FFF1FEC50F54E2081318151
:10D7D000428153812B833C834D835E83A8014F5F3D
:10D7E0005F4F5E8B4D8BA5E0A69DC001A79D900D60
:10D7F0001124988B8F87FC01E00FF11FEE0FFF1FA4
:10D80000EE0FFF1FE45BFD4E208131814281538189
:10D810002F83388749875A87E981FA81EE0FFF1FE6
:10D82000EE0FFF1FEC50F54EA50194016081718150
:10D83000828193810F945F4D698B7A8B8B8B9C8B4C
:10D84000A5019401C701B6010F945F4D2B013C0166
:10D8500085E049815A81849F1001859F300C1124F5
:10D86000F101E00FF11FEE0FFF1FEE0FFF1FE45B52
:10D87000FD4E2F81388549855A856081718182816D
:10D8800093810F945F4D29893A894B895C890F9464
:10D890005A4EA30192010F94D4462F8138854985B1
:10D8A0005A850F94604D6B017C01EF85F889AD8935
:10D8B000BE89EA0FFB1FEE0FFF1FEE0FFF1FE45B99
:10D8C000FD4E80809180A280B380FD01E20DF31DAA
:10D8D000EE0FFF1FEE0FFF1FE45BFD4EA50194014D
:10D8E00060817181828193810F945F4D29893A898A
:10D8F0004B895C890F945A4EA30192010F94D44630
:10D90000A50194010F94604DA70196010F945F4DFE
:10D910004B015C01ED89FE89EE0FFF1FEE0FFF1F2B
:10D92000EC50F54E2B813C814D815E81608171818F
:10D93000828193810F945F4D9B01AC01C501B401BD
:10D940000F945A4E4B015C012B813C814D815E81CD
:10D950006B857C858D859E850F945F4D9B01AC0109
:10D96000C501B4010F94D446A70196010F94604DF0
:10D9700066960FB6F894DEBF0FBECDBFDF91CF9194
:10D980001F910F91FF90EF90DF90CF90BF90AF90DD
:10D990009F908F907F906F905F904F903F902F90CF
:10D9A000089567FFE1CE60E0DFCE67FF05CF60E05E
:10D9B00003CFFC017081472F50E0062E02C0559521
:10D9C00047950A94E2F740FF14C04091F10850E0F7
:10D9D000062E02C0559547950A94E2F740FF09C00C
:10D9E00021E030E001C0220F6A95EAF72095272355
:10D9F0002083089580918C11811106C081E090915F
:10DA00008D1193300CF480E0089580910B19909162
:10DA10000C19891B8F7089F48091981681110DC0A3
:10DA20008091020B9091030B892B39F481E0909146
:10DA3000A009911103C080E0089581E00895CF937B
:10DA4000DF93C0916A18D0916B1881E0CE31D10577
:10DA5000E4F020E030E040E05FE360916618709110
:10DA6000671880916818909169180F94604D0F9411
:10DA7000CC4E6C1B7D0B77FF03C0719561957109CE
:10DA800081E0633071050CF080E0DF91CF91089563
:10DA9000CF93C82FCB010E941B2983E09AE10E94FB
:10DAA0001B2984EF99E1CC2311F089EF99E1CF9103
:10DAB0000C947B404F925F926F927F928F929F92D5
:10DAC000AF92BF92CF92DF92EF92FF920F931F938C
:10DAD000CF93DF93CDB7DEB76C970FB6F894DEBF68
:10DAE0000FBECDBF8C015B015A834983FC01E05C12
:10DAF000FF4F20813181428153812D873E874F879F
:10DB0000588BCA01B9010F9473466B017C01D50192
:10DB10002D913D914D915C910F94D4460F943E4EC2
:10DB20002B013C01E981FA812081318142815381BD
:10DB3000C701B6010F94D4460F943E4E4B015C01D1
:10DB4000C301B2010F94D34E69877A878B879C8774
:10DB5000683771058105910540F428E730E040E021
:10DB600050E029873A874B875C87C501B4010F9441
:10DB7000D34E6D837E838F839887683771058105C7
:10DB8000910540F488E790E0A0E0B0E08D839E83AB
:10DB9000AF83B887F801E45BFF4F80809180A2805B
:10DBA000B380D80195962D913D914D915C919897B8
:10DBB00029833A834B835C8381149104A104B104CB
:10DBC00009F45DC1A7019601C701B6010F94D446BF
:10DBD0002B013C0169857A858B859C850F94734662
:10DBE0009B01AC010F94D4466D8B7E8B8F8B988FED
:10DBF000C501B4010F947546698B7A8B8B8B9C8B16
:10DC00009B01AC0160E070E080E09FE30F945A4E0E
:10DC10004B015C012D893E894F89588DC301B201AA
:10DC20000F945F4DA50194010F94D446698F7A8FAC
:10DC30008B8F9C8F0F943E4E0F94D34E6B017C01C3
:10DC40006D817E818F8198850F9473469B01AC0115
:10DC50000F94D4469B01AC01C301B2010F945F4DF8
:10DC6000A50194010F94D4462B013C010F94024F5F
:10DC70000F94D34E4B015C01D701C601880D991D4D
:10DC8000AA1DBB1D29813A814B815C81281B390B60
:10DC90004A0B5B0BDA01C901B7FF5FC069817A816A
:10DCA0008B819C810F947346298D3A8D4B8D5C8DB1
:10DCB0000F94604DA30192010F945F4D20E030E07E
:10DCC00040E05FE30F94D4460F943E4E6B017C011D
:10DCD00020E030E0A9010F94C04F18161CF0C12CB1
:10DCE000D12C7601C701B6010F94D34E6B017C0194
:10DCF00089819A81AB81BC818C159D05AE05BF05DC
:10DD000010F46C017D0189809A80AB80BC808C18F6
:10DD10009D08AE08BF08C701B6010F9473462B01DA
:10DD20003C0129893A894B895C89CA01B9010F9460
:10DD3000604D9B01AC01C301B2010F94D4462D8903
:10DD40003E894F89588D0F94604D0F940E500F945B
:10DD5000D34E6D877E878F87988BD8019A96CD9208
:10DD6000DD92ED92FC929D9789819A81AB81BC8175
:10DD700088199909AA09BB09F80186A797A7A0AB3A
:10DD8000B1ABEC5BFF4F29853A854B855C852083E1
:10DD900031834283538334968D819E81AF81B885D0
:10DDA00080839183A283B383F80187A990ADA1AD4D
:10DDB000B2AD892B8A2B8B2B09F44AC0F1A544E024
:10DDC000F49F900111242F5E364F3A872987D8019E
:10DDD00091966D917D918D919C9194970F9473463E
:10DDE000E985FA8520813181428153810F94D4469F
:10DDF0006B017C0169817A818B819C810F947346D0
:10DE00009B01AC01C701B6010F945A4E6B017C0116
:10DE10006D857E858F8598890F947346A70196013D
:10DE20000F94D4460F94D34ED801DD967C936E9315
:10DE3000DC976D817E818F8198850F947346A70151
:10DE400096010F94D4460F94D34EF80177AF66AF86
:10DE50006C960FB6F894DEBF0FBECDBFDF91CF91A9
:10DE60001F910F91FF90EF90DF90CF90BF90AF90F8
:10DE70009F908F907F906F905F904F900895812C2E
:10DE8000912C5401C12CD12C760167CFCF93C09136
:10DE90000C08CF7759F58091131B83FD2AC00E948F
:10DEA0001E26882319F180910B1B90910C1BA091C9
:10DEB0000D1BB0910E1B0097A105B105B9F0BC0177
:10DEC000CD016D597F4F8F4F9F4F24E630E040E0EA
:10DED00050E00F94B24C60910F1B7091101B809119
:10DEE000111B9091121B0F94B24CC22F8C2FCF910B
:10DEF0000895C4E6FBCF84E690E090938608809373
:10DF000085081092A5081092A4080C94D9FB0F93D1
:10DF1000AB010091A30821E0022724EA38E0BC010C
:10DF200085E898E00E9409270F910895CF93DF9329
:10DF300000D01F92CDB7DEB780918C098823A9F05D
:10DF400083E390E09C838B831A8219829E012F5F6A
:10DF50003F4F40E150E06DE879E0CE0103960E942A
:10DF60000B4086E69BE10E947B400F900F900F9044
:10DF70000F90DF91CF910895CF93DF9300D01F9240
:10DF80001F92CDB7DEB781E080938C0980E1EDE888
:10DF9000F9E0DF011D928A95E9F70E94966F86E10C
:10DFA0008D8382E390E09C838B831A8219829E0189
:10DFB0002F5F3F4F41E050E0BE016B5F7F4FCE01CE
:10DFC00003960E940B400F900F900F900F900F90B0
:10DFD000DF91CF9108954F925F926F927F928F92CF
:10DFE0009F92AF92BF92CF92DF92EF92FF92CF9328
:10DFF000DF9300D000D0CDB7DEB79E838D830E9423
:10E00000766B2B013C0120919B0830919C0840913C
:10E010009D0850919E08AD81BE8118966D917D91AD
:10E020008D919C911B970F945F4D4B015C01A30157
:10E0300092010F945F4D6B017C018091AB13909125
:10E04000AC13A091AD13B091AE1389839A83AB83C7
:10E05000BC8320E030E0A901BC01CD010F946E46E5
:10E06000882349F020E030E0A901C701B6010F94F0
:10E070006E461816ECF0AD81BE811896CD92DD92F9
:10E08000ED92FC921B9726960FB6F894DEBF0FBE5A
:10E09000CDBFDF91CF91FF90EF90DF90CF90BF90F9
:10E0A000AF909F908F907F906F905F904F9008956A
:10E0B00029813A814B815C81C501B4010F94C04F25
:10E0C00087FD07C0ED81FE8180869186A286B3869A
:10E0D000DACF209193113091941140919511509184
:10E0E0009611C301B2010F94D4469B01AC0160E0CC
:10E0F00070E080E89FE30F945F4D9B01AC01C70186
:10E10000B6010F945A4EAD81BE8118966D937D93E2
:10E110008D939C931B97B7CF80E00895FC0190816D
:10E1200093FB882780F993FF0E948C70811102C0B5
:10E1300081E0089580E008958F929F92AF92BF9200
:10E14000CF92DF92EF92FF920F931F93CF93DF93C3
:10E15000EC018A01072E000C880B990B0F94754671
:10E160004B015C01C880D980EA80FB80A701960141
:10E170000F94C04F18162CF488829982AA82BB8211
:10E1800010C0B801110F880B990B0F9475464B0105
:10E190005C01AC019B01C701B6010F94C04F18167A
:10E1A0005CF3DF91CF911F910F91FF90EF90DF9083
:10E1B000CF90BF90AF909F908F900895AF92BF92F5
:10E1C000CF92DF92EF92FF920F931F93CF93DF9343
:10E1D000D091BA13DD5F09EA11E184E2A82E88E04C
:10E1E000B82EC12CD12C7601C394C0E0F801619106
:10E1F0007191819191918F010F947346F801248957
:10E200003589468957890F94D4460F94D34EF5012A
:10E2100061937193819391935F01C33010F0DC138C
:10E2200007C0C616D706E806F90610F46B017C0194
:10E23000CF5FC530D9F66FEF7FEFCB01A701960115
:10E240000F94B24C20935A0830935B0840935C08BB
:10E2500050935D08DF91CF911F910F91FF90EF9048
:10E26000DF90CF90BF90AF90089590910B1980915F
:10E270000C19981306C08091971190919811892BD1
:10E2800021F080E00E943845F0CF089590910B195D
:10E2900080910C19981308C0809197119091981152
:10E2A000892B11F40C94FFF180E00E943845EECFE9
:10E2B0008F929F92AF92BF92CF92DF92EF92FF9296
:10E2C000CF93DF932091AF13222309F490C0EC0188
:10E2D0008090AB139090AC13A090AD13B090AE13A0
:10E2E000C884D984EA84FB8420E030E0A901C50118
:10E2F000B4010F946E46882309F484C020E030E016
:10E30000A901C701B6010F946E4618160CF07AC029
:10E31000A7019601C501B4010F946E4618160CF0C2
:10E3200054C0A701960160918F1170919011809156
:10E330009111909192110F946E46882321F1C09211
:10E340008F11D0929011E0929111F0929211209140
:10E350009311309194114091951150919611C701EC
:10E36000B6010F94D4469B01AC0160E070E080E8F8
:10E370009FE30F945F4D6093150270931602809394
:10E380001702909318028090150290901602A090A8
:10E390001702B090180220E030E0A901C501B401D5
:10E3A0000F946E46882389F0CE010E94766B9B0104
:10E3B000AC01C501B4010F94D446A70196010F9496
:10E3C000604D688779878A879B8720919B08309169
:10E3D0009C0840919D0850919E08688579858A85A2
:10E3E0009B850F94604D688779878A879B87DF912B
:10E3F000CF91FF90EF90DF90CF90BF90AF909F9024
:10E400008F900895812C912C80E8A82E8FE3B82E50
:10E41000CBCF7F928F929F92AF92BF92CF92DF929B
:10E42000EF92FF920F931F93CF93DF937090B913E6
:10E43000CFE0D8E09AE3C92E92E0D92E29E1E22E6E
:10E4400022E0F22E01EB13E1772009F45EC0F8011F
:10E4500080809180A280B38020E030E0A901C501D6
:10E46000B4010F946E46882309F44FC020E030E0D9
:10E4700040E05FE3C501B4010F94D4469B01AC01B9
:10E480000F94D4462BED3FE049E450E40F94D4467A
:10E490009B01AC0160E070E080E89FE30F945A4E6E
:10E4A0004B015C0189929992A992B992F60161910E
:10E4B00071916F01072E000C880B990B0F94754614
:10E4C0002AE037ED43E25CE30F94D446A5019401C2
:10E4D0000F94D446F70161937193819391937F01D7
:10E4E0000C5F1F4FF8E0C731DF0709F0ADCFDF91B8
:10E4F000CF911F910F91FF90EF90DF90CF90BF9041
:10E50000AF909F908F907F900895812C912C80E800
:10E51000A82E8FE3B82EC6CF80910B1990910C19BD
:10E52000891B8F7019F490E080E00895909108198C
:10E53000992351F0833030F48FEF890F19F08093D5
:10E540000819F1CF1092081980910C1925E6829FC5
:10E55000C0011124885D944FFC01208120FDE3CF90
:10E5600020910C192F5F2F702093091930910C19ED
:10E5700020910A19321304C02091091920930A1915
:10E58000089590916F0081E091FD02C080E00895B0
:10E5900090916F009D7F90936F000895EFE6F0E0FB
:10E5A00080818260808308952F923F924F925F9284
:10E5B0006F927F928F929F92AF92BF92CF92DF9293
:10E5C000EF92FF920F931F93CF93DF93CDB7DEB7F8
:10E5D000C358D1090FB6F894DEBF0FBECDBF7C0182
:10E5E0008B01242EE3963FAF2EAFE3978091600816
:10E5F00093E0940F892E912C27969FAE8EAE27978D
:10E60000F401EE0FFF1FEE0FFF1FEF53FE4E808051
:10E610009180A280B3808417D9F18D5FC82ED12C50
:10E62000F601EE0FFF1FEE0FFF1FEF53FE4EA50189
:10E63000940160817181828193810F946E46882359
:10E6400039F160913D1970913E1980913F19909177
:10E6500040190F947546A50194010F94D446F60114
:10E66000EE0FFF1FEE0FFF1FE05EFD4E2081318198
:10E67000428153810F94D4460F94CD4F60933D193E
:10E6800070933E1980933F1990934019209260082F
:10E69000D7012D913D914D915C91A9962CAF3DAF45
:10E6A0004EAF5FAFA9972091C1113091C211409137
:10E6B000C3115091C411A9966CAD7DAD8EAD9FADC7
:10E6C000A9970F94D4460F94CD4FEB966CAF7DAFC6
:10E6D0008EAF9FAFEB97D70114962D913D914D9141
:10E6E0005C911797AD962CAF3DAF4EAF5FAFAD9736
:10E6F0002091C5113091C6114091C7115091C81198
:10E70000AD966CAD7DAD8EAD9FADAD970F94D446FB
:10E710000F94CD4FEF966CAF7DAF8EAF9FAFEF975D
:10E72000D70118962D913D914D915C911B97E196E3
:10E730002CAF3DAF4EAF5FAFE1972091C911309143
:10E74000CA114091CB115091CC11E1966CAD7DADC9
:10E750008EAD9FADE1970F94D4460F94CD4FC15825
:10E76000DF4F688379838A839B83CF57D040D7015B
:10E770001C962D913D914D915C911F9769962CAF00
:10E780003DAF4EAF5FAF6997A501940169966CAD3F
:10E790007DAD8EAD9FAD69970F94D4460F94CD4F4C
:10E7A000A5966CAF7DAF8EAF9FAFA5978091A91353
:10E7B00083FF1CC0A5968CAC9DACAEACBFACA5973E
:10E7C00080923D1990923E19A0923F19B092401943
:10E7D00069968CAC9DACAEACBFAC699780922D199C
:10E7E00090922E19A0922F19B0923019D8013C9016
:10E7F00011968C9011978BAA12969C9012979BAEB3
:10E800001396AC90AFAE80910B1990910C19891BA7
:10E8100080958F7019F40E943845F5CFB0900B1990
:10E82000CD57DF4FB882C358D04070900B198091FC
:10E83000971190919811892B11F00C944B84809131
:10E84000311990913219A0913319B0913419EB9686
:10E850008CAC9DACAEACBFACEB97881A990AAA0AF7
:10E86000BB0A8BA29CA2ADA2BEA280913519909149
:10E870003619A0913719B0913819EF968CAC9DAC30
:10E88000AEACBFACEF97881A990AAA0ABB0A8FA24E
:10E8900098A6A9A6BAA68091391990913A19A09183
:10E8A0003B19B0913C19C158DF4F88809980AA80EC
:10E8B000BB80CF57D040881A990AAA0ABB0A809118
:10E8C0003D1990913E19A0913F19B0914019A5961C
:10E8D0002CAD3DAD4EAD5FADA597281B390B4A0B56
:10E8E0005B0B2DA73EA74FA758AB232B242B252B23
:10E8F00009F48BC0822D0E948122882331F1A596D4
:10E900008CAD9DADAEADBFADA59780933D199093F5
:10E910003E19A0933F19B093401969962CAD3DADB7
:10E920004EAD5FAD699720932D1930932E1940930A
:10E930002F19509330190E943E2B8EE09BE10E94CC
:10E940001B291DA61EA61FA618AA34E0239E80011F
:10E950001124075E1D4F6DA57EA58FA598A90F9464
:10E960007546D8012D913D914D915C910F94D446FF
:10E970006B017C0120E030E0A9010F94C04F87FFBC
:10E9800004C0F7FAF094F7F8F0942796EEADFFADD7
:10E990002797EE0FFF1FEE0FFF1FEF53FE4E20E0F5
:10E9A00030E048E453E460817181828193810F9467
:10E9B000D446A70196010F946E4687FF26C0A59600
:10E9C0002CAD3DAD4EAD5FADA59720933D19309375
:10E9D0003E1940933F195093401969968CAD9DADF7
:10E9E000AEADBFAD699780932D1990932E19A0936A
:10E9F0002F19B09330190E943E2B8FEE9AE10E949E
:10EA00001B291DA61EA61FA618AA8BA19CA1ADA1FD
:10EA1000BEA18827B7FD83959927AA27BB27182F62
:10EA20002FA138A549A55AA557FD1260B7FC14605F
:10EA30008DA59EA5AFA5B8A9B7FD1860A22DB0E021
:10EA40006596BFAFAEAF6597AA0FBB1FAA0FBB1FDE
:10EA50006B96BFAFAEAF6B97A75EBD4F7D016DA547
:10EA60007EA58FA598A90F947546F7012081318165
:10EA7000428153810F94D4466B017C0120E030E049
:10EA8000A9010F94C04F87FFC3C4C701B6019058B6
:10EA9000272D30E03AAB29AB45E6749E9001112456
:10EAA000D901A85DB44FBCA7ABA720E030E040E09F
:10EAB0005FE30F94604D0F94D34E6FAB78AF89AF87
:10EAC0009AAFEBA5FCA5108216AB2B968CAE9DAE33
:10EAD000AEAEBFAE2B97B7FE0DC022273327A901DC
:10EAE000281939094A095B092B962CAF3DAF4EAF67
:10EAF0005FAF2B978FA198A5A9A5BAA525968CAF36
:10EB00009DAFAEAFBFAF2597B7FF0DC0B095A09535
:10EB1000909581959F4FAF4FBF4F25968CAF9DAF7E
:10EB2000AEAFBFAF25972BA13CA14DA15EA12F9603
:10EB30002CAF3DAF4EAF5FAF2F9757FF0DC0509535
:10EB40004095309521953F4F4F4F5F4F2F962CAFFB
:10EB50003DAF4EAF5FAF2F972F968CAD9DADAEAD55
:10EB6000BFAD2F97EBA5FCA5858B968BA78BB08FA0
:10EB700025962CAD3DAD4EAD5FAD2597218F328FE3
:10EB8000438F548F2B962CAD3DAD4EAD5FAD2B9783
:10EB9000258F368F478F50A36BA17CA18DA19EA19D
:10EBA0000F9475462091201230912112409122122B
:10EBB000509123120F94D44663966CAF7DAF8EAF05
:10EBC0009FAF6397698B7A8B8B8B9C8B6FA178A59A
:10EBD00089A59AA50F94754620912412309125128B
:10EBE00040912612509127120F94D4462B013C01DC
:10EBF0004D8A5E8A6F8A788EC501B4010F9475467E
:10EC0000209128123091291240912A1250912B12F2
:10EC10000F94D446A1966CAF7DAF8EAF9FAFA197F6
:10EC2000698F7A8F8B8F9C8F2796EEADFFAD2797DC
:10EC3000EE0FFF1FEE0FFF1FE05EFD4E20813181C2
:10EC400042815381C701B6010F94D4466B017C0108
:10EC5000CD8EDE8EEF8EF8A22F962CAD3DAD4EAD53
:10EC60005FAD2F9726303105410551050CF0D3C318
:10EC700025968CAD9DADAEADBFAD25970697A10590
:10EC8000B1050CF0C8C32B962CAD3DAD4EAD5FADBC
:10EC90002B9726303105410551050CF0BCC320E00F
:10ECA00030E0A901C701B6010F94C04F87FF04C02F
:10ECB000F7FAF094F7F8F09485E689A89AA8889D69
:10ECC000F001899DF00D1124E85DF44FC586D686CC
:10ECD000E786F08A85E689A89AA8889DF001899D33
:10ECE000F00D1124E85DF44F8FA898ACA9ACBAAC34
:10ECF00081A292A2A3A2B4A2458D568D678D70A168
:10ED0000018D128D238D348DC588D688E788F08CCF
:10ED10005A01F62FE72F401751076207730718F4BF
:10ED20005801F22FE32FC501AF2FBE2F8C159D0583
:10ED3000AE05BF0510F4D701C6018FA898ACA9ACE9
:10ED4000BAAC88159905AA05BB0510F4D501C40114
:10ED5000F5E6BF2E89A89AA8B89CF001B99CF00DE1
:10ED60001124E85DF44F85A396A3A7A3B0A7069747
:10ED7000A105B10510F40C942E84DF01A05BBF4FF8
:10ED80008091B0138C9321A6CD28CE28CF2841F4B2
:10ED9000012B022B032B21F4452B462B472B11F083
:10EDA0000E94E82485E6A9A8BAA88A9DF0018B9D57
:10EDB000F00D1124E85DF44F85899689A789B08DFF
:10EDC000892B8A2B8B2B19F080E00E940AF285E6B2
:10EDD00089A89AA8889DF001899DF00D1124E85D0D
:10EDE000F44F818D928DA38DB48D892B8A2B8B2B23
:10EDF00019F081E00E940AF285E6A9A8BAA88A9DC6
:10EE0000F0018B9DF00D1124E85DF44F858D968DFA
:10EE1000A78DB0A1892B8A2B8B2B19F082E00E9441
:10EE20000AF28FA898ACA9ACBAAC89288A288B289A
:10EE300011F40C944D840E94E82480915E0888238C
:10EE400019F0815080935E0880915F08882319F043
:10EE5000815080935F08222029F080918E118823B1
:10EE600009F44FC480E00E9416E480E280935E08BB
:10EE70009924939429104DC481E00E94BDF180E251
:10EE800080935F08E090F511F090F6110091F71172
:10EE90001091F8119701A801632D7BA98BAD9FAD4F
:10EEA0000F946E4687FD04C0E32CFBA80BAD1FAD8D
:10EEB00085E6A9A8BAA88A9DF0018B9DF00D1124C2
:10EEC000E85DF44F85849684A784B088A5019401F9
:10EED00060E070E080E89FE30F945A4E2F966CAF8D
:10EEE0007DAF8EAF9FAF2F979701A8010F94D446A7
:10EEF0006B017C0180910B1990910919891B8F700E
:10EF000022968FAF2297A701960160E074E284E712
:10EF100099E40F945A4E0F94CD4F2B013C01229649
:10EF20008FAD229782508630A0F56091BD1170910F
:10EF3000BE118091BF119091C011641975098609A5
:10EF4000970916161706180619061CF5660F771F7F
:10EF5000881F991F2296AFAD22972A2F30E050E0EC
:10EF600040E00F94D44CCA01B9010F9475460F9438
:10EF7000CC4E640D751D861D971D0F9475469B0123
:10EF8000AC0160E074E284E799E40F945A4E6B019F
:10EF90007C01A7019601C501B4010F94D446639684
:10EFA0006CAF7DAF8EAF9FAF639785E689A89AA8B7
:10EFB000889D8001899D100D1124085D144F639672
:10EFC0008CAC9DACAEACBFAC6397D80111968D9262
:10EFD0009D92AD92BC92149795968D909D90AD9018
:10EFE000BC9098978BAA9CAAADAABEAAC501B401F1
:10EFF0000F9473466BAF7CAF8DAF9EAF9B01AC019E
:10F00000C701B6010F94D4460F943E4E0F94D34ED1
:10F01000A1966CAF7DAF8EAF9FAFA197F801E05C7A
:10F02000FF4F6083718382839383FE0171962196E3
:10F03000FFAFEEAF21979E012F5F3F4F29963FAF65
:10F040002EAF299745ED51E1E5965FAF4EAFE597BD
:10F05000CE014D969AA389A3E7963FAF2EAFE797CF
:10F06000212C312C90E89BA3AFE3AFA32196EEAD0A
:10F07000FFAD219721913191419151912196FFAF9F
:10F08000EEAF2197C701B6010F94D4464B015C0146
:10F09000E796AEADBFADE7978D929D92AD92BD92D2
:10F0A000E796BFAFAEAFE79720E030E0A9010F943D
:10F0B000C04F87FF04C0B7FAB094B7F8B094E59694
:10F0C000EEADFFADE5974190519061907190E5965E
:10F0D000FFAFEEAFE597A5019401C301B2010F9414
:10F0E0006E4687FF12C0A5019401C301B2010F94BF
:10F0F0005A4E5B018C0191014BA15FA10F946E46AA
:10F1000087FF03C015010BA31FA389A09AA0219616
:10F11000AEACBFAC21978A149B0409F0A7CF2D8D0C
:10F120003E8D4F8D58A1C701B6010F94D4466B0197
:10F130007C01CD86DE86EF86F88A20E030E0A901EA
:10F140000F94C04F4601570187FF04C0B7FAB0942F
:10F15000B7F8B0942796EEADFFAD2797EE0FFF1FDF
:10F16000EE0FFF1FEB52FE4E408051806280738095
:10F17000A5019401C301B2010F946E4687FF12C02E
:10F18000A5019401C301B2010F945A4E5B018C0199
:10F1900091014BA15FA10F946E4687FF03C015013B
:10F1A0000BA31FA320E030E040E85FE3B1018BA197
:10F1B0009FA10F946E4687FF65C091014BA15FA18F
:10F1C00069817A818B819C810F94D44669837A838B
:10F1D0008B839C8391014BA15FA16D817E818F8187
:10F1E00098850F94D4466D837E838F839887910191
:10F1F0004BA15FA169857A858B859C850F94D44648
:10F2000069877A878B879C8791014BA15FA1C70192
:10F21000B6010F94D4466D877E878F87988B85E6DD
:10F2200089A89AA8889D8001899D100D1124085DE8
:10F23000144F780120E4E20EF11CA1966CAD7DAD77
:10F240008EAD9FADA1970F94734691014BA15FA125
:10F250000F94D4460F94D34ED7016D937D938D9325
:10F260009C93139791014BA15FA163966CAD7DAD0B
:10F270008EAD9FAD63970F94D446F801618372837E
:10F28000838394832BAD3CAD4DAD5EAD2F966CADBD
:10F290007DAD8EAD9FAD2F970F94D4466FA378A709
:10F2A00089A79AA785E689A89AA8889DF001899DD3
:10F2B000F00D1124E85DF44F85889688A788B08CFE
:10F2C0008BA29CA2ADA2BEA289288A288B2809F015
:10F2D0002CC2818D928DA38DB48D892B8A2B8B2B83
:10F2E00009F023C2858D968DA78DB0A1892B8A2B1D
:10F2F0008B2B09F01AC22091ED113091EE11409143
:10F30000EF115091F0116FA178A589A59AA50F94DE
:10F31000D4460F943E4E0F94D34E2B013C01312C1A
:10F3200085E6A9A8BAA88A9D80018B9D100D11249D
:10F33000085D144FF801E45BFF4F40825182628206
:10F340007382C301B2010F9473466B017C012FA13C
:10F3500038A549A55AA50F945A4E2F966CAF7DAF8C
:10F360008EAF9FAF2F97D80151966D937D938D935C
:10F370009C9354972DEB37E346E051E4C701B60167
:10F380000F94D4460F94D34EF80162AB73AB84ABA9
:10F3900095AB17AA10AE11AE12AE13AE332009F41E
:10F3A00087C46B96EEADFFAD6B97EF5EF64F208195
:10F3B000318142815381C701B6010F94D4460F9425
:10F3C000D34EF80167AB70AF81AF92AF81A192A12C
:10F3D000A3A1B4A1880F991FAA1FBB1F4BA95CA9A9
:10F3E0006DA97EA922E076956795579547952A9550
:10F3F000D1F7FB96481759076A077B0708F458C4EA
:10F4000020812F5F2083880F991FAA1FBB1FF2CF77
:10F41000C701B6013DCBE396AEADBFADE397CD904E
:10F42000DD90ED90FC9020E030E0A901C701B6012D
:10F430000F946E46882309F424C185E629A93AA9C8
:10F44000829FF001839FF00D1124E85DF44FC58683
:10F45000D686E786F08A80912308012F08272BA102
:10F460003CA14DA15EA1232B242B252B09F40E7F5B
:10F470002FA138A549A55AA5232B242B252B09F408
:10F480000D7F89288A288B2809F40B7F8027809399
:10F49000230860912102611125C080911708909185
:10F4A0001808A0911908B0911A08892B8A2B8B2B68
:10F4B000C9F480911B0890911C08A0911D08B0917F
:10F4C0001E08892B8A2B8B2B69F480911F08909141
:10F4D0002008A0912108B0912208892B8A2B8B2B20
:10F4E00009F4F8CB70E090E080E00F94734620E0E0
:10F4F00030E04FE753E40F945A4E4B015C0149E76B
:10F5000058E058A74FA337E1C32E38E0D32EF12C93
:10F51000E12C812F90E023969FAF8EAF2397A02FF1
:10F52000B0E02D96BFAFAEAF2D97A5019401505816
:10F530002BA33CA34DA35EA3AFA1B8A54D905D90B6
:10F540006D907D90B8A7AFA320E030E0A901C30182
:10F55000B2010F946E46882309F487C023968EADBE
:10F560009FAD23970E2C02C0959587950A94E2F7DC
:10F57000B82FB1702896BFAF28972D962EAD3FAD0E
:10F580002D970E2C02C0359527950A94E2F720FF9F
:10F5900032C080FFB1C07BA16CA19DA18EA187016B
:10F5A000000F111F000F111F07551E4E272F362F5A
:10F5B000492F582FC301B2010F94D446F801208D72
:10F5C000318D428D538D0F94D4462B013C01D601D1
:10F5D0006D917D918D919C910F9475469B01AC012D
:10F5E000C301B2010F94604D0F94CC4EF6016083BD
:10F5F000718382839383F60180819181A281B3819B
:10F60000AC01BD01442777FD439555276627772731
:10F610002896FFAD2897F41328C00097A105B105DF
:10F6200021F1F701EE0FFF1FEE0FFF1F2BA53CA5E9
:10F63000E20FF31FB7FF07C0B095A0959095819595
:10F640009F4FAF4FBF4F458956896789708D840F93
:10F65000951FA61FB71F858B968BA78BB08FD601E2
:10F660001D921D921D921C921397BFEFEB1AFB0A7D
:10F67000E4E0CE0ED11CF3E0EF16F10409F05CCF0C
:10F6800029CB63962CAD3DAD4EAD5FAD6397CA01FE
:10F69000B9010F94D4466B017C01A3019201C3010F
:10F6A000B2010F94D4469B01AC01C701B6010F947F
:10F6B000604D6B017C01A1962CAD3DAD4EAD5FADB3
:10F6C000A197CA01B9010F94D4469B01AC01C701AF
:10F6D000B6010F94604D0F940E5025E649A95AA922
:10F6E000249FF001259FF00D1124E85DF44F6587FC
:10F6F00076878787908BAFCE782D692D9A2D8B2DAD
:10F700004ECF80915E0881110C9457840E949DF128
:10F71000AFCB80918E118111AFCB80915F088111A9
:10F72000B1CB81E00E949DF1ADCB8FA898ACA9AC84
:10F73000BAAC89288A288B2809F4B1C12091E91133
:10F740003091EA114091EB115091EC116FA178A525
:10F7500089A59AA50F94D4460F943E4E0F94D34E8C
:10F760002B013C018FA898ACA9ACBAAC89288A2897
:10F770008B2809F49DC16B96EEADFFAD6B97EF5EE4
:10F78000F64F80809180A280B3808FAA98AEA9AEF8
:10F79000BAAE20E030E0A901C501B4010F946E4675
:10F7A000882309F485C18DA49EA4AFA4B8A8181419
:10F7B00019041A041B040CF07BC12091211930910B
:10F7C00022194091231950912419A9966CAD7DAD51
:10F7D0008EAD9FADA9970F945F4D6DA77EA78FA7A4
:10F7E00098AB2091251930912619409127195091F5
:10F7F0002819AD966CAD7DAD8EAD9FADAD970F94D4
:10F800005F4D4B015C012091291930912A194091DB
:10F810002B1950912C19E1966CAD7DAD8EAD9FAD3D
:10F82000E1970F945F4D6B017C012DA53EA54FA57F
:10F8300058A9CA01B9010F94D4466DA77EA78FA716
:10F8400098ABA5019401C501B4010F94D4469B0166
:10F85000AC016DA57EA58FA598A90F94604D4B01B5
:10F860005C01A7019601C701B6010F94D4469B0124
:10F87000AC01C501B4010F94604D0F940E506B01A3
:10F880007C0120912D1930912E1940912F19509102
:10F89000301969966CAD7DAD8EAD9FAD69970F94B3
:10F8A0005F4DA70196010F945A4E6B017C0120E039
:10F8B00030E040E450E40F94C04F18160CF4F8C048
:10F8C000A70196016FA978AD89AD9AAD0F94D44682
:10F8D0009B01AC016091FE0A7091FF0A8091000BC0
:10F8E0009091010B0F945A4E2FA138A549A55AA506
:10F8F0000F94D4460F94D34E64157505860597056D
:10F9000010F42B013C013324339480915A089091D8
:10F910005B08A0915C08B0915D08EBA5FCA5C18CCB
:10F92000D28CE38CF48C858C968CA78CB0A08DA6A1
:10F930009EA6AFA6B8AA81A092A0A3A0B4A08FAAA9
:10F9400098AEA9AEBAAE8BA89CA8ADA8BEA88815E3
:10F950009905AA05BB0508F4ADC08BA09CA0ADA07D
:10F96000BEA081149104A104B104F1F060912408B7
:10F9700070912508809126089091270864157505D7
:10F980008605970588F42BA93CA94DA95EA90F947B
:10F99000A24CA50194010F94B24C241535054605DF
:10F9A000570510F429013A01C114D104E104F1040E
:10F9B000F1F0609128087091290880912A089091AF
:10F9C0002B08641575058605970588F42BA93CA9B5
:10F9D0004DA95EA90F94A24CA70196010F94B24CB9
:10F9E000241535054605570510F429013A018DA463
:10F9F0009EA4AFA4B8A881149104A104B104F1F0AD
:10FA000060912C0870912D0880912E0890912F08FC
:10FA1000641575058605970588F42BA93CA94DA9A1
:10FA20005EA90F94A24CA50194010F94B24C241529
:10FA300035054605570510F429013A018FA898AC01
:10FA4000A9ACBAAC81149104A104B10409F468CC46
:10FA50006596EEADFFAD6597EE0FFF1FEE0FFF1F32
:10FA6000E05DF74F60817181828193816415750536
:10FA70008605970508F054CC2BA93CA94DA95EA991
:10FA80000F94A24CA50194010F94B24C2415350596
:10FA90004605570508F044CC29013A0141CC209194
:10FAA000F1113091F2114091F3115091F4114ECEB9
:10FAB000312C2BCF8BA09CA0ADA0BEA089288A287A
:10FAC0008B28B9F16091240870912508809126084F
:10FAD00090912708641575058605970550F50F94D4
:10FAE00073462BAD3CAD4DAD5EAD0F94D4464B018E
:10FAF0005C016BA17CA18DA19EA10F9473469B011B
:10FB0000AC01C501B4010F945A4E4B015C01C30115
:10FB1000B2010F9473469B01AC01C501B4010F946F
:10FB20006E4687FF06C0C501B4010F94D34E2B016A
:10FB30003C01C114D104E104F104A9F16091280849
:10FB40007091290880912A0890912B0864157505F9
:10FB50008605970540F50F9473462BAD3CAD4DAD32
:10FB60005EAD0F94D4464B015C01C701B6010F9402
:10FB700073469B01AC01C501B4010F945A4E6B0151
:10FB80007C01C301B2010F9473469B01AC01C70114
:10FB9000B6010F946E4687FF06C0C701B6010F94E9
:10FBA000D34E2B013C018DA49EA4AFA4B8A8811410
:10FBB0009104A104B104A9F160912C0870912D0861
:10FBC00080912E0890912F0864157505860597057C
:10FBD00040F50F9473462BAD3CAD4DAD5EAD0F942B
:10FBE000D4466B017C01C501B4010F9473469B019F
:10FBF000AC01C701B6010F945A4E6B017C01C301E1
:10FC0000B2010F9473469B01AC01C701B6010F947A
:10FC10006E4687FF06C0C701B6010F94D34E2B0175
:10FC20003C018FA898ACA9ACBAAC81149104A10492
:10FC3000B10409F475CB6596EEADFFAD6597EE0F97
:10FC4000FF1FEE0FFF1FE05DF74F60817181828122
:10FC50009381641575058605970508F061CB0F94AF
:10FC600073462BAD3CAD4DAD5EAD0F94D4466B01EC
:10FC70007C01C501B4010F9473469B01AC01C7011F
:10FC8000B6010F945A4E6B017C01C301B2010F946F
:10FC900073469B01AC01C701B6010F946E4687FF06
:10FCA0003FCBC701B6010F94D34E2B013C0138CB9B
:10FCB00085E689A89AA8889DF001899DF00D1124F8
:10FCC000E85DF44F91809FAAA280ABAEB3802696E8
:10FCD000BFAE269784808FAE22EF3AE061963FAFA9
:10FCE0002EAF619729964EAC5FAC299730E1430E59
:10FCF000511C62EF262E6AE0362E29966EAC7FAC40
:10FD000029979BA2AFA2BDA68BAA10E0D301CD90EC
:10FD1000DD90ED90FD903D0120E030E0A901C701AC
:10FD2000B6010F94C04F87FF04C0F7FAF094F7F8BC
:10FD3000F094F10161917191819191911F0120E005
:10FD400030E0A9010F94604D4B015C01A7019601C1
:10FD50000F946E4687FF29C0112309F415C3A5012E
:10FD600094016FA97BAD26968FAD26979FAD0F941A
:10FD7000D4464B015C012BA13FA14DA55BA9C70156
:10FD8000B6010F94D4469B01AC01C501B4010F9498
:10FD90006E4687FF0AC0A7019601C501B4010F9402
:10FDA0005A4E6BA37FA38DA79BAB4614570409F053
:10FDB000ADCF22968FAC2297882009F437C32090CC
:10FDC0000D1930900E1900910F19109110192DEB8B
:10FDD00037E346E855E3B101C8010F946E4687FD4D
:10FDE00025C39101A8016FA97BAD26968FAD2697FB
:10FDF0009FAD0F946E4687FFDBC29101A8016FA9EA
:10FE00007BAD26968FAD26979FAD0F945A4E6D967B
:10FE10006CAF7DAF8EAF9FAF6D972FA83BAC269692
:10FE20000FAD26971FAD21E139E123963FAF2EAFED
:10FE30002397412C512C40E8642E4FE3742E649696
:10FE40001FAE64972396AEADBFAD23976D917D91A4
:10FE50008D919D912396BFAFAEAF23976D962CAD3C
:10FE60003DAD4EAD5FAD6D970F94D4464B015C0137
:10FE70002996EEADFFAD2997C190D190E190F19018
:10FE80002996FFAFEEAF29976496FFAD6497FF23E5
:10FE900071F0A30192010F94D4464B015C01A301C0
:10FEA0009201C701B6010F94D4466B017C01A701F2
:10FEB0009601C501B4010F94C04F20E030E0A901C4
:10FEC00018160CF092C2C701B6010F94C04F181655
:10FED0004CF020E030E0A901C501B4010F946E465A
:10FEE00087FF73C2A7019601C501B4010F945F4D4E
:10FEF0006B017C016196AEADBFAD61976D917D9157
:10FF00008D919D916196BFAFAEAF619720E030E0DB
:10FF1000A9010F94604D4B015C01A70196010F945C
:10FF20006E4687FF15C0A7019601C501B4010F9465
:10FF30005A4E9B01AC01C301B2010F94D4462B0170
:10FF40003C016496BFAD6497BF5F6496BFAF649792
:10FF5000E1E2F9E123968EAC9FAC2397E815F90511
:10FF600009F070CF64969FAC6497992041F0A3018B
:10FF70009201B101C8010F94D4461B018C0124EAFF
:10FF800030E74DE75FE3B101C8010F94D4466B0140
:10FF90007C012091560830915708409158085091A3
:10FFA00059080F946E4687FF0AC02BA13FA14DA5AB
:10FFB0005BA9C701B6010F946E4687FD37C28BA1BE
:10FFC0009FA1ADA5BBA98093560890935708A09315
:10FFD0005808B093590825E6A9A8BAA82A9DC001D7
:10FFE0002B9D900D11249C01285D344F79019101C6
:10FFF000A801B101C8010F94D446D70119966D9399
:020000021000EC
:100000007D938D939C931C972F966CAD7DAD8EAD9B
:100010009FAD2F9790589B01AC010F94604DEBA5BD
:10002000FCA525853685478550890F94D4469B01CC
:10003000AC016BE077ED83E29BE30F945F4D4B01E6
:100040005C018BE097EDA3E2BBE3F7018583968328
:10005000A783B087ABA5BCA58C9181608C932FA999
:100060003BAD26964FAD26975FAD6FA97BAD26962B
:100070008FAD26979FAD0F94D4469B01AC01C5016F
:10008000B4010F94C04F87FD05C0EBA5FCA580818E
:100090008260808380E1FE013196A1E1B9E10190A7
:1000A0000D928A95E1F785E689A89AA8889DF001C6
:1000B000899DF00D1124E85DF44F81819281A38127
:1000C000B48180930D1990930E19A0930F19B093DA
:1000D0001019EB968CAC9DACAEACBFACEB9780929C
:1000E000311990923219A0923319B0923419EF96C7
:1000F0008CAC9DACAEACBFACEF97809235199092B2
:100100003619A0923719B0923819C158DF4F88803C
:100110009980AA80BB80CF57D040809239199092A5
:100120003A19A0923B19B0923C19A5968CAC9DACA3
:10013000AEACBFACA59780923D1990923E19A092AB
:100140003F19B0924019DF01AF5ABF4FE0915508F7
:1001500024E0E29FF0011124E45FFD4E40815181D3
:10016000628173814D935D936D937C931397C090DF
:100170002D19D0902E19E0902F19F0903019209160
:10018000B5123091B6124091B7125091B8126091E9
:1001900025197091261980912719909128190F948B
:1001A000604D2B013C012091B9123091BA1240915F
:1001B000BB125091BC126091291970912A1980913B
:1001C0002B1990912C190F94604D4B015C010BA5DC
:1001D0001CA50B5A1F4F2091B1123091B2124091C1
:1001E000B3125091B412609121197091221980912B
:1001F0002319909124190F94604DD8016D937D932C
:100200008D939C931397EBA5FCA5E75AFF4F408273
:10021000518262827382EBA5FCA5E35AFF4F808274
:100220009182A282B382EBA5FCA5EF59FF4FC08259
:10023000D182E282F382A9968CAC9DACAEACBFAC0D
:10024000A9978092211990922219A0922319B09215
:100250002419AD968CAC9DACAEACBFACAD97809282
:10026000251990922619A0922719B0922819E19683
:100270008CAC9DACAEACBFACE1978092291990924A
:100280002A19A0922B19B0922C1969968CAC9DACAE
:10029000AEACBFAC699780922D1990922E19A092A6
:1002A0002F19B092301990910B1980910C19981355
:1002B00003C084E680930819CD57DF4F8881C35867
:1002C000D0408F5F8F7080930B1980910B199091A4
:1002D0000A1981508F70891709F4D7C110910B1931
:1002E00020900A1980910B19281609F432C1115077
:1002F0001F70D12CC12C121509F42BC1812E912C09
:1003000035E6A32E1A9DC00111249C01285D344FAF
:100310003CA72BA7C9010E948E70882309F416C13F
:10032000ABA4BCA4AB2811F125E6B22EB89CF00119
:10033000B99CF00D1124E85DF44FB1840285A384CB
:1003400034844580568067807084A30192016B2DB0
:10035000702F8A2D932D0F946E4681116FC0C1149A
:10036000D10421F0D6018C9180FD6CC011501F701A
:10037000822D20900A19281609F45DC0181709F477
:10038000E8C08F5F8F70F5CFA7019601C501B4015A
:100390000F945A4E9B01AC016BA17FA18DA59BA927
:1003A0000F94D4466BA37FA38DA79BAB11E0FDCC2C
:1003B000812C912C50E8A52E5FE3B52E6D968CAE66
:1003C0009DAEAEAEBFAE6D972ECDF7FAF094F7F8B6
:1003D000F094A7019601C501B4010F94C04F1816FF
:1003E0000CF088CD7501640185CDC701B6010F946D
:1003F0006E4687FD09C020E030E0A901C501B401C7
:100400000F94C04F18162CF4A5019401C701B60132
:100410006DCDB7FAB094B7F8B094A5019401C701B7
:10042000B6010F946E4687FF65CDDCCF2BA03FA0B1
:100430000DA51BA9C4CDCBA4DCA45DCFC114D104F0
:1004400009F45CC0F601C580D680E780F084B5E68B
:10045000B89DF001B99DF00D1124E85DF44F808145
:1004600081FD28C0618972898389948990589B0194
:10047000AC010F94604DEBA5FCA52585368547851D
:1004800050890F94D4469B01AC01C701B6010F946B
:100490005F4D6B0189AB9BA39B01AC016B2D702F52
:1004A0008A2D932D0F946E4687FD04C0BC2C0D2D14
:1004B000A9A83BA02B2D302F4A2D532DC301B201EB
:1004C0000F946E46882309F451CFF5E6F89DC001DC
:1004D000F99D900D11249C01285D344F6901D901CB
:1004E0008C9181608C938BA59CA50E946DE48823E0
:1004F00019F1F60180818E7F808338CFE396AEAD0F
:10050000BFADE3971896CD90DD90ED90FC901B97D2
:100510002BE037ED43E25BE3C701B6010F94C04F18
:1005200018160CF494CF9BE0C92E97EDD92E93E2C8
:10053000E92E9BE3F92E8BCF8B2D902FAA2DB32D77
:10054000F60185839683A783B08710CFDCA6CBA660
:100550000DCF10910A19F12CE12C05E680910B19B1
:10056000811709F492C0812E912C109FC001112493
:100570009C01285D344F3CA72BA7C9010E948E70B7
:10058000882309F47FC0E114F10409F46CC0C701A9
:100590000E946DE4811167C0D7018C9181FD4EC02E
:1005A000089DC001099D900D1124AC01485D544F78
:1005B0001A01DA0115964D905D906D907C90189718
:1005C000F701A580B680C780D084A6019501C3013C
:1005D000B2010F94C04F18168CF5D70151966D914A
:1005E0007D918D919C91549790589B01AC010F94F3
:1005F000604DF70125853685478550890F94D4468F
:100600009B01AC01C601B5010F945F4D6B017C01EC
:10061000AC019B01C301B2010F94C04F181674F4D2
:10062000D1018C9181608C938BA59CA50E946DE477
:100630008823F1F0F10180818E7F8083089DF00195
:10064000099DF00D1124E85DF44F21853285438525
:10065000548565817681878190850F946E468111DE
:1006600002C010930A191F5F1F70EBA4FCA476CF81
:10067000D1011596CD92DD92ED92FC9218971093D0
:100680000A19DCCFFCA6EBA6EECFF0900C19E09097
:100690000B1905E6FE1409F480C01FEF1E0D1F7034
:1006A000109FC0011124885D944F0E948E70882392
:1006B00009F471C0A12CB12C1BA619AA10E000E00E
:1006C000FE1409F471C0B5E6FB9EC0011124FC01C3
:1006D000E85DF44F6F01CF010E948E70882309F40A
:1006E0005EC0D60115966D917D918D919C91189764
:1006F0000F940E503B014C010115110509F442C045
:10070000F601808180FF04C0D8018C9181608C93B8
:10071000F801808180FF36C0C8010E946DE481111C
:100720002DC0D80111962D913D914D915C9114975A
:1007300060E070E080E89FE30F945A4E1B012C01AB
:10074000AC019B01B301C4010F94D44669837A8341
:100750008B839C8395014BA559A9C201B1010F94CC
:10076000D446698B7A8B8B8B9C8BAE014F5F5F4F2E
:10077000BE016F5E7F4FC8010E945A6DF8018081F3
:100780008E7F8083F394FF2DFF70FF2E53018BA685
:1007900099AA860195CFE12E7DCFEF2C8BCF350125
:1007A0008BA499A86801EECF0115110509F456C074
:1007B000E396AEADBFADE39718966D917D918D91A7
:1007C0009C911B970F940E506B017C012DEC3CEC1F
:1007D0004CE45DE30F94C04F181644F08DECC82E26
:1007E0008CECD82E8CE4E82E8DE3F82EF801808175
:1007F00081608083C8010E946DE481112BC0D80103
:1008000011962D913D914D915C91149760E070E0AF
:1008100080E89FE30F945A4E2B013C01A7019601FB
:100820000F94D44669837A838B839C83A3019201BE
:10083000B5018BA599A90F94D446698B7A8B8B8BC4
:100840009C8BAE014F5F5F4FBE016F5E7F4FC80153
:100850000E945A6DF80180818E7F80830E94CE7243
:1008600081E0CD57DF4F0FB6F894DEBF0FBECDBF8E
:10087000DF91CF911F910F91FF90EF90DF90CF907C
:10088000BF90AF909F908F907F906F905F904F90B0
:100890003F902F90089580E0E4CFE090F911F09020
:1008A000FA110091FB111091FC110C944A77B1E000
:1008B0002B120C948D7B0C943C77CF92DF92FF929D
:1008C0000F931F93CF93DF93CDB7DEB760970FB62B
:1008D000F894DEBF0FBECDBFFC018B01F42E690181
:1008E00090E1DE01119601900D929A95E1F7CE010B
:1008F00001960E9458718091971190919811892BBF
:10090000A9F496014F2DB801CE0101960E94D47230
:1009100060960FB6F894DEBF0FBECDBFDF91CF91CA
:100920001F910F91FF90DF90CF90089580E0F0CF5E
:10093000CF92DF92EF92FF92E091BA13E0936008BA
:10094000DC01CD90DD90ED90FC90ED5FB4E0EB9F8D
:10095000F0011124EF53FE4E2081318142815381F9
:10096000C701B6010F94D4460F94CD4F60933D1943
:1009700070933E1980933F1990934019C0922D199E
:10098000D0922E19E0922F19F092301990910B19F4
:1009900080910C19981731F0FF90EF90DF90CF9075
:1009A0000D9442110E9435710E94C17240913D190F
:1009B00050913E1960913F19709140194093CC08B5
:1009C0005093CD086093CE087093CF08882331F000
:1009D000FF90EF90DF90CF900C94CE72FF90EF904D
:1009E000DF90CF9008954F925F926F927F928F9297
:1009F0009F92AF92BF92CF92DF92EF92FF920F93AE
:100A00001F93CF93DF93CDB7DEB760970FB6F894FF
:100A1000DEBF0FBECDBF8C018091BA1380936008FA
:100A200090E1F801A1E2B9E101900D929A95E1F708
:100A30008D5F94E0899FF0011124EF53FE4ED801A1
:100A40001C962D913D914D915C911F976081718114
:100A5000828193810F94D4460F94CD4F6B017C011A
:100A60002091C9113091CA114091CB115091CC11F4
:100A7000F80160857185828593850F94D4460F9423
:100A8000CD4F4B015C012091C5113091C6114091B1
:100A9000C7115091C811D80114966D917D918D9117
:100AA0009C9117970F94D4460F94CD4F2B013C0186
:100AB0002091C1113091C2114091C3115091C411C4
:100AC000F80160817181828193810F94D4460F94E3
:100AD000CD4F6093311970933219809333199093ED
:100AE0003419409235195092361960923719709224
:100AF00038198092391990923A19A0923B19B09204
:100B00003C19C0923D19D0923E19E0923F19F092E3
:100B1000401990910B1980910C199817C9F00F94F6
:100B2000421160960FB6F894DEBF0FBECDBFDF91C5
:100B3000CF911F910F91FF90EF90DF90CF90BF90DA
:100B4000AF909F908F907F906F905F904F9008959F
:100B500080E1E1E3F9E1DE01119601900D928A95C1
:100B6000E1F7CE0101967C0110E0812F0E947C23E9
:100B7000D7018D909D90AD90BD907D01FD01349782
:100B8000DC01CB01880D991DAA1DBB1D80839183BB
:100B9000A283B3831F5F133041F70E9435710E9417
:100BA000C172182FCE0101960E9464E4112309F44A
:100BB000B8CF0E94CE72B5CFCF93DF93CDB7DEB75B
:100BC00060970FB6F894DEBF0FBECDBFFC0190E179
:100BD000DE01119601900D929A95E1F7CE010196F2
:100BE0000E945871CE0101960E94F38460960FB660
:100BF000F894DEBF0FBECDBFDF91CF9108950F9364
:100C00001F93CF93DF9301EC11E1C0E2D2E1F80131
:100C100021913191419151918F0160E070E080E824
:100C20009FE30F945A4E6993799389939993F2E1D4
:100C3000C433DF0761F789E792E00E94DC85DF912A
:100C4000CF911F910F910C94DE70CF92DF92EF92B3
:100C5000FF921F93CF93DF93182F0E94C17294E0ED
:100C6000199FE0011124FE01E054F74FC080D180AC
:100C7000E280F38081110E94CE72C701B6010F9409
:100C800075466B017C01812F0E947C23C05EDD4E86
:100C90000F9475469B01AC01C701B6010F945F4DDF
:100CA000288139814A815B810F94D446DF91CF91AD
:100CB0001F91FF90EF90DF90CF900895CF92DF9239
:100CC000EF92FF921F93CF93DF93182F0E94C17270
:100CD00024E0129FE0011124FE01EC54F74FC08084
:100CE000D180E280F38081110E94CE72812F0E9418
:100CF0007C23C05EDD4EA7019601261B370B480BF7
:100D0000590BCA01B9010F947546288139814A816E
:100D10005B810F94D446DF91CF911F91FF90EF90AC
:100D2000DF90CF9008950E94C17290910C1990931A
:100D30000B1990930A199093091994E69093081946
:100D400020ED33E0309398112093971181110E9488
:100D5000CE7281E08093B30808950E9477C70C9407
:100D600071C7CF93DF9324E0829FC0011124EC016F
:100D7000CF54DD4EFC01E953FC4E85549C4EDC0102
:100D80002D913D914D915C91608171818281938122
:100D90000F94604D688379838A839B83DF91CF9121
:100DA0000895CF92DF92EF92FF92282F30E041E03A
:100DB00050E0082E01C0440F0A94EAF79091F00A1F
:100DC000942B9093F00A9091F108492B4093F108ED
:100DD000811135C09091BA13913061F04091590260
:100DE000423069F5C12CD12C3CE4E32E32ECF32ED9
:100DF0009923C1F0C0904012D0904112E09042126D
:100E0000F090431220E030E0A901C701B6010F9431
:100E1000C04F18163CF0C12C20ECD22E29E0E22E57
:100E200024E4F22EC0927902D0927A02E0927B0200
:100E3000F0927C02FF90EF90DF90CF900895220F08
:100E4000331F220F331FF901EA55F54E4591559195
:100E500065917491F901E758FD4F40835183628396
:100E6000738310920E0810920D0825543C4EF90120
:100E70001082118212821382FF90EF90DF90CF9048
:100E80000C94B186CF93DF931F92CDB7DEB78983E1
:100E900060E0CE0101960E94D96C61E0CE0101961E
:100EA0000E94D96C62E0CE0101960E94D96C8981C2
:100EB0000F90DF91CF9108950F931F931092F20836
:100EC0001092F3081092F4081092F50880935408D9
:100ED000882381F18091810290918202A091830206
:100EE000B091840240917D0250917E0260917F0218
:100EF000709180020091790210917A0220917B0218
:100F000030917C02009348081093490820934A08C6
:100F100030934B0840934C0850934D0860934E0813
:100F200070934F088093500890935108A0935208F3
:100F3000B09353081F910F91089580938E1167FF0E
:100F40006093BA130C9413E58F929F92AF92BF9265
:100F5000CF92DF92EF92FF92CF93DF9320915A02CC
:100F6000222309F48EC0EC018091F108E82E80FF65
:100F70002CC080905C0290905D02A0905E02B090C8
:100F80005F02288139814A815B81C501B4010F94D8
:100F9000C04F181624F488829982AA82BB8280905E
:100FA000680290906902A0906A02B0906B0228815A
:100FB00039814A815B81C501B4010F946E4687FF78
:100FC00004C088829982AA82BB82E1FE2CC08090F4
:100FD000600290906102A0906202B09063022C8146
:100FE0003D814E815F81C501B4010F94C04F181639
:100FF00024F48C829D82AE82BF8280906C0290909D
:101000006D02A0906E02B0906F022C813D814E81E6
:101010005F81C501B4010F946E4687FF04C08C82C6
:101020009D82AE82BF82E2FE2CC0C0906402D0904E
:101030006502E0906602F0906702288539854A854E
:101040005B85C701B6010F94C04F181624F4C886FB
:10105000D986EA86FB86C0907002D0907102E0903B
:101060007202F0907302288539854A855B85C70135
:10107000B6010F946E4687FF04C0C886D986EA86FB
:10108000FB86DF91CF91FF90EF90DF90CF90BF90E4
:10109000AF909F908F900895CF93DF93CDB7DEB739
:1010A0002C970FB6F894DEBF0FBECDBF19821A82FF
:1010B0001B821C821D821E821F82188619861A8638
:1010C0001B861C869E012F5F3F4F4091BA13BC01C7
:1010D00089E792E00E945D842C960FB6F894DEBFFB
:1010E0000FBECDBFDF91CF9108954F925F926F9267
:1010F0007F928F929F92AF92BF92CF92DF92EF92A8
:10110000FF920F931F93CF93DF93CDB7DEB72C974A
:101110000FB6F894DEBF0FBECDBF2B013C0129876F
:101120003A874B875C8747015801F601E080F180E0
:101130000281138120E030E0A901B701C8010F94BA
:101140006E46882309F484C05E2D4F2D302F212F49
:10115000852F942FA32FB22F89839A83AB83BC83CF
:1011600020E030E0A901B701C8010F946E4681115B
:1011700004C0E12CF12C00E810E4C701D8018D83F4
:101180009E83AF83B887A50194016091810270911D
:10119000820280918302909184020F946E4687FFB1
:1011A0000CC08092810290928202A0928302B0923F
:1011B0008402CE0105960E944C884092790250929A
:1011C0007A0260927B0270927C0289859A85AB8557
:1011D000BC8580937D0290937E02A0937F02B093A2
:1011E0008002CE0101960E944C88A5019401609175
:1011F00081027091820280918302909184020F9407
:10120000C04F181664F48092810290928202A092DC
:101210008302B0928402CE0105960E944C880E94FF
:1012200035712C960FB6F894DEBF0FBECDBFDF919F
:10123000CF911F910F91FF90EF90DF90CF90BF90D3
:10124000AF909F908F907F906F905F904F90089598
:1012500050E040E035E023E47BCFCF92DF92EF9285
:10126000FF920F931F936A01E0908102F090820237
:101270000091830210918402FB012081318142811F
:101280005381FC0160817181828193810E94758804
:101290001F910F91FF90EF90DF90CF900895CF9224
:1012A000DF92EF92FF920F931F936B01FC01E0809E
:1012B000F18002811381E9E7F2E0248135814681E2
:1012C000578160817181828193810E9475881F910D
:1012D0000F91FF90EF90DF90CF900895EF92FF92E3
:1012E0000F931F93CF93DF937C018B010E94C02546
:1012F000C9E7D2E0E091BA1384E0E89FF00111243D
:10130000E75EFD4F2081318142815381F701608189
:101310007181828193810F945A4E2C853D854E8533
:101320005F850F94604D6C877D878E879F87C8018E
:101330000E944C88DF91CF911F910F91FF90EF9009
:101340000C94357189E792E00C94DC852F923F92E2
:101350004F925F926F927F928F929F92AF92BF92C5
:10136000CF92DF92FF920F931F93CF93DF93F82ECC
:10137000C82FD0E081110BC08091BA13CC24CA943D
:10138000DC2C882389F0CC24C394D12C0DC0FE0121
:10139000EE5AFB4CC4900C2C000CDD0882E0F812D5
:1013A00003C081E08093EA08B6010D2C000C880B85
:1013B000990B0F9475464B015C011E01220C331CE6
:1013C000220C331CF101ED51F54E259135914591DB
:1013D0005491C501B4010F94D4462B013C01F10195
:1013E000E952F54E659175918591949120E030E038
:1013F00040EC5FE30F94D446A50194010F94D446CA
:10140000AB01BC0100E010E098018F2D0F94930D0B
:1014100020E030E0A901C301B2010F946E46882399
:1014200009F446C0B301A201705800E010E0980131
:101430008F2D0F94930DA3019201C301B2010F945C
:10144000604D2B013C01CC52D54EFE01C491C1111F
:1014500007C00E943E2B82EB9AE10E941B29CAE042
:10146000FF2039F0F1E060E070E080E793E4FF12E4
:1014700004C060E070E88BE395E420E030E040E7F2
:1014800052E40F945A4E4B015C016C2F70E090E0D7
:1014900080E00F9473469B01AC01C501B4010F9429
:1014A0005A4E8B019C01B301A2018F2D0F94930D15
:1014B00082E0F8124CC08090970890909808A09015
:1014C0009908B0909A0820E030E0A901C501B40164
:1014D0000F94C04F2401350187FF04C077FA709440
:1014E00077F8709420E030E0A901C301B2010F94B5
:1014F0006E46882351F120E030E0A901C501B40116
:101500001C141D0444F40F94C04F181644F081E0DD
:101510008093E70807C00F946E4687FFF8CF81E0FD
:101520008093E8081C141D0424F477FA709477F86B
:10153000709400E010E09801B301A20182E00F94E2
:10154000930D1092E8081092E7081092EA088F2D88
:101550000E94D1860E94A289F101E756FE4ED10178
:10156000A758BD4F8D919D910D90BC91A02D80836A
:101570009183A283B383DF91CF911F910F91FF904D
:10158000DF90CF90BF90AF909F908F907F906F90A3
:101590005F904F903F902F9008952F923F924F92DF
:1015A0005F926F927F928F929F92AF92BF92CF92F3
:1015B000DF92EF92FF920F931F93CF93DF93CDB7FC
:1015C000DEB7C054D1090FB6F894DEBF0FBECDBF51
:1015D00089E991E10E94A4878091A91383FD76C0D7
:1015E00020918502309186024091870250918802B5
:1015F0006091A5117091A6118091A7119091A811E9
:101600000F946E46882309F461C08091BA130E943A
:101610008122182F882331F00E943E2B89E79AE11E
:101620000E941B29209185023091860240918702F9
:10163000509188026091A5117091A6118091A71117
:101640009091A8110F945F4D6B017C0120E030E078
:10165000A9010F94C04F87FF04C0F7FAF094F7F880
:10166000F094E091BA1324E0E29FF0011124E75EC8
:10167000FD4F2081318142815381C701B6010F9412
:10168000D44620E030E048E453E40F94C04F1816ED
:10169000DCF40E943E2B8AE59AE10E941B2980918E
:1016A000A5119091A611A091A711B091A8118093B6
:1016B000850290938602A0938702B093880285EA00
:1016C00091E10E94988402C01111E9CF80915408E1
:1016D000882349F080915902813009F470C01CF0D0
:1016E00084300CF484C12AE037ED43E25CE360917E
:1016F00075027091760280917702909178020F9432
:10170000D4466B017C016091510270915202072E08
:10171000000C880B990B0F9475469B01AC01C70117
:10172000B6010F94D44669A37AA38BA39CA380919E
:10173000AF13882311F18090AB139090AC13A0905D
:10174000AD13B090AE13C090A111D090A211E09053
:10175000A311F090A41120E030E0A901C501B4016B
:101760000F946E46882309F4C5C1A5019401C701F1
:10177000B6010F946E4687FDBDC119821A821B8285
:101780001C821D821E821F82188619861A861B865D
:101790001C869E012F5F3F4F4091BA13BE016F5DC3
:1017A0007F4F89E991E10E945D8480E1E9E9F1E1FF
:1017B000A9E7B2E001900D928A95E1F75BC0C09075
:1017C0008502D0908602E0908702F0908802809097
:1017D000500890905108A0905208B0905308209162
:1017E000A5113091A6114091A7115091A811C701E0
:1017F000B6010F946E46811157C08091F208909106
:10180000F308A091F408B091F5088F3F9F4FAF4FB8
:10181000BF4F09F449C080E1E9E9F1E1A9E7B2E08D
:1018200001900D928A95E1F7C090A111D090A2117C
:10183000E090A311F090A411A5019401C701B60195
:101840000F94C04F181644F4C0925008D09251081B
:10185000E0925208F09253080F94C61268517C4FE0
:101860008F4F9F4F6093F2087093F3088093F408B2
:101870009093F508C05CDF4F0FB6F894DEBF0FBE43
:10188000CDBFDF91CF911F910F91FF90EF90DF902F
:10189000CF90BF90AF909F908F907F906F905F9010
:1018A0004F903F902F9008958091DD119091DE111F
:1018B000A091DF11B091E01189AB9AABABABBCAB9F
:1018C0008091480890914908A0914A08B0914B082E
:1018D000898B9A8BAB8BBC8B80914C0890914D0877
:1018E000A0914E08B0914F088D8B9E8BAF8BB88F17
:1018F000898E9A8EAB8EBC8ECD8EDE8EEF8EF8A248
:1019000019821A821B821C821D821E821F821886E7
:1019100019861A861B861C869E012F5F3F4F4091B9
:10192000BA13BE016F5C7F4FCE0141960E945D8469
:10193000882309F456C080E1E9E7F2E0DE01119660
:1019400001900D928A95E1F780915008909151088D
:10195000A0915208B091530889879A87AB87BC87BA
:1019600019A21AA21BA21CA21DA21EA21FA218A687
:1019700019A61AA61BA61CA6A090BA13E090D9110E
:10198000F090DA110091DB111091DC119090D511DB
:10199000B090D611C090D711D090D811292D3B2DE1
:1019A000A601B701C8010F94C04F18161CF4E92C0A
:1019B000FB2C8601C701D8018DA79EA7AFA7B8ABA6
:1019C0009E012F5D3F4F4A2DBE01635D7F4FCE01CB
:1019D00001960E945D84882321F0CE01C1960E9469
:1019E0004C880E9413E580E00E945C877CCE809149
:1019F000BA13811178CE10928E110E9413E5C09017
:101A00007902D0907A02E0907B02F0907C0280E133
:101A1000E9E7F2E0DE01519601900D928A95E1F737
:101A20008091320290913302A0913402B09135023C
:101A3000898B9A8BAB8BBC8BCE0141960E94DC8547
:101A400080E1FE017196DE01119601900D928A955A
:101A5000E1F780915902A7019601823079F56091F2
:101A600055027091560280915702909158020F943E
:101A7000604D69837A838B839C8319A21AA21BA26F
:101A80001CA21DA21EA21FA218A619A61AA61BA65A
:101A90001CA69E012F5D3F4F41E065ED71E1CE0137
:101AA00001960E945D84882309F41DCE0E94357141
:101AB0000E94A28981E080938E1193CF60E070E84C
:101AC0008CEF93E40F945F4D6B017C0120E030E8D4
:101AD0004CEF53E40F946E4687FD07C0C12C90E88D
:101AE000D92E9CEFE92E93E4F92EC982DA82EB829B
:101AF000FC82C3CF2091790230917A0240917B021F
:101B000050917C026091991170919A1180919B1172
:101B100090919C110F945F4D6DAB7EAB8FAB98AFE6
:101B200020917D0230917E0240917F02509180028F
:101B300060919D1170919E1180919F119091A011C3
:101B40000F945F4D69AF7AAF8BAF9CAF209181024C
:101B5000309182024091830250918402C701B60104
:101B60000F945F4D21966CAF7DAF8EAF9FAF2197E5
:101B7000209185023091860240918702509188021F
:101B80006091A5117091A6118091A7119091A81153
:101B90000F945F4D4B015C0120E030E0A9016DA97D
:101BA0007EA98FA998AD0F946E4681110CC020E0DC
:101BB00030E0A90169AD7AAD8BAD9CAD0F946E4656
:101BC000882309F4DACD2DA93EA94FA958ADCA0141
:101BD000B9010F94D4466B017C0129AD3AAD4BADF0
:101BE0005CADCA01B9010F94D4469B01AC01C70199
:101BF000B6010F94604D6B017C0121962CAD3DAD7B
:101C00004EAD5FAD2197CA01B9010F94D4469B0137
